:100000000C946A080C9495080C9495080C94950827
:100010000C9495080C9495080C9495080C949508EC
:100020000C9495080C9495080C941F730C9499717A
:100030000C9495080C9495080C9495080C949508CC
:100040000C9495080C94831B0C9495080C949508BB
:100050000C9495080C9495080C94DB230C94BF6CBD
:100060000C9495080C9495080C9495080C9495089C
:100070000C9495080C9495080C9495080C9495088C
:100080000C9495080C9495080C9495080C9495087C
:100090000C9495080C949508084AD73B3BCE016E0A
:1000A00084BCBFFDC12F3D6C74319ABD56833DDACF
:1000B0003D00C77F11BED9E4BB4C3E916BAAAABEDE
:1000C000000000803F05A84CCDB2D44EB93836A907
:1000D000020C50B9918688083CA6AAAA2ABE000044
:1000E00000803F6563686F3A0043616E6E6F7420F5
:1000F000656E746572207375626469723A00457248
:10010000726F723A006572726F72207772697469E9
:100110006E6720746F2066696C65004E6F742053A3
:1001200044207072696E74696E67002F005344201A
:100130007072696E74696E67206279746520002E32
:100140000044656C6574696F6E206661696C6564F6
:100150002C2046696C653A200046696C6520646510
:100160006C657465643A002E006F70656E20666180
:10017000696C65642C2046696C653A200057726989
:1001800074696E6720746F2066696C653A20002E72
:10019000006F70656E206661696C65642C2046692D
:1001A0006C653A20002E006F70656E206661696C88
:1001B00065642C2046696C653A200046696C6520B0
:1001C00073656C6563746564002053697A653A00F1
:1001D00046696C65206F70656E65643A002E006F2D
:1001E00070656E206661696C65642C2046696C657B
:1001F0003A2000776F726B446972206F70656E20D1
:100200006661696C656400776F726B446972206F18
:1002100070656E206661696C65640053442063619B
:100220007264206F6B006F70656E526F6F74206622
:1002300061696C656400766F6C756D652E696E69B9
:1002400074206661696C656400534420696E69744A
:10025000206661696C0024F404D9201BC40C5C0E78
:100260009804C4095F0265077101F405F900FB04F5
:10027000B30048048700C103690058035500030315
:100280004500BE023A008402310053022A002902CE
:10029000250004022000E4011C00C8011900AF0180
:1002A000170098011400840113007101100061010E
:1002B000100051010E0043010D0036010B002B010F
:1002C0000B0020010B00150109000C0109000301BE
:1002D0000800FB000800F3000800EB000700E40042
:1002E0000600DE000600D8000600D2000600CC00A2
:1002F0000500C7000500C2000500BD000400B900EC
:100300000400B5000400B1000400AD000400A90021
:100310000400A5000300A20003009F0004009B004E
:100320000300980003009500020093000300900072
:1003300003008D0002008B0003008800020086008D
:10034000020084000300810002007F0002007D00A3
:1003500002007B00020079000200770001007600B5
:1003600002007400020072000100710002006F00C0
:1003700002006D0001006C0002006A0001006900CB
:1003800002006700010066000100650001006400D2
:1003900002006200010061000100600001005F00D6
:1003A00002005D0001005C0001005B0001005A00DA
:1003B00001005900010058000100570001005600DB
:1003C00001005500010054000100530000005300DB
:1003D00001005200010051000100500001004F00D7
:1003E00001004E0000004E0001004D0001004C00D5
:1003F00001004B0000004B0001004A0001004900D1
:1004000001004800000048000100470001004600CC
:1004100000004600010045000000450001004400C6
:1004200001004300000043000100420000004200C0
:1004300001004100000041000100400001003F00B8
:1004400000003F0001003E0000003E0001003D00B2
:1004500000003D0001003C0000003C0000003C00AA
:1004600001003B0000003B0001003A0000003A00A0
:100470000100390000003900010038000000380098
:10048000000038000100370000003700010036008E
:100490000000360000003600010035000000350085
:1004A000000035000100340000003400000034007A
:1004B000010033000000330000003300010032006F
:1004C0000000320000003200010031000000310065
:1004D000000031000100300000003000000030005A
:1004E00001002F0000002F0000002F0000002F004F
:1004F00001002E0000002E0000002E0001002D0043
:1005000000002D0000002D0000002D0001002C0037
:1005100000002C0000002C0000002C0001002B002B
:1005200000002B0000002B0000002B0001002A001F
:1005300000002A0000002A0000002A000100290013
:100540000000290000002900000029000000290007
:1005500001002800000028000000280000002800FA
:1005600000002800010027000000270000002700ED
:1005700000002700000027000100260000002600E0
:1005800000002600000026000000260001002500D3
:1005900000002500000025000000250000002500C7
:1005A00000002500010024000000240000002400B9
:1005B00000002400000024000100230000002300AC
:1005C000000023000000230000002300000023009F
:1005D0000000230001002200000022000000220091
:1005E0000000220000002200000022000100210083
:1005F0000000210000002100000021000000210077
:100600000000210000002100010020000000200067
:10061000000020000000200000002000000020005A
:10062000000020000000200001001F0000001F004B
:1006300000001F0000001F0000001F0000001F003E
:1006400000001F0001001E0000001E0000001E0030
:1006500000001E00000024F4D43050C38E20C2A23B
:100660004017828B7011127A910D816CD90AA861A2
:10067000E108C7586607615143061E4B5D05C14539
:10068000A7041A411104093D98037139310340361A
:10069000DB0265339102D4305402802E1D02632C9C
:1006A000EE01752AC501B028A001102781018F2510
:1006B00064012B244B01E0223401AC211F018D2069
:1006C0000D01801FFC00841EED00971DDF00B81C8B
:1006D000D200E61BC600201BBC00641AB200B2198F
:1006E000A8000A19A0006A189900D11791004017B4
:1006F0008B00B516840031167E00B31579003A15CB
:100700007300C7146F0058146A00EE136600881354
:10071000630025135E00C7125B006C1257001512B0
:100720005400C111510070114F0021114B00D6101F
:1007300049008D1047004610440002104200C00FCF
:100740004000800F3E00420F3C00060F3B00CB0EE6
:100750003800930E37005C0E3500270E3400F30D81
:100760003200C10D3100900D3000600D2E00320DB1
:100770002D00050D2C00D90C2B00AE0C2900850C8A
:1007800029005C0C2700350C27000E0C2600E80B16
:100790002400C40B2400A00B23007D0B23005A0B64
:1007A0002100390B2100180B2000F80A1F00D90A7C
:1007B0001E00BB0A1E009D0A1D00800A1D00630A60
:1007C0001C00470A1B002C0A1B00110A1A00F7091B
:1007D0001A00DD091900C4091900AB0919009209B2
:1007E00017007B091800630917004C091600360929
:1007F0001600200916000A091500F5081500E00882
:100800001400CC081400B8081400A40814009008C0
:1008100013007D0812006B081300580812004608E8
:1008200012003408110023081100120811000108F9
:100830001100F0071000E0071000D0071000C007FB
:100840001000B0070F00A107100091070E008307EA
:100850000F0074070F0065070E0057070E004907C9
:100860000E003B070D002E070E0020070D0013079A
:100870000D0006070D00F9060C00ED060D00E00660
:100880000C00D4060C00C8060C00BC060C00B00618
:100890000C00A4060B0099060C008D060B008206C6
:1008A0000B0077060B006C060B0061060A0057066A
:1008B0000B004C060A0042060A0038060A002E0603
:1008C0000A0024060A001A060A0010060900070694
:1008D0000A00FD050900F4050900EB050900E20521
:1008E0000900D9050900D0050900C7050900BE05A2
:1008F0000900B5050800AD050800A50509009C051F
:100900000800940508008C050800840508007C0593
:100910000800740508006C050700650508005D0502
:100920000700560508004E0507004705070040056B
:10093000080038050700310507002A0507002305D0
:1009400007001C050600160507000F05070008052F
:10095000060002050700FB040600F5040700EE048C
:100960000600E8040600E2040700DB040600D504E4
:100970000600CF040600C9040600C3040600BD0437
:100980000600B7040600B1040500AC040600A60486
:100990000600A00405009B040600950405009004D1
:1009A00006008A04050085040500800406007A0418
:1009B000050075040500700405006B04050066045D
:1009C0000500610405005C0405005704050052049D
:1009D00005004D04050048040500430405003E04DD
:1009E00004003A04050035040500300404002C041A
:1009F000050027040400230405001E0404001A0453
:100A0000040016040500110404000D040400090488
:100A100005000404040000040400FC030400F803BF
:100A20000400F4030400F0030400EC030400E803F2
:100A30000400E4030400E0030400DC030400D80322
:100A40000400D4030400D0030400CC030400C80352
:100A50000300C50303006563686F3A00205A3A003B
:100A600020593A0020583A00656E6473746F7073B1
:100A7000206869743A20004572726F723A005465BA
:100A80006D70657261747572652068656174656406
:100A900020626564207377697463686564206F669B
:100AA000662E204D415854454D5020747269676739
:100AB00065726564202121003A204578747275645E
:100AC0006572207377697463686564206F66662E4B
:100AD000204D494E54454D502074726967676572C8
:100AE00065642021003A204578747275646572202F
:100AF0007377697463686564206F66662E204D4164
:100B00005854454D5020747269676765726564205A
:100B10003A292100202D20496E76616C6964206598
:100B200078747275646572206E756D6265722021CD
:100B300000202D20496E76616C696420657874729E
:100B400075646572206E756D626572210020403A91
:100B5000006F6B20543A00504944204175746F7403
:100B6000756E65206661696C656420212C20546572
:100B70006D706572617475726520746F2068696745
:100B80006800204B643A2000204B693A2000204B3B
:100B9000703A2000204E6F206F76657273686F6F19
:100BA000742000204B643A2000204B693A2000203A
:100BB0004B703A200020536F6D65206F766572731D
:100BC000686F6F742000204B643A2000204B693A14
:100BD0002000204B703A200020436C617369632031
:100BE00050494420002054753A2000204B753A208B
:100BF00000206D61783A2000206D696E3A20002057
:100C0000643A200020626961733A20004572726F75
:100C1000723A005072696E7465722068616C746516
:100C2000642E206B696C6C28292063616C6C656490
:100C3000202121006F6B00526573656E643A006578
:100C400063686F3A002200556E6B6E6F776E20639B
:100C50006F6D6D616E643A22007A5F6D696E3A0065
:100C6000795F6D696E3A00785F6D696E3A005A3A45
:100C700000593A0020436F756E7420583A00453A87
:100C8000005A3A00593A00583A004649524D5741E5
:100C900052455F4E414D453A4D61726C696E20562A
:100CA000313B20537072696E7465722F6772626C8B
:100CB000206D617368757020666F722067656E368F
:100CC000202853657020313220323031322F3233B8
:100CD0003A35393A343129204649524D5741524527
:100CE0005F55524C3A687474703A2F2F7777772E8D
:100CF0006D656E64656C2D70617274732E636F6DBB
:100D00002050524F544F434F4C5F56455253494F1A
:100D10004E3A312E30204D414348494E455F54599B
:100D200050453A4D656E64656C20455854525544A3
:100D300045525F434F554E543A310A0020423A0023
:100D400020453A00543A0020573A0020453A0054D2
:100D50003A0020403A0020423A006F6B20543A009B
:100D6000456E642066696C65206C69737400426529
:100D700067696E2066696C65206C69737400446FE6
:100D80006E65207072696E74696E672066696C6545
:100D9000006F6B004E6F204C696E65204E756D6262
:100DA0006572207769746820636865636B73756D1D
:100DB0002C204C617374204C696E653A004E6F2094
:100DC000436865636B73756D2077697468206C691F
:100DD0006E65206E756D6265722C204C6173742097
:100DE0004C696E653A00636865636B73756D206D61
:100DF00069736D617463682C204C617374204C6955
:100E00006E653A004C696E65204E756D62657220A4
:100E10006973206E6F74204C617374204C696E6529
:100E2000204E756D6265722B312C204C61737420DD
:100E30004C696E653A00446F6E6520736176696E29
:100E4000672066696C652E006F6B002020506C6116
:100E50006E6E657242756666657242797465733A44
:100E600020002046726565204D656D6F72793A20CD
:100E7000006572696B00207C20417574686F723A5E
:100E80002000323031322D30322D323500204C618D
:100E9000737420557064617465643A2000312E309B
:100EA0002E3020524332004D61726C696E3A200040
:100EB00020536F66747761726520526573657400A4
:100EC000205761746368646F6720526573657400AE
:100ED0002042726F776E206F75742052657365744F
:100EE000002045787465726E616C2052657365747C
:100EF00000506F77657255700073746172740022D0
:100F000000656E717565696E672022007C3C3E5EEF
:100F10002B3D3F2F5B5D3B2C2A225C006563686F95
:100F20003A0020746F6F206C6F6E67206578747262
:100F30007573696F6E2070726576656E7465640096
:100F400020636F6C6420657874727573696F6E20AE
:100F500070726576656E7465640001290229042942
:100F600008291029202940298029012C022C01263A
:100F70000226042608261026202640268026402CFD
:100F8000802C012302230423082310232023402341
:100F9000802301200220042008201020202040204F
:100FA0008020102C202C012F022F042F082F102F0F
:100FB000202F402F802F7EFE7EFD7EFB7EF77EEF72
:100FC0007EDF7EBF7E7F00010000FA0F120002006C
:100FD000000C1043000300004F10040103090453E8
:100FE0001018020309046D10160303090485100C80
:100FF0000001C102018036018136120100020200A7
:101000000020C0168304000101020301090243000D
:10101000020100C03209040000010202010005249F
:101020000010010524010001042402060524060025
:10103000010705820308004009040100020A0000BC
:101040000007050302400000070584024000000479
:1010500003090418035400650065006E00730079ED
:10106000006400750069006E006F000000160355F3
:1010700000530042002000530065007200690061C7
:10108000006C0000000C03310032003300340035E6
:10109000000000494E46494E4954594E414ECDCC70
:1010A000CC3D0AD7233C17B7D13877CC2B32959556
:1010B000E6241FB14F0A000020410000C842004052
:1010C0001C4620BCBE4CCA1B0E5AAEC59D74EB35E7
:1010D0006B6FE63511241FBECFEFD0E2DEBFCDBF70
:1010E00012E0A0E0B1E0E0E1F2EF00E00BBF02C0EF
:1010F00007900D92AC3DB107D9F71BBE1DE0ACEDDA
:10110000B2E001C01D92A93BB107E1F710E1C2EDC9
:10111000D0E104C02297FE010E94AE78CE3CD107F8
:10112000C9F70E94DB6F0C94FC780C940000A0E0DF
:10113000B0E0EDE9F8E00C94CB78EC015B016115CF
:10114000710519F0FB0191838083F9908F2D90E058
:101150000E94B278892BC9F7FDE2FF1621F4F990BD
:10116000EE24E39405C02BE2F21609F4F990EE2484
:101170008E0101501040C80163E970E143E050E086
:1011800062D2892BF9F48E010E5F1F4FC80166E908
:1011900070E145E050E057D2892B19F48E01095FC8
:1011A0001F4FA114B10419F0F50111830083E0FC75
:1011B00004C070E090E080E813C070E090E080E848
:1011C0006FEF07C1C8016BE970E143E050E03BD22B
:1011D000892B69F4A114B10429F470E090E080EC4B
:1011E0006FE7F7C02296F501D183C083F6CF88243C
:1011F000992440E050E060E070E0EF2DE053EA30E9
:10120000A0F5F2E0EF2A8E2D90E09C01287030705E
:10121000E2FE06C0232B79F50894811C911C2BC09B
:10122000232B19F0089481089108DB01CA0112E010
:10123000880F991FAA1FBB1F1A95D1F7480F591F76
:101240006A1F7B1F440F551F661F771F4E0F511DCE
:10125000611D711D483929E9520729E9620729E111
:10126000720748F084E0E82A06C0EE3F31F4E3FC60
:1012700039C098E0E92AF990C0CFE53311F0E531A3
:1012800089F529912D3219F4E0E1EE2A05C02B32BF
:1012900019F081E090E003C0299182E090E0E22F14
:1012A000E053EA3018F0C81BD90B1CC020E030E036
:1012B000FCE020383F075CF4C901880F991F880FB4
:1012C000991F280F391F220F331F2E0F311DE9914F
:1012D000E053EA3068F3E4FE03C0309521953F4FB8
:1012E000820E931ECE2CDD24E1FE07C0A114B104B2
:1012F00021F02197F501D183C083CB01BA010E946F
:1013000017757B018C01F3E0CF22DD2423E0C216A8
:10131000D10421F417FB109517F9109557016801B6
:10132000C801B70120E030E040E050E00E9477744F
:10133000882309F44AC097FE0DC022EBE22E20E17B
:10134000F22E9094819491089394C0E2D0E000E052
:1013500010E012C09AECE92E90E1F92EF6CFF701D9
:101360002591359145915491C601B5010E94577759
:101370005B016C018C1A9D0A8C169D0684F7D5952D
:10138000C7950F5F1F4F0630110529F08CEF9FEFB7
:10139000E80EF91EF1CFC501D6017C018D018C2D1F
:1013A000880F8D2D881F8F3F51F0C601B50120E0B9
:1013B00030E040E050E00E947774882331F482E20C
:1013C00090E09093B80D8093B70D7E2D9F2D802FC8
:1013D000612F272F392F482F562FB901CA01CDB7BA
:1013E000DEB7ECE00C94E7782F923F925F926F9219
:1013F0007F928F929F92AF92BF92CF92DF92EF92A5
:10140000FF920F931F93CF93DF938C011B01EA018F
:101410006115710519F0FB0191838083209749F0D4
:10142000CE010297839728F020E030E040E050E0C2
:10143000F6C0F801A1908F018A2D90E00E94B27849
:10144000892BB9F7FDE2AF1631F4F801A1908F01B5
:101450005524539407C0FBE2AF1619F4F801A1908C
:101460008F015524209719F0C031D105C1F4F0E364
:10147000AF1679F4F8018081883711F0883549F486
:10148000F801A1800E5F1F4FF2E05F2AC0E1D0E0BB
:1014900006C0209721F480E3A816E9F427C0C830DD
:1014A000D10531F1C930D10524F4C230D10531F56F
:1014B0000CC0CA30D10589F0C031D105F9F4C12C76
:1014C000D12CE12CB8E0FB2E28C0C12CD12CE12C72
:1014D000A0E4FA2E22C0CAE0D0E0FCECCF2EFCEC57
:1014E000DF2EFCECEF2EFCE0FF2E17C0C8E0D0E0B2
:1014F000C12CD12CE12CE0E1FE2E0FC09E0144272F
:1015000037FD4095542F60E070E080E090E80E9445
:101510005B78C901DA016C017D0120E030E040E038
:1015200050E060E03E01882477FC8094982C70EDB8
:10153000B72EBA0CE9E0EB1570F48A2D81548A318C
:1015400018F499ECB92E06C08A2D81568A3150F5CF
:1015500089EAB82EBA0C8B2D90E08C179D0714F5F4
:101560006F3FE1F0C216D306E406F506B0F0CA01FB
:10157000B901A40193010E9429789B01AC012B0DB4
:10158000311D411D511D2130F0E03F07F0E04F07B4
:10159000F0E85F0710F461E001C06FEFF801A1907F
:1015A0008F01C5CF2114310481F0662331F0015041
:1015B0001040F1011183008308C051FE1AC002508F
:1015C0001040F1011183008314C067FF12C050FC6A
:1015D00005C02FEF3FEF4FEF5FE704C020E030E0A2
:1015E00040E050E882E290E09093B80D8093B70D10
:1015F00016C050FE08C050954095309521953F4F3C
:101600004F4F5F4F0CC057FF0AC082E290E09093AB
:10161000B80D8093B70D2FEF3FEF4FEF5FE7B901A4
:10162000CA01DF91CF911F910F91FF90EF90DF9052
:10163000CF90BF90AF909F908F907F906F905F9072
:101640003F902F900895FB01DC014150504088F0FD
:101650008D9181341CF08B350CF4805E6591613482
:101660001CF06B350CF4605E861B611171F3990BF5
:101670000895881BFCCFFB01DC0104C08D91019013
:10168000801921F441505040C8F7881B990B0895E8
:10169000FB01DC0102C001900D9241505040D8F78F
:1016A0000895FB01DC010D900020E9F711970190EE
:1016B0000D920020E1F70895FC018191861721F039
:1016C0008823D9F7992708953197CF010895FB0111
:1016D000DC0101900D920020E1F70895FB01DC018F
:1016E0004150504030F08D910190801919F4002044
:1016F000B9F7881B990B0895FB01DC01415050405C
:1017000048F001900D920020C9F701C01D92415090
:101710005040E0F70895FB0151915523A9F0BF0116
:10172000DC014D9145174111E1F759F4CD010190CC
:10173000002049F04D9140154111C9F3FB014111C1
:10174000EFCF81E090E001970895AEE0B0E0EBEAE2
:10175000FBE00C94D3780D891E8986E08C831A8374
:1017600009838FEF9FE79E838D839E01275E3F4F06
:10177000CE0101966F89788DA9010AD02F81388515
:10178000020F131FF80110822E96E4E00C94EF78FC
:10179000ABE0B0E0EEECFBE00C94C5783C012B0133
:1017A0005A01FC0117821682838181FD03C06FEF0D
:1017B0007FEFB9C19AE0892E1E010894211C311CCB
:1017C000F3012381F20123FD859123FF81912F01F4
:1017D000882309F4A5C1853239F423FD859123FFBF
:1017E00081912F01853221F490E0B301B7D1E8CF88
:1017F000982FFF24EE249924FFE1FF15D0F09B32AF
:1018000069F09C3228F4903259F0933291F40EC072
:101810009D3249F0903369F441E024C052E0F52A4A
:1018200084E0F82A28C098E0F92A25C0E0E1FE2AE1
:1018300022C0F7FC29C0892F80538A3070F4F6FE4D
:1018400005C0989C902C1124980E15C0E89CE02CA3
:101850001124E80EF0E2FF2A0EC09E3229F4F6FCB5
:101860005FC140E4F42A07C09C3619F450E8F52A19
:1018700002C0983649F4F20123FD959123FF91911E
:101880002F01992309F0B8CF892F8554833018F0A0
:101890008052833038F444E050E0A40EB51E5FE37C
:1018A00059830FC0933631F0933779F0933509F0AF
:1018B00052C01FC0F5018081898342E050E0A40E30
:1018C000B51E610101E010E011C0F501C080D180BA
:1018D000F6FC03C06FEF7FEF02C0692D70E042E0BD
:1018E00050E0A40EB51EC6012ED18C015FE7F52293
:1018F00013C0F501C080D180F6FC03C06FEF7FEF0D
:1019000002C0692D70E042E050E0A40EB51EC60191
:101910000FD18C0150E8F52AF3FE06C018C080E212
:1019200090E0B3011BD1EA948E2D90E008171907BF
:10193000B0F30DC0F601F7FC8591F7FE81916F01C0
:1019400090E0B3010BD1E110EA9401501040011571
:10195000110581F7E2C0943611F0993661F5F7FE72
:1019600008C0F501208131814281538184E090E0FB
:101970000AC0F501808191819C01442737FD409583
:10198000542F82E090E0A80EB91E9FE6F92257FF7F
:1019900009C050954095309521953F4F4F4F5F4F6F
:1019A000E0E8FE2ACA01B901A1012AE030E002D133
:1019B000D82ED2183FC0953729F41F2D1F7E2AE05C
:1019C00030E01DC01F2D197F9F3661F0903720F445
:1019D000983509F0A5C00FC0903739F0983709F055
:1019E0009FC004C028E030E00AC0106114FD1460FC
:1019F00020E130E004C014FD166020E132E017FF62
:101A000008C0F501608171818281938144E050E0DA
:101A100008C0F50180819181BC0180E090E042E046
:101A200050E0A40EB51EA101C5D0D82ED2188FE764
:101A3000F82EF122F6FE0BC05EEFF522D91438F431
:101A4000F4FE07C0F2FC05C08FEEF82202C01D2D87
:101A500001C0192DF4FE0DC0FE01ED0DF11D8081B8
:101A6000803319F499EEF92208C01F5FF2FE05C019
:101A700003C08F2D867809F01F5F0F2DF3FC13C074
:101A8000F0FE0EC01E1510F09D2C0AC09D2C9E0C61
:101A9000911A1E2D05C080E290E0B3015FD01F5F58
:101AA0001E15C8F304C01E1510F4E11A01C0EE247F
:101AB00004FF0EC080E390E0B30150D002FF1BC0D2
:101AC00001FD03C088E790E00EC088E590E00BC000
:101AD000802F867881F001FF02C08BE201C080E296
:101AE000F7FC8DE290E0B30139D005C080E390E0CF
:101AF000B30134D09A94D914C8F3DA94F101ED0DFE
:101B0000F11D808190E0B30129D0DD20B1F705C03F
:101B100080E290E0B30122D0EA94EE20C9F750CEE3
:101B2000F30166817781CB012B96E2E10C94E17899
:101B3000FC010590615070400110D8F78095909598
:101B40008E0F9F1F0895FC0161507040019001109D
:101B5000D8F7809590958E0F9F1F08950F931F9330
:101B6000CF93DF938C01EB018B8181FF1BC082FF40
:101B70000DC02E813F818C819D812817390764F427
:101B8000E881F9810193F983E88306C0E885F98546
:101B9000802F0995892B31F48E819F8101969F8337
:101BA0008E8302C00FEF1FEFC801DF91CF911F910D
:101BB0000F910895FA01AA27283051F1203181F1BF
:101BC000E8946F936E7F6E5F7F4F8F4F9F4FAF4F45
:101BD000B1E03ED0B4E03CD0670F781F891F9A1F58
:101BE000A11D680F791F8A1F911DA11D6A0F711D0C
:101BF000811D911DA11D20D009F468943F912AE018
:101C0000269F11243019305D3193DEF6CF010895FF
:101C1000462F4770405D4193B3E00FD0C9F7F6CF30
:101C2000462F4F70405D4A3318F0495D31FD4052F8
:101C3000419302D0A9F7EACFB4E0A695979587958E
:101C400077956795BA95C9F700976105710508956D
:101C50009B01AC010A2E0694579547953795279519
:101C6000BA95C9F7620F731F841F951FA01D0895B1
:101C70002F923F924F925F926F927F928F929F929C
:101C8000AF92BF92CF92DF92EF92FF920F931F938A
:101C9000DF93CF93CDB7DEB7CD55D0400FB6F894D4
:101CA000DEBF0FBECDBF2F969FAF8EAF2F97619631
:101CB0007FAF6EAF61972A0162962FAF62976396EE
:101CC0000FAF63976496EFAE64976896ACAEBDAE07
:101CD000CEAEDFAE6897E22EFF24EE0CFF1CEE0CBA
:101CE000FF1C9A012E0D3F1D2D963FAF2EAF2D9755
:101CF000D9016D907D908D909C90FC01EE0DFF1DA3
:101D0000C401B30120813181428153810E949E73BD
:101D100069AF7AAF8BAF9CAF10E0000F111F000FBF
:101D2000111FF201E00FF11F2B96FFAFEEAF2B97C3
:101D3000A080B180C280D3802F96EEADFFAD2F97EB
:101D4000E00FF11FC601B50120813181428153812D
:101D50000E949E736DAB7EAB8FAB98AF64962FAD38
:101D60006497E22FF0E0EE0FFF1FEE0FFF1F2F969C
:101D7000AEADBFAD2F97AE0FBF1F4D915D916D9171
:101D80007C9129964CAF5DAF6EAF7FAF299761967E
:101D90006EAD7FAD6197E60FF71F60817181828123
:101DA000938129962CAD3DAD4EAD5FAD29970E9434
:101DB0009D7369AB7AAB8BAB9CAB6196AEADBFAD9F
:101DC00061971C968D919D910D90BC91A02D2596AB
:101DD0008CAF9DAFAEAFBFAF25972F96AEADBFAD69
:101DE0002F971C962D913D914D915C911F972196B7
:101DF0002CAF3DAF4EAF5FAF2197A4019301505878
:101E00002DA73EA74FA758ABB601A501705849A70B
:101E10005AA76BA77CA761966EAD7FAD6197E60E62
:101E2000F71ED7016D917D918D919C9129AD3AADB1
:101E30004BAD5CAD0E949D733B014C016196EEADD4
:101E4000FFAD61970E0F1F1FD8016D917D918D9190
:101E50009C912DA93EA94FA958AD0E949D735B018D
:101E60006C016DA57EA58FA598A9A60195010E947C
:101E700057777B018C0169A57AA58BA59CA5A40148
:101E800093010E9457779B01AC01C801B7010E94E2
:101E90009D731B012C016DA57EA58FA598A9A4019A
:101EA00093010E9457777B018C0169A57AA58BA5C8
:101EB0009CA5A60195010E9457779B01AC01C80122
:101EC000B7010E949E739B01AC01C201B1010E9447
:101ED00011745B016C0120E030E040E050E00E94B2
:101EE0007774882354F4C601B5012BED3FE049EC2B
:101EF00050E40E949E735B016C01E7968FADE797FB
:101F0000882351F0C601B5012BED3FE049EC50E4C8
:101F10000E949D735B016C01C601B501E6962CAD74
:101F20003DAD4EAD5FADE6970E94577729A93AA91E
:101F30004BA95CA95F770E9492767B018C012FE60A
:101F400032E143E85AE30E94777487FD5FC2C8011B
:101F5000B7010E9454750E94EB7478A76FA380E0CC
:101F600090E00E9417757B018C01C601B501A801A4
:101F700097010E947E746BA37CA38DA39EA369A985
:101F80007AA98BA99CA9A80197010E947E746F8FE2
:101F900078A389A39AA325966CAD7DAD8EAD9FAD38
:101FA000259721962CAD3DAD4EAD5FAD21970E949A
:101FB0009D73A80197010E947E746B8F7C8F8D8F1B
:101FC0009E8F6BA17CA18DA19EA120E030E040E01E
:101FD0005FEB0E9457772BA13CA14DA15EA10E940F
:101FE000577720E030E040E85FE30E949E736F8BFC
:101FF000788F898F9A8F64962FAD6497E22FF0E0E7
:10200000EE0FFF1FEE0FFF1F9E012F5F3F4FE20FEE
:10201000F31F29964CAD5DAD6EAD7FAD2997408322
:102020005183628373832F96AEADBFAD2F971C96FD
:102030004D915D916D917C911F974D875E876F8764
:10204000788B41E050E05A8B498B662462967FADD5
:102050006297672F70E0660F771F660F771FC901C1
:10206000860F971F6A969FAF8EAF6A976396BFAD34
:102070006397AB2FB0E0AA0FBB1FAA0FBB1F21E0D5
:1020800030E02C0F3D1F2A0F3B1F6C963FAF2EAF49
:102090006C976E96FFAFEEAF6E9790C138E1361534
:1020A0000CF446C06DA57EA58FA598A92BA13CA1D7
:1020B0004DA15EA10E9457777B018C0169A57AA58D
:1020C0008BA59CA52F89388D498D5A8D0E945777F5
:1020D0009B01AC01C801B7010E949E737B018C017A
:1020E0006DA57EA58FA598A92F89388D498D5A8D0C
:1020F0000E9457775B016C0169A57AA58BA59CA509
:102100002BA13CA14DA15EA10E9457779B01AC0180
:10211000C601B5010E949D736DA77EA78FA798ABDE
:102120006394C701D80189A79AA7ABA7BCA765C0CC
:1021300049895A89BA0180E090E00E9417752BA165
:102140003CA14DA15EA10E9457777B018C01C80183
:102150000E947B746B8B7C8B8D8B9E8BB701C8012F
:102160000E94BA773B014C012D96AEADBFAD2D97C5
:10217000ED90FD900D911C9117FB109517F910959E
:102180002B96EEADFFAD2B9720803180428053809F
:10219000C801B7012B893C894D895E890E94577718
:1021A0005B016C01C201B101A40193010E94577748
:1021B0009B01AC01C601B5010E949E736DA77EA76D
:1021C0008FA798ABC801B701A40193010E9457776C
:1021D0007B018C01C201B1012B893C894D895E894B
:1021E0000E9457779B01AC01C801B7010E949D7303
:1021F00069A77AA78BA79CA7662469AD7AAD8BAD3A
:102200009CAD2DA53EA54FA558A90E949E736A9628
:10221000AEADBFAD6A976D937D938D939C931397ED
:102220006DA97EA98FA998AD29A53AA54BA55CA556
:102230000E949E736C96EEADFFAD6C9760837183C8
:10224000828393836E96AEADBFAD6E976D917D9197
:102250008D919C912F8D38A149A15AA10E949E7306
:102260006E96EEADFFAD6E9760837183828393832C
:10227000ED84FE840F85188969817A818B819C8128
:1022800020E030E040E050E00E947774882344F47E
:1022900080E090E0A0E0B0E089839A83AB83BC83C8
:1022A0006D817E818F81988520E030E040E050E0B4
:1022B0000E947774882344F480E090E0A0E0B0E0CE
:1022C0008D839E83AF83B88769857A858B859C854E
:1022D00020E030E040E050E00E947774882344F42E
:1022E00080E090E0A0E0B0E089879A87AB87BC8768
:1022F00069817A818B819C8120E030E044EC52E45A
:102300000E948576181644F480E090E0A4ECB2E4D4
:1023100089839A83AB83BC836D817E818F8198850D
:1023200020E030E04EEB52E40E948576181644F42B
:1023300080E090E0AEEBB2E48D839E83AF83B887FC
:1023400069857A858B859C8520E030E040EF52E4FA
:102350000E948576181644F480E090E0A0EFB2E485
:1023600089879A87AB87BC87C801B7012B8D3C8DC5
:102370004D8D5E8D0E949E736D877E878F87988BB3
:10238000CE010196BE016B5F7F4FAE01475F5F4F8D
:102390009E01235F3F4F6896ECACFDAC0EAD1FADC8
:1023A0006897F7E7CF2ED12CCC0EDD1E0E940E5F72
:1023B00029893A892F5F3F4F3A8B298B49895A895E
:1023C0006FA178A54617570708F468CE61964EAD01
:1023D0005FAD6197485F5F4F61962EAD3FAD6197EE
:1023E000245F3F4F61968EAD9FAD6197DC011496DF
:1023F000BD016896ECACFDAC0EAD1FAD6897E7E78C
:10240000CE2ED12CCC0EDD1E0E940E5FC35ADF4FA4
:102410000FB6F894DEBF0FBECDBFCF91DF911F91F5
:102420000F91FF90EF90DF90CF90BF90AF909F9073
:102430008F907F906F905F904F903F902F90089576
:10244000DF93CF930F92CDB7DEB7FC016983A081F4
:10245000B18112962D913C911397BE016F5F7F4F12
:1024600041E050E0F90109950F90CF91DF91089577
:10247000FC01148A178A138A28EC32E0328B218BF4
:1024800014AA17AA13AA32AB21ABEE5AFF4F10823F
:10249000339610823497108232932293B196108231
:1024A0003396108234971082329322937F9689E17B
:1024B000808333961082789610823A9610823396F3
:1024C000108234971082329322937E96108211826A
:1024D0001282138238961082118212821382E45D76
:1024E000F040118212821082E852FF4F81E0808317
:1024F000E85DF040108A17860FB6F8948091A40D1D
:102500009091A50DA091A60DB091A70D0FBEE0531F
:10251000FF4F88579C4EAF4FBF4F80839183A2835C
:10252000B3830895FC01118212820895FC01828117
:10253000882311F081E081830895FC01818181115C
:10254000118208950F931F938C010E94701B0E94AB
:102550004D1BF801118280E091E00E944C501F91C8
:102560000F910895CF93DF93DB010D900020E9F7E1
:102570001197A61BB70BEC01E881F9810280F3816A
:10258000E02DAD010995DF91CF910895FC0188EC14
:1025900092E0918380838681882321F0CF01039686
:1025A0000C9428520895EF92FF920F931F937C0191
:1025B0008C010F541F4FC8010E94DB51C8010E94BB
:1025C0002852F70110821F910F91FF90EF9008950C
:1025D000CF92DF92EF92FF920F931F93CF93DF93EF
:1025E0007C016B01DB010D900020E9F78D010150AA
:1025F0001040061B170BE1EBF0E0EE0EFF1ED701BB
:102600001C92EFE4FFEFEE0EFF1ECB016EE470E0D4
:1026100053D8EC01009731F4F8013197EC0DFD1D12
:1026200086010CC060E270E047D88C010F5F1F4F3D
:10263000CE016AE270E040D8FC0131978DE08183E1
:102640008AE082831382C70182559F4FB8010E949E
:10265000586B81EB90E0E80EF91ED7018C9188232E
:10266000F1F0EEEFF0E06491EF0106C089EA9DE041
:10267000E7DE2196FE0164916623C1F7E5E0F1E013
:102680006491EF0106C089EA9DE0DADE2196FE0141
:1026900064916623C1F789EA9DE06AE0D1DEDF91AB
:1026A000CF911F910F91FF90EF90DF90CF90089501
:1026B000EF92FF920F93CF93DF937C01FC01828115
:1026C000882309F43DC0EDE2F1E06491EF0106C01A
:1026D00089EA9DE0B5DE2196FE0164916623C1F78B
:1026E00084ED90E0E80EF91EF7014081518162818E
:1026F00073818CE29FEFE80EF91E89EA9DE02AE0E3
:1027000000E00E942770EBE2F1E06491EF0106C067
:1027100089EA9DE095DE2196FE0164916623C1F76A
:102720008CEC90E0E80EF91EF70140815181628146
:10273000738189EA9DE02AE000E00E9427700DC0C5
:10274000EBE1F1E06491EF0106C089EA9DE078DEFB
:102750002196FE0164916623C1F789EA9DE06AE053
:102760006FDEDF91CF910F91FF90EF9008952F9240
:102770003F924F925F926F927F928F929F92AF9211
:10278000BF92CF92DF92EF92FF920F931F93DF934E
:10279000CF93CDB7DEB7AC970FB6F894DEBF0FBEC0
:1027A000CDBF5C014B014CA7FC018281882309F459
:1027B00090C131EB432E512C4A0C5B1CC2010E948C
:1027C0002852F5011182198A1C8A188A88EC92E035
:1027D0009F878E87C501419690AB87A7F4018081C2
:1027E0008F3209F07BC0C4016FE270E00E945C0B85
:1027F0007C010894E11CF11C3E010894611C711CD1
:1028000021E1222E312C2C0E3D1E63C0C7016FE248
:1028100070E00E945C0B6C01009709F467C0E81639
:10282000F90608F063C08C010E191F09C301B70136
:10283000A8010E947C0B060D171DF801108289EA81
:102840009DE0B3018FDE89EA9DE06AE0F9DDF501E4
:1028500067A570A96115710519F460E070E002C008
:102860006D5F7F4FC101A30121E00E94AA58882318
:1028700029F5EFEDF1E064917F0108C089EA9DE060
:10288000DFDD0894E11CF11CF70164916623B1F7C8
:1028900089EA9DE0BE016F5F7F4F64DEEDEDF1E000
:1028A00064917F0108C089EA9DE0CADD0894E11CBB
:1028B000F11CF70164916623B1F704C12EE030E00A
:1028C0002C0F3D1FF50130AB27A776010894E11CC2
:1028D000F11CE114F10409F099CF05C0C501C196BE
:1028E000F50190AB87A7082DD92C02C00E2DDF2C47
:1028F000F50167A570A9FCA5FF2309F499C061152E
:10290000710519F460E070E002C06D5F7F4FC20195
:10291000402F5D2D21E00E94AA58882309F464C04D
:10292000A50144535F4F22EC30E0A20EB31EF50127
:1029300080819181A281B3812EE33FEFA20EB31E6D
:10294000FA0180839183A283B383E0EDF1E0649187
:102950007F0108C089EA9DE073DD0894E11CF11C49
:10296000F70164916623B1F789EA9DE0602F7D2D20
:10297000F9DDE9ECF1E064917F0108C089EA9DE0AE
:102980005FDD0894E11CF11CF70164916623B1F747
:102990002CEC30E0A20EB31EF50140815181628122
:1029A000738189EA9DE02AE000E00E94277089EAAD
:1029B0009DE06AE045DD28E030E0A20EB31EF5019F
:1029C0001082118212821382EBEBF1E064917F019D
:1029D00008C089EA9DE034DD0894E11CF11CF70190
:1029E00064916623B1F76EC0E7EAF1E064917F017C
:1029F00008C089EA9DE024DD0894E11CF11CF70180
:102A000064916623B1F789EA9DE0602F7D2DAADDF0
:102A1000E5EAF1E064917F0108C089EA9DE010DDFC
:102A20000894E11CF11CF70164916623B1F74AC0D8
:102A30006115710519F460E070E002C06D5F7F4FB1
:102A4000C201402F5D2D26E50E94AA58882321F55A
:102A5000E1E9F1E064917F0108C089EA9DE0F0DCE2
:102A60000894E11CF11CF70164916623B1F789EA2F
:102A70009DE0602F7D2D76DDEFE8F1E064917F0130
:102A800008C089EA9DE0DCDC0894E11CF11CF70138
:102A900064916623B1F716C081E0F5018083EDE70C
:102AA000F1E064917F0108C089EA9DE0C9DC0894E7
:102AB000E11CF11CF70164916623B1F789EA9DE0FE
:102AC000B40150DD89EA9DE06AE0BADCCE010E96E1
:102AD0005DDDAC960FB6F894DEBF0FBECDBFCF91D3
:102AE000DF911F910F91FF90EF90DF90CF90BF90FB
:102AF000AF909F908F907F906F905F904F903F909E
:102B00002F9008952F923F924F925F926F927F92F3
:102B10008F929F92AF92BF92CF92DF92EF92FF92ED
:102B20000F931F93DF93CF93CDB7DEB7AB970FB65D
:102B3000F894DEBF0FBECDBF5C014B01FC0182816A
:102B4000882309F4F4C0C5018F549F4F0E94285276
:102B5000F5011182198A1C8A188A88EC92E09F87F5
:102B60008E87C501419690AB87A7F40180818F3293
:102B700009F07CC0C4016FE270E00E945C0B7C0134
:102B80000894E11CF11C3E010894611C711C5EE07C
:102B9000252E312C2C0E3D1E41E1442E512C4C0E85
:102BA0005D1E5FC0C7016FE270E00E945C0B6C01AC
:102BB000009709F463C0E816F90608F05FC08C01BD
:102BC0000E191F09C301B701A8010E947C0B060D55
:102BD000171DF801108289EA9DE0B301C3DC89EA80
:102BE0009DE06AE02DDCF50167A570A9611571050E
:102BF00019F460E070E002C06D5F7F4FC201A30175
:102C000021E00E94AA58882329F5E9E6F1E06491C1
:102C10007F0108C089EA9DE013DC0894E11CF11CE7
:102C2000F70164916623B1F789EA9DE0BE016F5F09
:102C30007F4F98DCE7E6F1E064917F0108C089EA04
:102C40009DE0FEDB0894E11CF11CF7016491662312
:102C5000B1F766C0F50130AA27A676010894E11CF9
:102C6000F11CE114F10409F09DCF05C0C501C19626
:102C7000F50190AB87A7D82C092D02C0DE2C0F2DB3
:102C8000F50187A590A9009719F480E090E001C0B4
:102C900003966D2D702F0E9476598823F1F0E9E597
:102CA000F1E064917F0108C089EA9DE0C9DB0894E6
:102CB000E11CF11CF70164916623B1F789EA9DE0FC
:102CC0006D2D702F4FDC84ED90E0A80EB91EF5013C
:102CD000108211821282138227C0E1E4F1E0649134
:102CE0007F0108C089EA9DE0ABDB0894E11CF11C80
:102CF000F70164916623B1F789EA9DE06D2D702F8D
:102D000031DCEFE3F1E064917F0108C089EA9DE0E6
:102D100097DB0894E11CF11CF70164916623B1F77D
:102D200089EA9DE06AE08CDBCE010E962FDCAB9643
:102D30000FB6F894DEBF0FBECDBFCF91DF911F91CC
:102D40000F91FF90EF90DF90CF90BF90AF909F904A
:102D50008F907F906F905F904F903F902F9008954D
:102D6000EF92FF920F931F93CF93DF937C01FC01AF
:102D700012828789882321F0C70144960E94285235
:102D8000870105571F4FC80160E04AE10E94843463
:102D90008823D9F4E3EEF0E06491EF0106C089EAFC
:102DA0009DE04EDB2196FE0164916623C1F7E9E4C4
:102DB000F2E06491EF0106C089EA9DE041DB2196D3
:102DC000FE0164916623C1F76BC0E701C057DF4F76
:102DD000CE01B80141E00E945E2E882311F5CE019C
:102DE000B80140E00E945E2E8823D9F4EEEFF0E0B7
:102DF0006491EF0106C089EA9DE022DB2196FE0185
:102E000064916623C1F7E6E3F2E06491EF0106C046
:102E100089EA9DE015DB2196FE0164916623C1F7E6
:102E20003FC0C7014496BE010E94A8548823D9F42C
:102E3000EEEFF0E06491EF0106C089EA9DE000DB6F
:102E40002196FE0164916623C1F7E6E2F2E0649107
:102E5000EF0106C089EA9DE0F3DA2196FE01649154
:102E60006623C1F71DC081E0F7018283E3EEF0E045
:102E70006491EF0106C089EA9DE0E2DA2196FE0145
:102E800064916623C1F7EBE1F2E06491EF0106C0C3
:102E900089EA9DE0D5DA2196FE0164916623C1F7A7
:102EA00089EA9DE06AE0CCDAC7014196F70190AB70
:102EB00087A7C701C49620E930E0E20EF31EB701F0
:102EC0000E94A854882389F4E7E0F2E06491EF01BE
:102ED00006C089EA9DE0B4DA2196FE01649166237A
:102EE000C1F789EA9DE06AE0ABDADF91CF911F91EB
:102EF0000F91FF90EF9008952F923F924F925F9223
:102F00007F928F929F92AF92BF92CF92DF92EF9279
:102F1000FF920F931F93DF93CF93CDB7DEB7CC55BE
:102F2000D0400FB6F894DEBF0FBECDBF7C01662344
:102F300059F528ED30E0E20EF31ED7018C91E8E25E
:102F4000FFEFEE0EFF1E882309F4F2C00FB6F894CF
:102F50002091A40D3091A50D4091A60D5091A70D83
:102F60000FBE60ED70E0E60EF71EF70180819181E3
:102F7000A281B38160E37FEFE60EF71E821793070D
:102F8000A407B50708F4D4C088ED90E0E80EF91E58
:102F9000D7011C92E8E2FFEFEE0EFF1ED70112965A
:102FA0008C91882339F4C701DBDEF7018281882305
:102FB00009F4BEC000D000D000D0EDB7FEB7319606
:102FC0008E010F5F1F4FADB7BEB712961C930E93C5
:102FD00011978CE091E093838283D7011F968D91A6
:102FE0009C915097958384830E94A50BCC24DD246B
:102FF000EDB7FEB736960FB6F894FEBF0FBEEDBF25
:1030000058010AC0D8018C91992787FD90950E949C
:10301000BA78F80181938F01C601F5010190002073
:10302000E9F73197EA19FB090894C11CD11C8E17E6
:103030009F0744F3E4E18E2E912C8E0C9F1CC4015B
:1030400040E050E060E070E00E94115177247DE3A1
:10305000A72EB12CAC0EBD1E1E010894211C311CE4
:103060006FE1462E512C4C0E5D1E48C0D6018C914E
:1030700090E00E94BA78F60181936F01C801F501D2
:1030800001900020E9F73197EA19FB090F5F1F4F04
:103090008E179F075CF327968FAD27978E3771F1B8
:1030A000C501B10145E050E00E946E0B009731F57B
:1030B00000D000D000D0EDB7FEB73196ADB7BEB7A7
:1030C00012965C924E92119725E131E03383228370
:1030D000358224820E94A50B6DB77EB76A5F7F4F51
:1030E0000FB6F8947EBF0FBE6DBFC2010E944C5058
:1030F0008CE191E00E944C5077247394C401B50197
:103100000E942154181624F4650100E010E0B6CFA7
:10311000772041F48FEF9FEFD70150969C938E93C9
:103120001F9706C0F701878590890196908B878746
:10313000C45ADF4F0FB6F894DEBF0FBECDBFCF919C
:10314000DF911F910F91FF90EF90DF90CF90BF9094
:10315000AF909F908F907F905F904F903F902F9077
:1031600008952F923F924F925F926F927F928F922B
:103170009F92AF92BF92CF92DF92EF92FF920F9306
:103180001F93DF93CF93CDB7DEB7CB58D0400FB6A8
:10319000F894DEBF0FBECDBF6C012B015A0183E056
:1031A00090E0A80EB91EF6013396CC57DF4FF98395
:1031B000E883C458D040CA57DF4F1882C658D04061
:1031C00014E6E12EF12CEC0EFD1EC7010B96C9573B
:1031D000DF4F99838883C758D040B9ED6B2E712C8F
:1031E0006C0C7D1CABED8A2E912C8C0C9D1CF6E496
:1031F0002F2E312C2C0E3D1EF1013396C757DF4F79
:10320000F983E883C958D040E3EEF0E08491C557D4
:10321000DF4F8883CB58D0401BC1F7018385482FEF
:1032200050E0BA01687170706031710509F018C121
:10323000F301208131812130310509F411C122309F
:10324000310509F40DC1F701DE011196908190322C
:1032500039F08E2F8E19883011F48EE28D939D9364
:103260003196C957DF4F88819981C758D040E817F8
:10327000F90761F71C921E86F2018081882331F4E0
:10328000CE010E9660E271E00E94510BCE010E96C7
:10329000B2010E94510BCE010E96BE016F5F7F4FAF
:1032A0000E94510BCE010E9660E271E00E94510B1C
:1032B0001BA61EA61AA688EC92E099A788A7CE01A5
:1032C0008B96B501AE014F5F5F4F21E00E94AA5877
:1032D000882349F5F30180819181892B21F5C55718
:1032E000DF4F6881CB58D04003EE10E007C089EA79
:1032F0009DE0A6D80F5F1F4FF80164916623B9F7D0
:1033000089EA9DE062E271E02DD989EA9DE06AE0F8
:1033100097D889EA9DE0BE016F5F7F4F23D989EA84
:103320009DE06AE08DD8C757DF4FA881B981C958A1
:10333000D040FE01BB968BE101900D928150E1F7E8
:103340008AA5F101828388EC92E091838083C60193
:10335000BE01625F7F4FA10104DFC10117D9CE0119
:10336000889614D975C0953E09F472C09E3209F44E
:103370006FC09F3509F46CC043FD6AC080E06031C6
:10338000710509F481E0F6018687882349F4F70185
:103390008085873409F05CC081858E3709F458C078
:1033A000CC57DF4FA881B981C458D040F701808144
:1033B000803241F08E2F8E19883011F48EE28D9379
:1033C00080818D933196C957DF4F88819981C75885
:1033D000D040E817F90759F71C92F30180819181D9
:1033E000009791F489EA9DE0B201BCD889EA9DE09A
:1033F000CC57DF4F68817981C458D040B3D889EA6F
:103400009DE06AE01DD824C08130910539F4F401B3
:10341000808191810196918380831AC00297C1F4C3
:10342000CA57DF4FF881C658D0402F2F30E0F40143
:103430008081918128173907C1F0CA57DF4FF88181
:10344000C658D040FF5FCA57DF4FF883C658D040F8
:10345000C501B7010E94215418160CF4DECE05C038
:10346000F7019081992309F07ECFC557DF4F0FB642
:10347000F894DEBF0FBECDBFCF91DF911F910F91AA
:10348000FF90EF90DF90CF90BF90AF909F908F9084
:103490007F906F905F904F903F902F900895EF92A4
:1034A000FF920F931F93DF93CF93CDB7DEB76E9745
:1034B0000FB6F894DEBF0FBECDBF7C0189ED90E062
:1034C000E80EF91EF7011182108287E29FEFE80EE5
:1034D000F91E87010C5E1F4FC80140E050E060E01C
:1034E00070E00E941151DE011496F8018BE1019009
:1034F0000D928150E1F7F70183898B8388EC92E08C
:103500009A838983C70165E371E08E010F5F1F4FC6
:10351000A80127DEC8013AD86E960FB6F894DEBF30
:103520000FBECDBFCF91DF911F910F91FF90EF9014
:10353000089510921003109212031092140308952C
:10354000809318020895EFE6F0E080818260808326
:103550000895099A0B9A0D9A0F9A6F9A779A6E9A14
:10356000769A3F9A479A3B9A439A6B98739A209817
:10357000289A6C98749A089A779A0A9A769A0C9A6A
:10358000479A0E9A439AA1E8B0E08C918F7E8C9373
:103590008C9188608C93E0E8F0E080818D7F80835F
:1035A00080818E7F808380818F73808380818F7CF8
:1035B00080838C91887F82608C9380E090E49093EC
:1035C0008900809388001092850010928400EFE6B5
:1035D000F0E08081826080831092180278940895D0
:1035E0001F93FC011FB7F89480819181A281B38160
:1035F0008093EA029093EB02A093EC02B093ED0269
:10360000FB0180819181A281B3818093EE0290932E
:10361000EF02A093F002B093F102FA018081918150
:10362000A281B3818093F2029093F302A093F402FB
:10363000B093F502F90180819181A281B3818093D9
:10364000F6029093F702A093F802B093F9021FBF1D
:103650001F910895FC012FB7F89480819181A28178
:10366000B3818093F6029093F702A093F802B0938F
:10367000F9022FBF0895E82F8FB7F894F0E0EE0F0E
:10368000FF1FEE0FFF1FE651FD4F20813181428168
:1036900053818FBFB901CA01089580916F008D7F5A
:1036A00080936F0006C080918A0D8F5F8F7080932A
:1036B0008A0D9091890D80918A0D981751F410927E
:1036C000DD021092DC0280916F00826080936F00B7
:1036D00008959091890D80918A0D981751F3E3CF49
:1036E0009091890D80918A0D981731F00E94F625EE
:1036F00081E00E941D36F4CF0895F2DF779A769A22
:10370000479A439A08951F920F920FB60F920BB6E5
:103710000F921124AF92BF92CF92DF92EF92FF925D
:103720000F931F932F933F934F935F936F937F93C9
:103730008F939F93AF93BF93CF93DF93EF93FF93B9
:103740008091DC029091DD02892B09F08BC1909170
:10375000890D80918A0D981719F4E0E0F0E014C00B
:1037600080918A0D90E02DE430E0829FF001839FEC
:10377000F00D929FF00D1124E754F74FE45BFF4FDB
:1037800081E08083EC54F040F093DD02E093DC02B2
:10379000309709F461C110921C0310921D0310921E
:1037A0001E0310921F0344AD55AD50931B0340936D
:1037B0001A032CE94134520718F040E45CE904C0D4
:1037C0003EE44132530730F056954795569547955C
:1037D00084E007C067E24131560730F056954795BF
:1037E00082E08093150308C081E080931503403286
:1037F000510510F440E250E08A010052104078E098
:1038000000301707E8F0412F50E0440F551F440FD8
:10381000551F4A5A5D4F9A012E5F3F4FF90185911E
:1038200094919C01AA27039FC001029F810D9A1FBA
:1038300006948A1F9A1F1124FA01459154911EC0C3
:10384000C801969587958C7F8A5A994FFC014591BE
:103850005491FC01329625913491802F90E087702D
:103860009070BC01269FC001279F900D369F900D40
:103870001124F3E096958795FA95E1F7481B590BCB
:1038800044365105A8F489EA9DE066E371E00E94A0
:10389000B212A80160E070E089EA9DE02AE000E051
:1038A0000E94277089EA9DE00E940B7044E650E078
:1038B000CA01A0E0B0E08093160390931703A09391
:1038C0001803B09319035093890040938800E09146
:1038D000DC02F091DD0240AD51AD7CE94134570787
:1038E00018F040E45CE904C08EE44132580730F03F
:1038F000569547955695479584E007C097E2413124
:10390000590730F05695479582E08093150308C01B
:1039100081E0809315034032510510F440E250E0FD
:103920008A0100521040E8E000301E07E8F0412F05
:1039300050E0440F551F440F551F4A5A5D4F9A01DE
:103940002E5F3F4FF901859194919C01AA27039F17
:10395000C001029F810D9A1F06948A1F9A1F11248D
:10396000FA01459154911EC0C801969587958C7FA8
:103970008A5A994FFC0145915491FC013296259148
:103980003491802F90E087709070BC01269FC00119
:10399000279F900D369F900D112433E096958795C3
:1039A0003A95E1F7481B590B44365105A8F489EACA
:1039B0009DE066E371E00E94B212A80160E070E051
:1039C00089EA9DE02AE000E00E94277089EA9DE0F4
:1039D0000E940B7044E650E0509321034093200373
:1039E000E091DC02F091DD0280899189A289B3899E
:1039F000B695A79597958795B095A0959095819543
:103A00009F4FAF4FBF4F8093FA029093FB02A0935A
:103A1000FC02B093FD028093FE029093FF02A093FC
:103A20000003B09301038093020390930303A093D8
:103A30000403B09305038093060390930703A093B8
:103A40000803B093090310920A0310920B0310921B
:103A50000C0310920D0306C080ED97E0909389004F
:103A600080938800E091DC02F091DD02309709F448
:103A70005AC580A180930E0380FF3BC08FEF8093D7
:103A80001402809118028823B9F1639902C080E082
:103A90002DC080910F03882341F180819181A28103
:103AA000B381181619061A061B06FCF48091EA0267
:103AB0009091EB02A091EC02B091ED028093DE02B6
:103AC0009093DF02A093E002B093E10281E0809343
:103AD000100380899189A289B38980930A03909306
:103AE0000B03A0930C03B0930D0381E080930F03AD
:103AF00003C081E08093140280910E0381FF3AC0DD
:103B00008FEF80931502809118028823B1F123B1C1
:103B1000217031E0232759F180911103882339F175
:103B200084819581A681B781181619061A061B068D
:103B3000F4F48091EE029091EF02A091F002B09126
:103B4000F1028093E2029093E302A093E402B09327
:103B5000E5023093120380899189A289B389809309
:103B60000A0390930B03A0930C03B0930D032093CF
:103B7000110303C081E080931502208131814281CD
:103B8000538184819581A681B781281739074A0717
:103B90005B0744F080910E0380FD02C0119A0FC0B4
:103BA00011980AC0281739074A075B074CF480911F
:103BB0000E0381FD03C0119A139802C01198139A45
:103BC00080910E0382FF3CC0159A8FEF80931602FE
:103BD000809118028823C1F1649902C080E02DC051
:103BE00080911303882341F180859185A285B38557
:103BF000181619061A061B06FCF48091F202909121
:103C0000F302A091F402B091F5028093E602909342
:103C1000E702A093E802B093E90281E080931403E5
:103C200080899189A289B38980930A0390930B03B9
:103C3000A0930C03B0930D0381E08093130304C0A1
:103C4000159881E08093160280910E0383FF03C0D4
:103C500017988FEF02C0179A81E08093170260E0F7
:103C600043C22091FA023091FB024091FC02509134
:103C7000FD0280819181A281B381280F391F4A1FE3
:103C80005B1F2093FA023093FB024093FC02509397
:103C9000FD02E480F580068117818091FE029091FB
:103CA000FF02A0910003B0910103E80EF91E0A1F64
:103CB0001B1FE092FE02F092FF020093000310939C
:103CC00001031216130614061506A4F51E141F048C
:103CD000100611067CF1109A129A80899189A289A6
:103CE000B389281B390B4A0B5B0B2093FA023093E4
:103CF000FB024093FC025093FD0210981298209111
:103D0000EA023091EB024091EC025091ED02809179
:103D10001402992787FD9095A92FB92F820F931F21
:103D2000A41FB51F8093EA029093EB02A093EC02CC
:103D3000B093ED028091FA029091FB02A091FC02F7
:103D4000B091FD02181619061A061B06E4F120911F
:103D5000FE023091FF0240910003509101031216C0
:103D60001306140615067CF5109A129A808991891B
:103D7000A289B389281B390B4A0B5B0B2093FE02E7
:103D80003093FF0240930003509301031098129860
:103D90002091EE023091EF024091F0025091F10239
:103DA00080911502992787FD9095A92FB92F820F31
:103DB000931FA41FB51F8093EE029093EF02A09370
:103DC000F002B093F1022091FA023091FB0240918F
:103DD000FC025091FD0212161306140615060CF093
:103DE000CAC0E090FE02F090FF0200910003109123
:103DF00001031E141F04100611060CF0BCC09091A4
:103E00000E03892F8695892780FF5BC0129A8089CF
:103E10009189A289B389281B390B4A0B5B0B20932C
:103E2000FA023093FB024093FC025093FD02129879
:103E30002091EA023091EB024091EC025091ED02A8
:103E400080911402992787FD9095A92FB92F820F91
:103E5000931FA41FB51F8093EA029093EB02A093D7
:103E6000EC02B093ED022091EE023091EF0240910E
:103E7000F0025091F10280911502992787FD9095EB
:103E8000A92FB92F820F931FA41FB51F8093EE0295
:103E90009093EF02A093F002B093F102129A8089FE
:103EA0009189A289B389E81AF90A0A0B1B0BE092DF
:103EB000FE02F092FF020093000310930103129898
:103EC0005AC0109A80899189A289B389281B390B1D
:103ED0004A0B5B0B2093FA023093FB024093FC02E7
:103EE0005093FD0210982091EA023091EB0240912C
:103EF000EC025091ED0280911402992787FD909574
:103F0000A92FB92F820F931FA41FB51F8093EA0218
:103F10009093EB02A093EC02B093ED022091EE029D
:103F20003091EF024091F0025091F1028091150220
:103F3000992787FD9095A92FB92F820F931FA41F52
:103F4000B51F8093EE029093EF02A093F002B0931E
:103F5000F102109A80899189A289B389E81AF90A35
:103F60000A0B1B0BE092FE02F092FF02009300038B
:103F700010930103109820853185428553858091E7
:103F8000020390910303A0910403B0910503280F4D
:103F9000391F4A1F5B1F2093020330930303409392
:103FA00004035093050312161306140615066CF548
:103FB000149A80899189A289B389281B390B4A0BED
:103FC0005B0B20930203309303034093040350934D
:103FD000050314982091F2023091F3024091F4020B
:103FE0005091F50280911602992787FD9095A92F8F
:103FF000B92F820F931FA41FB51F8093F2029093D5
:10400000F302A093F402B093F5022485358546852A
:1040100057858091060390910703A0910803B09102
:104020000903280F391F4A1F5B1F20930603309393
:10403000070340930803509309031216130614064E
:1040400015066CF5169A80899189A289B389281B77
:10405000390B4A0B5B0B2093060330930703409305
:1040600008035093090316982091F6023091F70245
:104070004091F8025091F90280911702992787FD2B
:104080009095A92FB92F820F931FA41FB51F80935E
:10409000F6029093F702A093F802B093F902809190
:1040A0000A0390910B03A0910C03B0910D030196AC
:1040B000A11DB11D80930A0390930B03A0930C03E1
:1040C000B0930D0320910A0330910B0340910C0330
:1040D00050910D0380899189A289B38928173907E6
:1040E0004A075B0730F46F5F8091150368170CF483
:1040F000B8CD20910A0330910B0340910C035091ED
:104100000D0384899589A689B78982179307A40727
:10411000B50708F4E4C0E0901603F090170300918F
:10412000180310911903A48CB58CC68CD78CA801E8
:104130009701C601B501AA27279FB12D389FE0013D
:10414000489FD00D479FC00DD11D289FB00DC11DA8
:10415000DA1F379FB00DC11DDA1F469FB00DC11D7C
:10416000DA1F369FB10DCA1FDA1FB695CA1FDA1FB4
:10417000112484AD95AD8C0F9D1F90931B038093EC
:104180001A0320AD31AD42AD53ADA0E0B0E0281729
:1041900039074A075B0720F430931B0320931A0367
:1041A00040911A0350911B037CE94134570718F0E2
:1041B00040E45CE904C08EE44132580730F0569583
:1041C00047955695479584E007C097E241315907D6
:1041D00030F05695479582E08093150308C081E042
:1041E000809315034032510510F440E250E08A01FB
:1041F00000521040E8E000301E07E8F0412F50E088
:10420000440F551F440F551F4A5A5D4F9A012E5FA8
:104210003F4FF901859194919C01AA27039FC0010A
:10422000029F810D9A1F06948A1F9A1F1124FA017A
:10423000459154911EC0C801969587958C7F8A5AE6
:10424000994FFC0145915491FC013296259134918E
:10425000802F90E087709070BC01269FC001279F3F
:10426000900D369F900D1124F3E096958795FA9561
:10427000E1F7481B590B44365105A8F489EA9DE043
:1042800066E371E00E94B212A80160E070E089EA82
:104290009DE02AE000E00E94277089EA9DE00E94EC
:1042A0000B7044E650E050938900409388009A01D7
:1042B00040E050E08091160390911703A0911803FD
:1042C000B0911903820F931FA41FB51F809316038B
:1042D00090931703A0931803B0931903FFC0209184
:1042E0000A0330910B0340910C0350910D03808D14
:1042F000918DA28DB38D82179307A407B50708F09F
:10430000E5C060911C0370911D0380911E03909184
:104310001F03248D358D468D578DAA27639FB12DA0
:10432000749F8001849F100D839F000D111D649F59
:10433000B00D011D1A1F739FB00D011D1A1F829F22
:10434000B00D011D1A1F729FB10D0A1F1A1FB695DD
:104350000A1F1A1F112480911A0390911B038017C2
:10436000910738F4E05CFF4F40815181E054F04008
:1043700003C0AC01401B510BE05CFF4F0081118179
:1043800022813381CA01A0E0B0E080179107A20723
:10439000B30708F4A8017CE94134570718F040E45A
:1043A0005CE904C08EE44132580730F056954795D9
:1043B0005695479584E007C097E24131590730F0A0
:1043C0005695479582E08093150308C081E080935D
:1043D00015034032510510F440E250E08A010052CA
:1043E0001040E8E000301E07E8F0412F50E0440F95
:1043F000551F440F551F4A5A5D4F9A012E5F3F4F7C
:10440000F901859194919C01AA27039FC001029F05
:10441000810D9A1F06948A1F9A1F1124FA01459153
:1044200054911EC0C801969587958C7F8A5A994FE2
:10443000FC0145915491FC01329625913491802FD5
:1044400090E087709070BC01269FC001279F900D5F
:10445000369F900D112423E0969587952A95E1F7D4
:10446000481B590B44365105A8F489EA9DE066E3E0
:1044700071E00E94B212A80160E070E089EA9DE05C
:104480002AE000E00E94277089EA9DE00E940B70FC
:1044900044E650E050938900409388009A0140E040
:1044A00050E080911C0390911D03A0911E03B091D8
:1044B0001F03820F931FA41FB51F80931C039093AB
:1044C0001D03A0931E03B0931F0308C08091200317
:1044D00090912103909389008093880020910A0392
:1044E00030910B0340910C0350910D03E091DC02DD
:1044F000F091DD0280899189A289B3892817390753
:104500004A075B0780F01092DD021092DC02909166
:10451000890D80918A0D981731F080918A0D8F5FF7
:104520008F7080938A0DFF91EF91DF91CF91BF91B2
:10453000AF919F918F917F916F915F914F913F913B
:104540002F911F910F91FF90EF90DF90CF90BF9030
:10455000AF900F900BBE0F900FBE0F901F9018954D
:10456000EF92FF920F931F93DF93CF930F92CDB7EC
:10457000DEB780911003882349F4809112038823C9
:1045800029F480911403882309F4E7C0E6E5FAE0F2
:1045900084918F017E010894E11CF11C0CC0898379
:1045A00089EA9DE0B70141E050E00E94546E0F5F40
:1045B0001F4FF8018491882391F7E8E6FAE084918F
:1045C0008F017E010894E11CF11C0CC0898389EAEB
:1045D0009DE0B70141E050E00E94546E0F5F1F4F15
:1045E000F8018491882391F780911003882391F139
:1045F000E4E6FAE084918F017E010894E11CF11C4D
:104600000CC0898389EA9DE0B70141E050E00E9437
:10461000546E0F5F1F4FF8018491882391F76091CA
:10462000DE027091DF028091E0029091E1020E942F
:10463000197520915D0830915E0840915F08509196
:1046400060080E947E74AB01BC0189EA9DE022E013
:104650000E94C37080911203882391F1E0E6FAE092
:1046600084918F017E010894E11CF11C0CC08983A8
:1046700089EA9DE0B70141E050E00E94546E0F5F6F
:104680001F4FF8018491882391F76091E2027091A5
:10469000E3028091E4029091E5020E941975209155
:1046A00061083091620840916308509164080E944B
:1046B0007E74AB01BC0189EA9DE022E00E94C370D8
:1046C00080911403882391F1ECE5FAE084918F0145
:1046D0007E010894E11CF11C0CC0898389EA9DE0ED
:1046E000B70141E050E00E94546E0F5F1F4FF80188
:1046F0008491882391F76091E6027091E70280919E
:10470000E8029091E9020E941975209165083091A4
:10471000660840916708509168080E947E74AB015A
:10472000BC0189EA9DE022E00E94C37089EA9DE015
:104730006AE471E00E94B2128AE0898389EA9DE00E
:10474000BE016F5F7F4F41E050E00E94546E1092B7
:10475000100310921203109214030F90CF91DF9167
:104760001F910F91FF90EF90089560E070E08FE748
:1047700093E420911D0230911E0240911F0250913E
:1047800020020E947E746093490370934A038093D1
:104790004B0390934C030895FC01E25DFC4F808134
:1047A00090E0089580E090E0089560E070E080E09F
:1047B00090E0089508951F920F920FB60F92112462
:1047C0002F933F934F935F938F939F93AF93BF9399
:1047D00090912B02992331F480912E038093320320
:1047E0008111459A80913203981708F045989F5F90
:1047F0009F7790932B0280913303833009F448C054
:10480000843028F48130E1F08230C0F50DC085306D
:1048100009F45CC0853008F457C0863009F458C0EC
:10482000873009F05EC056C010927B0083E480930D
:104830007C0080917A00806480937A0081E01BC0C4
:104840008091780090917900A0E0B0E02091400341
:10485000309141034091420350914303280F391F87
:104860004A1F5B1F20934003309341034093420350
:104870005093430382E08093330333C082E48093F8
:104880007C0080917A00806480937A0083E0F3CF8B
:104890008091780090917900A0E0B0E020913403FD
:1048A000309135034091360350913703280F391F5B
:1048B0004A1F5B1F20933403309335034093360324
:1048C0005093370384E0D7CF85E0D5CF86E0D3CFB0
:1048D00087E0D1CF10923303809144038F5F8093A0
:1048E000440380914403803108F44FC04091400359
:1048F0005091410350932703409326038FEF9FE38A
:104900002091340330913503821B930B909329033C
:104910008093280381E080932F0310924403109228
:1049200040031092410310924203109243031092ED
:104930003C0310923D0310923E0310923F031092ED
:1049400038031092390310923A0310923B031092ED
:10495000340310923503109236031092370380917E
:10496000290290912A024817590724F01092230334
:1049700010922203809130039091310384179507A0
:1049800024F01092230310922203BF91AF919F91C4
:104990008F915F914F913F912F910F900FBE0F908C
:1049A0001F9018952F923F924F925F926F927F9235
:1049B0008F929F92AF92BF92CF92DF92EF92FF922F
:1049C0000F931F93DF93CF9300D0CDB7DEB76C0169
:1049D000162F662389F1E7E7FAE064914F0109C0D9
:1049E00089EA9DE00E9420120894811C911CF40128
:1049F00064916623A9F7412F50E0662757FD609523
:104A0000762F89EA9DE00E94B270E4E1FBE06491B8
:104A10004F0109C089EA9DE00E9420120894811C80
:104A2000911CF40164916623A9F789EA9DE06AE08C
:104A30000E9420120E94F035A12FB0E0AA0FBB1FE8
:104A4000FD01EE5AFD4F208131812115310509F418
:104A500097C0E0EF8E2EEFE39E2E8C189D08AC5A87
:104A6000BD4F4D915C9161E06CC08D01000F111F35
:104A7000000F111FF901E00FF11F85919491881625
:104A800099060CF05DC0CD010197880F991F880F22
:104A9000991FFC013296E20FF31FC590D490820F4C
:104AA000931FFC01859194919A838983F801329632
:104AB000E20FF31FE590F490F901E00FF11FA590CC
:104AC000B490B601882777FD8095982F0E941975BC
:104AD0001B012C01B401E981FA816E1B7F0B882731
:104AE00077FD8095982F0E9419753B014C01EC18B9
:104AF000FD080027F7FC0095102FC801B7010E94A0
:104B000019759B01AC01C401B3010E9457777B0169
:104B10008C0189819A81A81AB90ACC24B7FCC09467
:104B2000DC2CC601B5010E9419759B01AC01C801BE
:104B3000B7010E947E749B01AC01C201B10137C074
:104B40006F5FA62FB0E0A417B5070CF48ECFA417A3
:104B5000B50729F0E0E070E080E060E02CC0FA01E9
:104B6000EE0FFF1FEE0FFF1F3297E20FF31F65914D
:104B70007491882777FD8095982F0E94197519C028
:104B8000B601882777FD8095982F0E94197520E03F
:104B900030E04AEF5EE30E94577720E030E040E8E3
:104BA0005DE30E94577720E030E040E050E00E9453
:104BB0009E73E62F692F2E2F372F482F562FB901BE
:104BC000CA010F900F90CF91DF911F910F91FF902D
:104BD000EF90DF90CF90BF90AF909F908F907F909D
:104BE0006F905F904F903F902F9008952F923F923B
:104BF0004F925F926F927F928F929F92AF92BF92ED
:104C0000CF92DF92EF92FF920F931F9380912F0329
:104C1000882309F489C18FB7F89410922F038FBFAE
:104C2000809126039091270360E0BCDE3B014C019C
:104C300060912A0370912B0380912C0390912D0396
:104C4000A40193010E949D737B018C0160934D032D
:104C500070934E0380934F039093500320E030E015
:104C600040E251E40E948576181624F481E0809396
:104C70005103EFC0C801B70120E030E040E251EC41
:104C80000E947774882324F481E080935103CCC080
:104C900080915103882371F080E090E0A0E0B0E0C3
:104CA0008093520390935303A0935403B0935503FE
:104CB00010925103C801B7012091190230911A02D4
:104CC00040911B0250911C020E9457771B012C013E
:104CD000609356037093570380935803909359033E
:104CE000C801B701209152033091530340915403FE
:104CF000509155030E949E735B016C01E090450347
:104D0000F09046030091470310914803A8019701D2
:104D10000E94777487FD12C0E0904903F0904A0327
:104D200000914B0310914C03C601B501A8019701F6
:104D30000E948576181614F086017501E0925203E0
:104D4000F09253030093540310935503C801B70125
:104D500020911D0230911E0240911F0250912002AD
:104D60000E9457775B016C0160935A0370935B0359
:104D700080935C0390935D03C401B30120915E03B3
:104D800030915F0340916003509161030E949D73D5
:104D9000209121023091220240912302509124025D
:104DA0000E94577720ED3CEC4CE45DE30E9457777E
:104DB0007B018C01609162037091630380916403B5
:104DC0009091650323E333E343E75FE30E94577762
:104DD0009B01AC01C801B7010E949E737B018C014D
:104DE00060936203709363038093640390936503FD
:104DF00060925E0370925F03809260039092610301
:104E0000C201B101A60195010E949E73A8019701FC
:104E10000E949D737B018C0120E030E040E050E077
:104E20000E94777488235CF40F2EF0E0EF2EF0E000
:104E3000FF2EF0E00F2FF0E01F2FF02D14C0C8015F
:104E4000B70120E030E04FE753E40E948576181662
:104E500054F40F2EF0E0EF2EF0E0FF2EFFE70F2FBF
:104E6000F3E41F2FF02D209126033091270380912A
:104E70003003909131038217930784F480912902C3
:104E800090912A02281739074CF4C801B7010E94F3
:104E9000E6747595679560932E0302C010922E03F9
:104EA0000FB6F8948091A40D9091A50DA091A60D38
:104EB000B091A70D0FBE209166033091670340911A
:104EC000680350916903821B930BA40BB50B8858A0
:104ED0009341A040B04040F10FB6F8948091A40DEA
:104EE0009091A50DA091A60DB091A70D0FBE809336
:104EF000660390936703A0936803B09369032091BE
:104F0000280330912903121613066CF48FE32F3F08
:104F100038074CF480912403909125032817390712
:104F200014F4449A01C044981F910F91FF90EF90A0
:104F3000DF90CF90BF90AF909F908F907F906F90B9
:104F40005F904F903F902F900895EF92FF920F93B4
:104F50001F93CF93DF937C01062F662369F1E7E768
:104F6000FAE06491EF0107C089EA9DE00E942012F7
:104F70002196FE0164916623B9F7402F50E0662721
:104F800057FD6095762F89EA9DE00E94B270E1E3BB
:104F9000FBE06491EF0107C089EA9DE00E942012C6
:104FA0002196FE0164916623B9F789EA9DE06AE0E3
:104FB0000E9420120E94F035A02FB0E0AA0FBB1F64
:104FC000FD01EE5AFD4FC081D181209709F468C0E0
:104FD000AC5ABD4F4D915C9121E047C0BD01660FB9
:104FE000771F660F771F6E5F7F4FFE01E60FF71F7B
:104FF000859194918E159F050CF036C09D0121502E
:105000003040220F331F220F331FCE01820F931F18
:10501000FC01059114912E5F3F4F2C0F3D1FF901AC
:1050200025913491FD01EE0FFF1FEE0FFF1FEC0FD6
:10503000FD1F85919491FE01E60FF71F6591749114
:10504000801B910BE21AF30A621B730B9C012E9DCD
:10505000C0012F9D900D3E9D900D11240E94487817
:10506000CB01800F911F17C02F5FA22FB0E0A417B4
:10507000B5070CF4B3CFA417B50719F080E090E0A2
:105080000AC0FA013197EE0FFF1FEE0FFF1FEC0F62
:10509000FD1F8591949160EF7FE3681B790B15C02C
:1050A000B701882777FD8095982F0E9419752FE604
:1050B00032E143E050E40E94577720E030E040E8DE
:1050C00051E40E9457770E94E674CB01DF91CF91A3
:1050D0001F910F91FF90EF90089580E090E060E0C5
:1050E00034DF80E090E0A0E0B0E080932A0390936A
:1050F0002B03A0932C03B0932D0310922303109243
:10510000220310922E034598E0E9F0E080818F7D24
:105110008083109225031092240344988081877F16
:105120008083089580E090E0A0E0B0E080934503A4
:1051300090934603A0934703B093480360E070E068
:105140008FE793E420911D0230911E0240911F02CF
:10515000509120020E947E746093490370934A0329
:1051600080934B0390934C033D9A3C9A3E9A87ED73
:1051700080937A00EEE7F0E010828081886080837F
:1051800080818460808380E888BDEEE6F0E08081E5
:10519000846080836AEF70E080E090E00E94FF6CA2
:1051A00085E090E060E0D1DE90933103809330039E
:1051B0008AEF90E060E0C9DE90932A028093290292
:1051C00008952F923F924F925F926F927F928F92AB
:1051D0009F92AF92BF92CF92DF92EF92FF920F9386
:1051E0001F93DF93CF93CDB7DEB7E4970FB6F89454
:1051F000DEBF0FBECDBF6F8F78A389A39AA38FE7C1
:1052000080932E030FB6F8942091A40D3091A50D34
:105210004091A60D5091A70D0FBE2D8B3E8B4F8B4D
:10522000588FE091A90DF091AA0D0280F381E02D35
:1052300089EA9DE06BE471E042E150E0099589EA7A
:105240009DE06AE00E9420128D899E89AF89B88D09
:10525000898B9A8BAB8BBC8B8D879E87AF87B88BE6
:105260001A8E198E11E05FE7652E712C812C912C1E
:105270004FE7242E312C412C512CE4E0FCE094919A
:105280009BA3EFEFFBE0A491ACA3E8EFFBE0B491AC
:10529000BDA3E1EFFBE024912EA3EBEEFBE0349104
:1052A0003FA3E5EEFBE0449148A7E8EDFBE0549115
:1052B00059A7E2EDFBE084918AA7ECECFBE0949126
:1052C0009BA7E6ECFBE0A491ACA7E5EBFBE0B49177
:1052D000BDA7EFEAFBE024912EA780912F0388233E
:1052E00009F4D2C38FB7F89410922F038FBF809127
:1052F00026039091270360E055DB6FA778AB89AB5D
:105300009AAB69817A818B819C812FA538A949A9A3
:105310005AA90E948576181644F08FA598A9A9A9C4
:10532000BAA989839A83AB83BC83C601B5012FA533
:1053300038A949A95AA90E94777487FD06C08FA58C
:1053400098A9A9A9BAA95C016D01112309F455C056
:105350006FA578A989A99AA92F8D38A149A15AA129
:105360000E94857618160CF08FC30FB6F8948091C2
:10537000A40D9091A50DA091A60DB091A70D0FBE03
:105380002D853E854F855889821B930BA40BB50B49
:1053900089589341A040B04008F476C3D401C301BA
:1053A00082199309A409B509B595A795979587958D
:1053B00080932E030FB6F8948091A40D9091A50DC3
:1053C000A091A60DB091A70D0FBE898B9A8BAB8BC8
:1053D000BC8B2D853E854F855889821B930BA40B72
:1053E000B50B89879A87AB87BC878F8D98A1A9A1B8
:1053F000BAA189839A83AB83BC836FA578A989A955
:105400009AA92F8D38A149A15AA10E9477748823A7
:105410000CF039C30FB6F8948091A40D9091A50DAE
:10542000A091A60DB091A70D0FBE29893A894B898D
:105430005C89821B930BA40BB50B89589341A04048
:10544000B04008F420C30FB6F8948091A40D909159
:10545000A50DA091A60DB091A70D0FBE8D879E87BB
:10546000AF87B88BA98DBA8DAB2B09F4F4C28D85AB
:105470009E85AF85B88929893A894B895C89821BC9
:10548000930BA40BB50B29853A854B855C85280FBA
:10549000391F4A1F5B1F2B8F3C8F4D8F5E8F2985D5
:1054A0003A854B855C85281B390B4A0B5B0BCA017F
:1054B000B901A20191010E9429782B8D3C8D4D8D5F
:1054C0005E8D0E947D78260D371D481D591D2431A3
:1054D0003105410551055CF424E1222E312C412C8B
:1054E000512C94E1692E712C812C912C1FC0390113
:1054F0004A013CEE63167104810491042CF08BEE9A
:10550000682E712C812C912C40E864167104810462
:1055100091041CF41301240109C00EEF202E312C3C
:10552000412C512C26183708480859086BA104E073
:105530001CE008C089EA9DE00E9420120F5F1F4F07
:10554000F80164916623B1F789EA9DE0B401A301F3
:105550000E94B2706CA10FEF1BE008C089EA9DE0C9
:105560000E9420120F5F1F4FF80164916623B1F76C
:1055700089EA9DE0B201A1010E94B2706DA108EF1D
:105580001BE008C089EA9DE00E9420120F5F1F4FB8
:10559000F80164916623B1F789EA9DE0B601A5019F
:1055A00022E00E94C3706EA101EF1BE008C089EAEF
:1055B0009DE00E9420120F5F1F4FF8016491662347
:1055C000B1F789EA9DE049815A816B817C8122E0B3
:1055D0000E94C37089EA9DE06AE00E942012298D32
:1055E0003A8D233031050CF436C2C201B1010E945C
:1055F000197520E030E040E850E40E9457777B01C5
:105600008C0169817A818B819C81A60195010E9420
:105610009D7320ED3FE049E450E40E94577720E07D
:1056200030E040E05FE30E9457779B01AC01C80186
:10563000B7010E947E746D837E838F8398876B8D04
:105640007C8D8D8D9E8D0E94197520E030E04AE79B
:1056500054E40E947E745B016C016FA10BEE1BE0B1
:1056600008C089EA9DE00E9420120F5F1F4FF801D9
:1056700064916623B1F789EA9DE04D815E816F8177
:10568000788522E00E94C37068A505EE1BE008C083
:1056900089EA9DE00E9420120F5F1F4FF80164917C
:1056A0006623B1F789EA9DE0B601A50122E00E94D8
:1056B000C37089EA9DE06AE00E9420126D817E81BC
:1056C0008F8198852AE939E949E15FE30E9457779C
:1056D0007B018C0169A528ED3BE03CAB2BAB0CC0FA
:1056E00089EA9DE00E9420124BA95CA94F5F5F4FA1
:1056F0005CAB4BABFA016491662391F789EA9DE0BC
:105700006AE00E9420126AA522ED3BE03CAB2BAB85
:105710000CC089EA9DE00E9420124BA95CA94F5F52
:105720005F4F5CAB4BABFA016491662391F789EA5A
:105730009DE0B801A70122E00E94C37089EA9DE0C4
:105740006AE00E9420126BA52CEC3BE03CAB2BAB3B
:105750000CC089EA9DE00E9420124BA95CA94F5F12
:105760005F4F5CAB4BABFA016491662391F7C801C4
:10577000B701A80197010E949E73A60195010E949E
:105780007E74AB01BC0189EA9DE022E00E94C370F7
:1057900089EA9DE06AE00E9420126CA526EC3BE0BD
:1057A0003CAB2BAB0CC089EA9DE00E9420124BA9B8
:1057B0005CA94F5F5F4F5CAB4BABFA016491662312
:1057C00091F7C801B701A60195010E94577720E023
:1057D00030E040E05EE30E945777AB01BC0189EA0C
:1057E0009DE022E00E94C37089EA9DE06AE00E9489
:1057F00020126D817E818F81988523EC35EF48EAF8
:105800005EE30E9457777B018C016DA525EB3BE0A1
:105810003CAB2BAB0CC089EA9DE00E9420124BA947
:105820005CA94F5F5F4F5CAB4BABFA0164916623A1
:1058300091F789EA9DE06AE00E9420126EA52FEAA6
:105840003BE03CAB2BAB0CC089EA9DE00E942012F0
:105850004BA95CA94F5F5F4F5CAB4BABFA01649106
:10586000662391F789EA9DE0B801A70122E00E9432
:10587000C37089EA9DE06AE00E942012E9EAFBE039
:105880006491FCABEBAB0CC089EA9DE00E94201256
:105890002BA93CA92F5F3F4F3CAB2BABF901649187
:1058A000662391F7C801B701A60195010E947E7495
:1058B000AB01BC0189EA9DE022E00E94C37089EA45
:1058C0009DE06AE00E942012E3EAFBE06491FCABF9
:1058D000EBAB0CC089EA9DE00E9420122BA93CA9E9
:1058E0002F5F3F4F3CAB2BABF9016491662391F7DF
:1058F000C801B701A60195010E94577720E030E06A
:1059000040E450E40E947E74AB01BC0189EA9DE052
:1059100022E00E94C37089EA9DE06AE00E942012A2
:105920006D817E818F8198852DEC3CEC4CE45EE3AB
:105930000E9457777B018C01E4E9FBE06491FCABAA
:10594000EBAB0CC089EA9DE00E9420122BA93CA978
:105950002F5F3F4F3CAB2BABF9016491662391F76E
:1059600089EA9DE06AE00E942012EEE8FBE0649183
:10597000FCABEBAB0CC089EA9DE00E9420122BA986
:105980003CA92F5F3F4F3CAB2BABF90164916623E1
:1059900091F789EA9DE0B801A70122E00E94C37057
:1059A00089EA9DE06AE00E942012E8E8FBE0649149
:1059B000FCABEBAB0CC089EA9DE00E9420122BA946
:1059C0003CA92F5F3F4F3CAB2BABF90164916623A1
:1059D00091F7C801B701A80197010E949E73A60123
:1059E00095010E947E74AB01BC0189EA9DE022E032
:1059F0000E94C37089EA9DE06AE00E942012E2E8FA
:105A0000FBE06491FCABEBAB0CC089EA9DE00E942B
:105A100020122BA93CA92F5F3F4F3CAB2BABF901C8
:105A20006491662391F7C801B701A60195010E9410
:105A3000577720E030E040E450E40E947E74AB01F0
:105A4000BC0189EA9DE022E00E94C37089EA9DE0E2
:105A50006AE00E942012D201C101860D971DA81D87
:105A6000B91DB595A7959795879580932E03298D98
:105A70003A8D2F5F3F4F3A8F298FAF8CB8A0C9A0C6
:105A8000DAA011E001C010E06F8D78A189A19AA180
:105A900020E030E040EA51E40E949E739B01AC019B
:105AA0006FA578A989A99AA90E94857618166CF520
:105AB000E7E5FBE064918F0108C089EA9DE00E9460
:105AC00020120F5F1F4FF80164916623B1F789EA36
:105AD0009DE06AE00E942012E4960FB6F894DEBFC3
:105AE0000FBECDBFCF91DF911F910F91FF90EF902F
:105AF000DF90CF90BF90AF909F908F907F906F90EE
:105B00005F904F903F902F9008950FB6F89480913A
:105B1000A40D9091A50DA091A60DB091A70D0FBE5B
:105B20002D893E894F89588D821B930BA40BB50B91
:105B3000815D9740A040B04008F4CFCB0FB6F894F9
:105B40008091A40D9091A50DA091A60DB091A70DE7
:105B50000FBE8D8B9E8BAF8BB88FE1E5FBE0649120
:105B60007F0109C089EA9DE00E9420120894E11C8F
:105B7000F11CF70164916623A9F7809126039091A7
:105B800027030E94D224AB01BC0189EA9DE022E0F8
:105B90000E94C370EDE4FBE064917F0109C089EAD3
:105BA0009DE00E9420120894E11CF11CF701649111
:105BB0006623A9F740912E0350E0662757FD6095B4
:105BC000762F89EA9DE00E94B27089EA9DE06AE042
:105BD0000E94201282CB80917005882389F1409128
:105BE0006A0350916B0360916C0370916D03809117
:105BF0006E0590916F052EE633E080D5882311F174
:105C00004091710550917205609173057091740512
:105C1000411551056105710589F080916E059091DE
:105C20006F052EE633E06AD5882361F01092710586
:105C300010927205109273051092740510927005FF
:105C400081E0089580E00895DF92EF92FF920F9334
:105C50001F937B018C01D42E80916A0390916B037A
:105C6000A0916C03B0916D038E159F05A007B1073D
:105C7000B1F0B1DF8823D9F080916E0590916F0566
:105C8000B801A7012EE633E00ED6882381F0E0921A
:105C90006A03F0926B0300936C0310936D03DD2095
:105CA00011F481E005C081E08093700501C080E0BF
:105CB0001F910F91FF90EF90DF9008958F929F9228
:105CC000AF92BF92CF92DF92EF92FF920F931F930A
:105CD000CF93DF936C01142F70936F0560936E0563
:105CE000FC01178A82E090E0A0E0B0E0808391831D
:105CF000A283B38310927005109271051092720501
:105D000010927305109274058FEF9FEFAFEFBFEF06
:105D100080936A0390936B03A0936C03B0936D031D
:105D2000442321F48824992454013FC0453008F0CD
:105D30001CC160E070E080E090E040E085DF8823F7
:105D400009F413C1C12FD0E02197FE0174E0EE0FDA
:105D5000FF1F7A95E1F7E259FC4FE254FE4F808134
:105D6000EE5BF14090E08F779070892B09F0FDC0D9
:105D7000E653FE4F80819181A281B38184369105E3
:105D8000A105B10508F4F1C064E0CC0FDD1F6A95F0
:105D9000E1F7CC5CDA4F88809980AA80BB808114BF
:105DA0009104A104B10409F4E0C0C501B40140E0CC
:105DB0004BDF882309F4D9C08091790390917A034D
:105DC0008050924009F0D1C020917E03222309F433
:105DD000CCC080917C0390917D03892B09F4C5C0D0
:105DE00080917B03882309F4C0C0F601228B809147
:105DF0007B038483158661E070E007C04F5FF60186
:105E000045874150483008F0B0C0F601458584818F
:105E100090E09B01042E02C0220F331F0A94E2F788
:105E20008217930759F72091840330918503211538
:105E3000310519F040E050E008C020919203309104
:105E400093034091940350919503F6012583368383
:105E500047835087E0907C03F0907D0300E010E0E2
:105E6000E80CF91C0A1D1B1DE38AF48A058B168BAE
:105E700080917F0390918003918F808F60917E034A
:105E800070E080E090E00E9429786E0D7F1D801FF9
:105E9000911FF601628F738F848F958F20917F03FE
:105EA0003091800355E0220F331F5A95E1F72150BE
:105EB0003E4F232F3327269540E050E0260F371F13
:105EC000481F591F26873787408B518B809181034C
:105ED00090918203009719F0A0E0B0E008C0809193
:105EE0008E0390918F03A0919003B091910385014F
:105EF0007401E21AF30A040B150BA8019701280F8D
:105F0000391F4A1F5B1FF601058404C0569547954B
:105F1000379527950A94D2F721873287438754878C
:105F2000253FFFE03F07F0E04F07F0E05F0720F478
:105F30008CE0F601878B19C0255F3F4F40405040F1
:105F400018F480E1F6010EC080919A0390919B03B2
:105F5000A0919C03B0919D03F601828F938FA48F33
:105F6000B58F80E2878B81E001C080E0DF91CF9127
:105F70001F910F91FF90EF90DF90CF90BF90AF9067
:105F80009F908F9008956F927F928F929F92AF9281
:105F9000BF92CF92DF92EF92FF920F931F93CF9316
:105FA000DF93EC015A016B01380149014230510580
:105FB0006105710508F45DC089859A85AB85BC854E
:105FC0000196A11DB11D84179507A607B70708F410
:105FD00050C08F89803129F4E52EF62E072F112726
:105FE0000CC0803209F045C07A018B0187E016951C
:105FF0000795F794E7948A95D1F78B899C89AD89A9
:10600000BE89E80EF91E0A1F1B1FC801B70141E037
:106010001BDE882371F18F89803149F4F501F0701E
:10602000EE0FFF1FE259FC4F718260820DC0F50137
:10603000EF77F070EE0FFF1FEE0FFF1FE259FC4FDE
:1060400060827182828293828A89823080F08D811F
:106050009E81AF81B885E80EF91E0A1F1B1FE092D2
:106060007105F0927205009373051093740581E039
:1060700001C080E0DF91CF911F910F91FF90EF90D1
:10608000DF90CF90BF90AF909F908F907F906F9058
:106090000895CF92DF92EF92FF920F931F93CF93C9
:1060A000DF93EC017A018B01690189859A85AB85C3
:1060B000BC850196A11DB11D84179507A607B707DA
:1060C00008F452C08F89803129F45527412F302F91
:1060D0002F2D0CC0803209F047C09A01AB0167E058
:1060E00056954795379527956A95D1F78B899C8961
:1060F000AD89BE89280F391F4A1F5B1F80916A0333
:1061000090916B03A0916C03B0916D032817390730
:106110004A075B0731F0CA01B90140E095DD8823E9
:1061200019F18F89803159F4F701F070EE0FFF1FDC
:10613000E259FC4F80819181A0E0B0E00EC0F701F0
:10614000EF77F070EE0FFF1FEE0FFF1FE259FC4FCD
:1061500080819181A281B381BF70F6018083918398
:10616000A283B38381E001C080E0DF91CF911F91D2
:106170000F91FF90EF90DF90CF900895AF92BF9274
:10618000CF92DF92EF92FF920F931F93DF93CF9303
:1061900000D000D0CDB7DEB76C017A018B0182E070
:1061A00090E0A0E0B0E0F60180839183A283B38306
:1061B0005E010894A11CB11CC601B801A70195019C
:1061C00068DF882339F1C601B801A70100E010E0BB
:1061D00020E030E0D8DE8823E9F0E980FA800B8106
:1061E0001C81F6018789803151F4F8EFEF16FFEF3B
:1061F000FF06F0E00F07F0E01F07F0F209C088EF9C
:10620000E8168FEFF8068FEF08078FE01807A0F267
:1062100081E001C080E00F900F900F900F90CF9120
:10622000DF911F910F91FF90EF90DF90CF90BF9083
:10623000AF9008954F925F926F927F928F929F924C
:10624000AF92BF92CF92DF92EF92FF920F931F9384
:10625000DF93CF9300D000D0CDB7DEB76C01498378
:106260005A836B837C833901EE24FF2487012E013E
:106270000894411C511C812CE2E09E2EA12CB12CD3
:1062800049815A816B817C81C601920102DF88239A
:1062900039F1D501C401F601058404C0880F991FA6
:1062A000AA1FBB1F0A94D2F7E80EF91E0A1F1B1F74
:1062B00029813A814B815C818789803131F4285F63
:1062C0003F4F40405040E0F205C0285F3F4F4F4FE6
:1062D0005F40B0F2F301E082F1820283138381E038
:1062E0000F900F900F900F90CF91DF911F910F9112
:1062F000FF90EF90DF90CF90BF90AF909F908F90E6
:106300007F906F905F904F9008952F923F924F92A1
:106310005F926F927F928F929F92AF92BF92CF9235
:10632000DF92EF92FF920F931F93DF93CF93CDB73E
:10633000DEB72F970FB6F894DEBF0FBECDBF1C019E
:106340004A875B876C877D873F872E87DC0119969C
:106350008D919D910D90BC91A02D0196A11DB11D17
:106360008E839F83A887B987F901008111812281DB
:106370003381011511052105310549F04801590105
:106380000894811C911CA11CB11C1D8210C0D1015C
:106390008D909D90AD90BC901D828A859B85AC852B
:1063A000BD850197A105B10511F491E09D837501AB
:1063B00064014424552432018E010F5F1F4FF10107
:1063C00081859285A385B485481659066A067B06A1
:1063D00008F08CC08E819F81A885B9858C159D059C
:1063E000AE05BF0550F4A2E08A2E912CA12CB12C51
:1063F000F2E0CF2ED12CE12CF12CC101B701A60186
:10640000980147DE882309F471C089819A81AB81A4
:10641000BC81A70196012F5F3F4F4F4F5F4F009701
:10642000A105B10519F049015A010DC02819390912
:106430004A095B098A859B85AC85BD852817390784
:106440004A075B0759F00894411C511C611C711CE0
:106450000894C11CD11CE11CF11CB1CFC101A601E3
:10646000B7010FEF1FEF2FEF3FE08DDD882391F491
:106470003DC02601370108944108510861087108A0
:10648000C101B301A201970186017DDD882371F16D
:10649000730162018C149D04AE04BF0450F3AE85F9
:1064A000BF854D915D916D917C91411551056105BF
:1064B000710531F0C1019501840165DD8823B1F0DA
:1064C000EE85FF8580829182A282B382FD81FF23C7
:1064D00059F00894811C911CA11CB11CD1018D9212
:1064E0009D92AD92BC92139781E001C080E02F96FF
:1064F0000FB6F894DEBF0FBECDBFCF91DF911F91D5
:106500000F91FF90EF90DF90CF90BF90AF909F9052
:106510008F907F906F905F904F903F902F90089555
:10652000FC014281242F30E0C90195958795806553
:106530008CBD40FF02C080E004C080E0463009F01E
:1065400081E08DBD8081E82FF0E00C948F6BDF92AD
:10655000EF92FF920F931F93CF93DF93EC01D62E10
:1065600079018A01DDDF0FB6F8948091A40D909136
:10657000A50DA091A60DB091A70D0FBE9C014FEFE8
:1065800010C00FB6F8948091A40D9091A50DA09124
:10659000A60DB091A70D0FBE821B930B8C5291409C
:1065A00038F44EBD0DB407FEFDCF8EB58F3F49F7D1
:1065B0008D2D80648EBD0DB407FEFDCF28E130E047
:1065C000D801C701022E04C0B695A7959795879567
:1065D0000A94D2F78EBD0DB407FEFDCF285030408F
:1065E0008FEF283F380761F7DD2011F485E906C0F9
:1065F00058E0D51611F487E801C08FEF8EBD0DB4B9
:1066000007FEFDCF8CE0D81631F48FEF8EBD0DB4B0
:1066100007FEFDCF8EB59FEF2FEF2EBD0DB407FE09
:10662000FDCF8EB587FF04C0992311F09150F5CFAF
:106630008B83DF91CF911F910F91FF90EF90DF90AF
:106640000895BF92CF92DF92EF92FF920F931F9324
:106650008C01B62E69017A0167E320E030E040E06A
:1066600050E075DFC8016B2DA701960170DF1F9107
:106670000F91FF90EF90DF90CF90BF900895FC01B5
:106680008081E82FF0E00C94896BDC016EBDFA018B
:1066900020E030E00DB407FEFDCF80818EBD0DB44B
:1066A00007FEFDCF81818EBD2E5F3F4F329682E087
:1066B0002030380779F70DB407FEFDCF8FEF8EBD80
:1066C0000DB407FEFDCF8FEF8EBD0DB407FEFDCFDD
:1066D0008FEF8EBD0DB407FEFDCF8EB513968C9354
:1066E00013978F71853011F481E0089583E111963D
:1066F0008C931197CD01C3DF80E00895CF92DF9294
:10670000EF92FF920F931F93CF93DF93EC017A01E7
:106710008B0169018C81833039F059E0EE0CFF1C4C
:10672000001F111F5A95D1F7CE0168E1A80197010A
:106730000EDF882311F086E036C0CE016EEFA60191
:10674000A4DF882389F10FB6F8948091A40D90916D
:10675000A50DA091A60DB091A70D0FBE9C014FEF06
:1067600010C00FB6F8948091A40D9091A50DA09142
:10677000A60DB091A70D0FBE821B930B88559240BA
:1067800040F44EBD0DB407FEFDCF1EB51F3F49F7C7
:1067900017C087E108C01EBD0DB407FEFDCF8EB542
:1067A0008823C1F086E18983CE0169DF80E0DF9133
:1067B000CF911F910F91FF90EF90DF90CF900895B0
:1067C000CE016DE020E030E040E050E0C0DE882304
:1067D00049F7E1CFCE0153DF81E0E9CFCF93DF93DB
:1067E000EC010FB6F8948091A40D9091A50DA091A5
:1067F000A60DB091A70D0FBEFC013FEF13C00FB661
:10680000F8948091A40D9091A50DA091A60DB09142
:10681000A70D0FBE8E1B9F0B8D52914018F02B833E
:1068200081E10BC03EBD0DB407FEFDCF2EB52F3F5D
:1068300031F32B832E3F31F08FE08983CE011FDFB0
:1068400080E02EC0DA011197452BD9F08FEF8EBD75
:1068500020E030E09FEF0BC00DB407FEFDCF8EB5FA
:10686000FB01E20FF31F80839EBD2F5F3F4F2A176E
:106870003B0790F30DB407FEFDCF8EB5A60FB71FF3
:106880008C938FEF8EBD0DB407FEFDCF8EB58FEFCD
:106890008EBD0DB407FEFDCF8EB5CE01F0DE81E0DA
:1068A000DF91CF910895CF92DF92EF92FF920F93F5
:1068B0001F93CF93DF93EC017A018B0169018C81E7
:1068C000833039F0A9E0EE0CFF1C001F111FAA95C0
:1068D000D1F7CE0161E1A801970139DE882331F0BB
:1068E00084E08983CE01CBDE80E005C0CE01B60115
:1068F00040E052E073DFDF91CF911F910F91FF9045
:10690000EF90DF90CF900895BF92CF92DF92EF92F9
:10691000FF920F931F93CF93DF93EC01B62E842F3A
:106920001C82198248830FB6F8942091A40D3091EF
:10693000A50D4091A60D5091A70D0FBE69010E94B3
:10694000756BCE019CDE23982B98229A219A269A69
:106950002E9A809180008F7D8093800085E08A83CD
:1069600082E58CBD1DBC80E09FEF9EBD0DB407FE8F
:10697000FDCF8F5F8A30C9F712C00FB6F8948091AF
:10698000A40D9091A50DA091A60DB091A70D0FBEDD
:106990008C199D09815D974010F081E05BC0CE01AC
:1069A00060E020E030E040E050E0D1DD182F8B8344
:1069B000813019F7CE0168E02AEA31E040E050E08A
:1069C000C6DD82FF02C01C8311C080E02FEF2EBD08
:1069D0000DB407FEFDCF9EB58F5F8430C1F79B835A
:1069E0009A3A11F082E036C082E08C838C8182304A
:1069F00021F0EE24FF24870118C0E12CF12C012D99
:106A000000E4102F12C00FB6F8948091A40D90915D
:106A1000A50DA091A60DB091A70D0FBE8C199D09D3
:106A2000815D974010F08AE015C0CE0169E2A801AF
:106A3000970107DE8B83882331F78C81823019F52B
:106A4000CE016AE320E030E040E050E080DD8823C2
:106A500029F088E08983CE0112DE20C08FEF8EBD41
:106A60000DB407FEFDCF8EB5807C803C11F483E031
:106A70008C8380E09FEF9EBD0DB407FEFDCF2EB549
:106A80008F5F8330C1F7CE01FADD86E08B1518F4F5
:106A900088E1898303C0BA8281E001C080E0DF9190
:106AA000CF911F910F91FF90EF90DF90CF90BF900B
:106AB0000895CF93DF930FB6F8948091A40D909131
:106AC000A50DA091A60DB091A70D0FBE80937906DC
:106AD00090937A06A0937B06B0937C06E091A20681
:106AE000F091A306EC55F94F8081882399F4E4E3F3
:106AF000FCE06491EF0107C089EA9DE00E9420124A
:106B00002196FE0164916623B9F789EA9DE06AE067
:106B10000E942012DF91CF9108958130910541F4B8
:106B20006F5F7F4F09F051C085E795E00C943812F4
:106B3000892B09F04AC06F5F7F4F09F046C088EC8F
:106B400092E090932406809323068091290688235F
:106B500021F086E296E00E94285288EC92E0909321
:106B6000E3058093E2058091E805882321F085EE16
:106B700095E00E94285288EC92E09093C50580939E
:106B8000C4058091CA05882321F087EC95E00E9416
:106B9000285288EC92E09093A7058093A6058091F7
:106BA000AC05882321F089EA95E00E94285288EC00
:106BB00092E0909387058093860580918C058823C9
:106BC00021F089E895E00C942852089580E090E047
:106BD0006FEF7FEFA2CF81E090E06FEF7FEF9DCF6F
:106BE000CF93DF93ECE0FCE06491EF0107C089EA0A
:106BF0009DE00E9420122196FE0164916623B9F760
:106C0000E3E1FCE06491EF0107C089EA9DE00E94A6
:106C100020122196FE0164916623B9F789EA9DE06E
:106C20006AE00E9420120E946D28779A769A479A0D
:106C3000439AF894DF91CF910895EF92FF920F93CA
:106C40001F930FB6F8948091A40D9091A50DA0917B
:106C5000A60DB091A70D0FBEE0907D06F0907E06C8
:106C600000917F06109180062091790630917A0676
:106C700040917B0650917C06821B930BA40BB50BB5
:106C8000E816F9060A071B0730F4E114F1040105C0
:106C9000110509F0A5DFE0904002F090410200915B
:106CA000420210914302E114F1040105110531F192
:106CB0000FB6F8948091A40D9091A50DA091A60D0A
:106CC000B091A70D0FBE2091790630917A064091C0
:106CD0007B0650917C06821B930BA40BB50BE81628
:106CE000F9060A071B0750F49091890D80918A0DCF
:106CF000981721F4779A769A479A439A0E94A35953
:106D00001F910F91FF90EF9008956F927F928F9255
:106D10009F92AF92BF92CF92DF92EF92FF920F932A
:106D20001F93F82E609181067091820680918306F0
:106D300090918406209185063091860640918706C1
:106D4000509188060E9492763B014C0160913C0272
:106D500070913D0200D000D000D00DB71EB70F5F7C
:106D60001F4F882777FD8095982F0E9419752091D5
:106D700044023091450240914602509147020E94E0
:106D8000577720E030E040E752E40E947E7420E034
:106D900030E048EC52E40E947E745B016C01F80123
:106DA0006082718282829382F482809177068583E9
:106DB0008BE596E06DE876E041E856E020E001E002
:106DC00032E0E32E0E94380E80918D0690918E065F
:106DD000A0918F06B091900680935B0690935C061D
:106DE000A0935D06B0935E06809191069091920605
:106DF000A0919306B091940680935F0690936006ED
:106E0000A0936106B09362068091950690919606D4
:106E1000A0919706B09198068093630690936406BC
:106E2000A0936506B09366068091990690919A06A4
:106E3000A0919B06B0919C0680936706909368068C
:106E4000A0936906B0936A060FB6F8948091A40DDA
:106E50009091A50DA091A60DB091A70D0FBE8093A6
:106E6000790690937A06A0937B06B0937C068DB743
:106E70009EB706960FB6F8949EBF0FBE8DBF1F91AA
:106E80000F91FF90EF90DF90CF90BF90AF909F90C9
:106E90008F907F906F900895CF92DF92EF92FF9244
:106EA0000F931F9360918D0670918E0680918F06CF
:106EB0009091900620E030E040E050E00E9477742E
:106EC000882364F480E090E0A0E0B0E080938D0639
:106ED00090938E06A0938F06B093900660919106D2
:106EE00070919206809193069091940620E030E094
:106EF00040E050E00E947774882364F480E090E0E2
:106F0000A0E0B0E08093910690939206A093930640
:106F1000B0939406609195067091960680919706BD
:106F20009091980620E030E040E050E00E947774B5
:106F3000882364F480E090E0A0E0B0E080939506C0
:106F400090939606A0939706B093980660918D064D
:106F500070918E0680918F069091900620E030E02F
:106F600044EC52E40E948576181664F480E090E0C8
:106F7000A4ECB2E480938D0690938E06A0938F06C6
:106F8000B09390066091910670919206809193065D
:106F90009091940620E030E04EEB52E40E9485761A
:106FA000181664F480E090E0AEEBB2E480939106B2
:106FB00090939206A0939306B093940660919506E1
:106FC00070919606809197069091980620E030E0A7
:106FD00040EF52E40E948576181664F480E090E059
:106FE000A0EFB2E48093950690939606A09397063F
:106FF000B09398060FB6F8948091A40D9091A50DCA
:10700000A091A60DB091A70D0FBE80937906909325
:107010007A06A0937B06B0937C0660913C02709147
:107020003D02882777FD8095982F0E941975209141
:1070300044023091450240914602509147020E941D
:10704000577720E030E040E752E40E947E7420E071
:1070500030E048EC52E40E947E747B018C018DE8A4
:1070600096E061E976E045E956E029E936E0E7E7B0
:10707000CE2EE6E0DE2E0E940E5F80918D0690916E
:107080008E06A0918F06B091900680935B06909338
:107090005C06A0935D06B0935E0680919106909188
:1070A0009206A0919306B091940680935F06909308
:1070B0006006A0936106B093620680919506909158
:1070C0009606A0919706B0919806809363069093D8
:1070D0006406A0936506B093660680919906909128
:1070E0009A06A0919B06B0919C06809367069093A8
:1070F0006806A0936906B0936A061F910F91FF90EE
:10710000EF90DF90CF900895CF93DF9389EA9DE0D1
:107110000E943C6EE7E3FCE06491EF0107C089EA5E
:107120009DE00E9420122196FE0164916623B9F72A
:107130004091A8065091A9066091AA067091AB06ED
:107140004F5F5F4F6F4F7F4F89EA9DE00E94B270A3
:1071500089EA9DE06AE00E942012ABDCDF91CF91CA
:1071600008954091A2065091A30620E630E0B901AF
:10717000469F9001479F300D569F300D1124682F78
:10718000772767FD7095C9018A54994F0E945C0B5F
:107190009C019093B1068093B00680E0232B09F008
:1071A00081E008950F931F93DF93CF93CDB7DEB7A0
:1071B000E0970FB6F894DEBF0FBECDBFDE0111968B
:1071C000E4EBF2E080E101900D928150E1F7DE0105
:1071D0005196E4EAF2E080E101900D928150E1F7EE
:1071E000DE019196E4E9F2E080E101900D92815098
:1071F000E1F789819A81AB81BC8180935D0890938E
:107200005E08A0935F08B093600889899A89AB896A
:10721000BC8980934D0890934E08A0934F08B0937B
:10722000500889A19AA1ABA1BCA180936D0890934D
:107230006E08A0936F08B09370088D819E81AF8116
:10724000B8858093610890936208A0936308B09317
:1072500064088D899E89AF89B88D80935108909379
:107260005208A0935308B09354088DA19EA1AFA1DA
:10727000B8A58093710890937208A0937308B09397
:10728000740889859A85AB85BC8580936508909341
:107290006608A0936708B0936808898D9A8DAB8DB6
:1072A000BC8D8093550890935608A0935708B093CF
:1072B000580889A59AA5ABA5BCA58093750890939D
:1072C0007608A0937708B09378088D859E85AF8562
:1072D000B8898093690890936A08A0936B08B0936B
:1072E0006C088D8D9E8DAF8DB8A1809359089093B9
:1072F0005A08A0935B08B0935C088DA59EA5AFA526
:10730000B8A98093790890937A08A0937B08B093EA
:107310007C0880E090E8ABE3B5E48093810890932B
:107320008208A0938308B093840880938508909383
:107330008608A0938708B093880820E030E040E0FA
:1073400050E020937D0830937E0840937F0850934F
:10735000800880E29EE4A0E0B0E08093490890932A
:107360004A08A0934B08B0934C082093950830939B
:107370009608409397085093980880E090E0A0EA20
:10738000B1E48093890890938A08A0938B08B09306
:107390008C088DEC9CECACECBEE380938D08909354
:1073A0008E08A0938F08B093900880E090E0A0EA48
:1073B000B0E48093910890939208A0939308B093BF
:1073C0009408EFE3FCE064918F0108C089EA9DE036
:1073D0000E9420120F5F1F4FF80164916623B1F7DE
:1073E00089EA9DE06EE571E00E94B21289EA9DE0B3
:1073F0006AE00E942012E0960FB6F894DEBF0FBE3E
:10740000CDBFCF91DF911F910F9108958091B0066C
:107410009091B106019660E070E04AE050E00C9473
:10742000F4098091B0069091B106019660E070E099
:107430000C949708AF92BF92CF92DF92EF92FF9297
:107440000F931F93CF93DF93FBE5EF2EF6E0FF2E14
:10745000CDE8D6E000E010E0F801EA5AFD4F808167
:1074600080DE882331F1DDDF5B016C01F801EC5A2D
:10747000F94F8081882311F061E002C060919D0680
:1074800070E0882777FD8095982F0E941975F70185
:1074900020813181428153810E9457779B01AC0149
:1074A000C601B5010E949E73688379838A839B839A
:1074B00009C0F70180819181A281B381888399837A
:1074C000AA83BB830F5F1F4F84E090E0E80EF91E94
:1074D00024960430110509F0BFCF86E442DE8823EC
:1074E000D9F09FDF7B018C0160939E0670939F060D
:1074F0008093A0069093A10620E030E040E050E0A9
:107500000E948576181644F4E0924402F0924502F7
:107510000093460210934702DF91CF911F910F9184
:10752000FF90EF90DF90CF90BF90AF90089582DFF3
:1075300089E417DE882349F074DF60938106709335
:10754000820680938306909384068AE40ADE882369
:1075500049F067DF609385067093860680938706FF
:107560009093880608952F923F924F925F926F9268
:107570007F928F929F92AF92BF92CF92DF92EF92C3
:10758000FF920F931F93DF93CF93CDB7DEB7A197F1
:107590000FB6F894DEBF0FBECDBF87E4E2DD8823CF
:1075A00009F4B7C43EDF0E94E6746430710581F1CE
:1075B0006530710554F46230710511F16330710565
:1075C00014F57723CCF40C940D4A6A35710509F44F
:1075D00041C46B35710534F46C31710511F00C94B4
:1075E0000D4A6DC06B35710509F438C46C357105F1
:1075F00011F00C940D4A37C41DDF4EDC0C94404A48
:1076000096DF81E002C093DF80E07FDB0C94404A8C
:1076100080E5A7DD882321F4EE24FF24870105C03F
:1076200000DF0E94EB747B018C0183E59ADD8823E7
:1076300059F0F7DE20E030E04AE754E40E94577743
:107640000E94EB747B018C010E94701B0FB6F894B2
:10765000A090A40DB090A50DC090A60DD090A70D40
:107660000FBEAE0CBF1CC01ED11E0FB6F894809189
:10767000A40D9091A50DA091A60DB091A70D0FBEE0
:107680008093790690937A06A0937B06B0937C064C
:1076900004C00E94F62581E0D0DA0FB6F8948091FC
:1076A000A40D9091A50DA091A60DB091A70D0FBEB0
:1076B0008A159B05AC05BD0560F30C940D4A8091BD
:1076C000440290914502A0914602B09147028093F6
:1076D000AC069093AD06A093AE06B093AF06809132
:1076E0003C0290913D02909359068093580684E69F
:1076F00090E090933D0280933C020FB6F894809105
:10770000A40D9091A50DA091A60DB091A70D0FBE4F
:107710008093790690937A06A0937B06B0937C06BB
:1077200081E00E94A01A80915B0690915C06A09176
:107730005D06B0915E0680938D0690938E06A093B1
:107740008F06B093900680915F0690916006A0919D
:107750006106B09162068093910690939206A09381
:107760009306B09394068091630690916406A0916D
:107770006506B09166068093950690939606A09351
:107780009706B09398068091670690916806A0913D
:107790006906B0916A068093990690939A06A09321
:1077A0009B06B0939C0680E090E0A0E0B0E0809360
:1077B000440290934502A0934602B093470288E5A5
:1077C000D0DC882351F489E5CCDC882331F48AE5C8
:1077D000C8DC882311F481E001C080E08093480276
:1077E000882329F488E5BDDC882309F4DAC00F2E4C
:1077F000F0E08F2EF0E09F2EF0E0AF2EF0E0BF2EF5
:10780000F02D80925B0690925C06A0925D06B0928D
:107810005E068BE596E06FE576E043E656E027E608
:1078200036E00E942A5A80E090E0A3E1B3EC809316
:107830008D0690938E06A0938F06B093900660916C
:107840002C0270912D0280912E0290912F02609354
:10785000440270934502809346029093470220E0D1
:1078600030E040E752E40E947E747B018C018DE899
:1078700096E061E976E045E956E029E936E0A7E7D8
:10788000CA2EA6E0DA2E0E940E5F0E94701B809224
:107890005B0690925C06A0925D06B0925E068BE558
:1078A00096E06FE576E043E656E027E636E00E9494
:1078B0002A5A80E090E0A0EAB0E480938D0690938D
:1078C0008E06A0938F06B09390066091440270914B
:1078D0004502809146029091470220E030E040E767
:1078E00052E40E947E747B018C018DE896E061E990
:1078F00076E045E956E029E936E00E940E5F0E94F5
:10790000701B80E090E0A0E2B1EC80938D06909334
:107910008E06A0938F06B093900660912C02709112
:107920002D0280912E0290912F0220E030E040E065
:107930005FE30E94577760934402709345028093FF
:1079400046029093470220E030E040E752E40E9474
:107950007E747B018C018DE896E061E976E045E973
:1079600056E029E936E00E940E5F0E94701B80926B
:107970005B0690925C06A0925D06B0925E068092D5
:107980008D0690928E06A0928F06B09290068092FD
:10799000440290924502A0924602B09247020E9491
:1079A000991A80914802882329F489E5DADB882333
:1079B00009F4DAC00F2EF0E08F2EF0E09F2EF0E0F9
:1079C000AF2EF0E0BF2EF02D80925F069092600601
:1079D000A0926106B09262068BE596E06FE576E0D4
:1079E00043E656E027E636E00E942A5A80E090E817
:1079F000AEE0B3EC8093910690939206A093930629
:107A0000B0939406609130027091310280913202FD
:107A10009091330260934402709345028093460232
:107A20009093470220E030E040E752E40E947E74E9
:107A30007B018C018DE896E061E976E045E956E04E
:107A400029E936E0F7E7CF2EF6E0DF2E0E940E5F41
:107A50000E94701B80925F0690926006A092610661
:107A6000B09262068BE596E06FE576E043E656E07D
:107A700027E636E00E942A5A80E090E0A0EAB0E4CF
:107A80008093910690939206A0939306B0939406E8
:107A900060914402709145028091460290914702A4
:107AA00020E030E040E752E40E947E747B018C01CC
:107AB0008DE896E061E976E045E956E029E936E0AF
:107AC0000E940E5F0E94701B80E090E0A0E2B1EC8B
:107AD0008093910690939206A0939306B093940698
:107AE00060913002709131028091320290913302A4
:107AF00020E030E040E05FE30E945777609344026B
:107B000070934502809346029093470220E030E054
:107B100040E752E40E947E747B018C018DE896E080
:107B200061E976E045E956E029E936E00E940E5F1A
:107B30000E94701B80925F0690926006A092610680
:107B4000B09262068092910690929206A09293065D
:107B5000B09294068092440290924502A09246020E
:107B6000B09247020E94991A80914802882329F412
:107B70008AE5F7DA882309F4DAC00F2EF0E08F2EB9
:107B8000F0E09F2EF0E0AF2EF0E0BF2EF02D8092BF
:107B9000630690926406A0926506B09266068BE535
:107BA00096E06FE576E043E656E027E636E00E9491
:107BB0002A5A80E090E0A4E3B3EC8093950690937A
:107BC0009606A0939706B093980660913402709140
:107BD000350280913602909137026093440270938F
:107BE0004502809346029093470220E030E040E750
:107BF00052E40E947E747B018C018DE896E061E97D
:107C000076E045E956E029E936E0E7E7CE2EE6E002
:107C1000DE2E0E940E5F0E94701B8092630690927F
:107C20006406A0926506B09266068BE596E06FE565
:107C300076E043E656E027E636E00E942A5A80E0E6
:107C400090E0A0E8BFE38093950690939606A093FA
:107C50009706B09398066091440270914502809116
:107C600046029091470220E030E040E752E40E9453
:107C70007E747B018C018DE896E061E976E045E950
:107C800056E029E936E00E940E5F0E94701B80E0FA
:107C900090E0A0E0B0EC8093950690939606A093B8
:107CA0009706B093980660913402709135028091E6
:107CB00036029091370220E030E040E05FE30E941E
:107CC00057776093440270934502809346029093E5
:107CD000470220E030E040E752E40E947E747B01DE
:107CE0008C018DE896E061E976E045E956E029E906
:107CF00036E00E940E5F0E94701B80926306909295
:107D00006406A0926506B0926606809295069092EF
:107D10009606A0929706B09298068092440290929E
:107D20004502A0924602B09247020E94991A88E545
:107D300018DA8823C9F06ADB6115710581059105A0
:107D400099F06FDB20916B0630916C0640916D06C7
:107D500050916E060E949E7360935B0670935C0662
:107D600080935D0690935E0689E5FBD98823C9F070
:107D70004DDB611571058105910599F052DB20916C
:107D80006F063091700640917106509172060E9404
:107D90009E7360935F067093600680936106909374
:107DA00062068AE5DED98823C9F030DB61157105EA
:107DB0008105910599F035DB2091730630917406A9
:107DC00040917506509176060E949E7360936306FB
:107DD0007093640680936506909366068BE596E043
:107DE0006FE576E043E656E027E636E00E942A5A41
:107DF00080E00E94A01A8091AC069091AD06A091FF
:107E0000AE06B091AF068093440290934502A093D2
:107E10004602B0934702809158069091590690937C
:107E20003D0280933C020FB6F8948091A40D90918E
:107E3000A50DA091A60DB091A70D0FBE8093790658
:107E400090937A06A0937B06B0937C060E94991AC1
:107E50000C940D4A10929D060C940D4A81E080937B
:107E60009D060C940D4A85E47CD9882311F40E9468
:107E7000701B7BE5E72E76E0F72E6BE6C62E66E0FC
:107E8000D62E00E010E0F801EA5AFD4F808169D952
:107E9000882389F1C6DAF60120813181428153813C
:107EA0000E949E73F7016083718382839383033002
:107EB00059F4B7DAF701608371838283938387E68D
:107EC00096E00E940D5A17C0ACDAF601208131818C
:107ED000428153810E949E73F70160837183828384
:107EE00093838BE596E06FE576E043E656E027E680
:107EF00036E00E942A5A0F5F1F4F44E050E0E40E24
:107F0000F51EC40ED51E0430110509F0BCCF0C942B
:107F10000D4A8DE426D9882311F40C94724981DA34
:107F20000E94E6746936710509F422C36A36710548
:107F30000CF070C06B31710509F47AC16C317105B8
:107F400084F56631710509F418C167317105BCF417
:107F50006231710509F427C66331710534F461316A
:107F6000710511F00C940D4AD3C06431710509F408
:107F7000D5C06531710511F00C940D4AF8C0683117
:107F8000710509F418C1683171050CF4FCC0693140
:107F9000710509F429C16A31710511F00C940D4A7B
:107FA00029C16235710509F4F7C563357105BCF463
:107FB0006E31710509F47EC16F31710534F46C3195
:107FC000710511F00C940D4A39C16F31710509F436
:107FD000B6C16A32710511F00C940D4A2BC2653599
:107FE000710509F429C66635710554F463357105C8
:107FF00009F4D5C56435710511F00C940D4AD3C54B
:108000006C35710509F42EC66836710511F00C94B3
:108010000D4A4FC26C3C710509F4D2C76D3C710525
:10802000A4F56337710509F43BC66437710594F410
:108030006B36710509F4ADC56B3671050CF481C55D
:108040006D36710509F420C36237710511F00C9487
:108050000D4A36C66E3B710509F4BFC46F3B71050E
:1080600054F46737710509F404C76C38710511F0D1
:108070000C940D4A6AC2693C710509F449C76B3C0E
:10808000710511F00C940D4A7DC751E06D327507F2
:1080900011F40C949D4881E06E327807ACF46E3C8C
:1080A000710511F40C945E486E3C71050CF4A8C780
:1080B0006C3D710511F40C947C486D3D710511F017
:1080C0000C940D4A0C948E4891E06039790711F4B4
:1080D0000C946949E1E061397E076CF4F1E06E329D
:1080E0007F0711F40C9456496F52714011F00C94B3
:1080F0000D4A0C945A4941E0653F740711F40C9401
:108100006C49665F714011F00C940D4A0C946E49F5
:1081100077987698479843980C940D4AEEE6FDE0E0
:1081200064918F0108C089EA9DE00E9420120F5FD0
:108130001F4FF80164916623B1F789EA9DE06AE078
:108140000E94201285E795E00E944F1AE0E6FDE0CC
:1081500064918F0108C089EA9DE00E9420120F5FA0
:108160001F4FF80164916623B1F70C94084A85E724
:1081700095E00E94B0160C940D4A85E795E00E94A8
:1081800092120C940D4A8091B0069091B10604961B
:108190006AE270E00E945C0BFC01009711F03197DD
:1081A00010826091B0067091B1066C5F7F4F85E7D9
:1081B00095E041E07BC085E795E00E9496120FB6FE
:1081C000F8948091A40D9091A50DA091A60DB09169
:1081D000A70D0FBE8093B2069093B306A093B4068A
:1081E000B093B5060C940D4A85E795E00E949D1268
:1081F0000C940D4A80917705882311F40C940D4A54
:1082000083E50E94B138882311F40C940D4AFED8FE
:10821000AB01BC014093490650934A0680934B063C
:1082200070934C0686E296E00E9411510C940D4A20
:1082300085E795E00E9458130C940D4A8091B00692
:108240009091B10604966AE270E00E945C0B8C018A
:10825000009719F12091A2063091A30680E690E0E4
:10826000AC01249FC001259F900D349F900D1124D7
:108270008A54994F6EE470E00E945C0B60E270E0FB
:108280000E945C0B9C012F5F3F4F3093B1062093FF
:10829000B00601501040F80110826091B006709154
:1082A000B1066C5F7F4F85E795E040E00E94B71311
:1082B0000C940D4A80917705882311F40C940D4A93
:1082C00085E795E00E94D3128091B0069091B106A7
:1082D00004966AE270E00E945C0B8C01009719F131
:1082E0002091A2063091A30680E690E0AC01249F85
:1082F000C001259F900D349F900D11248A54994FF1
:108300006EE470E00E945C0B60E270E00E945C0B27
:108310009C012F5F3F4F3093B1062093B006015070
:108320001040F80110826091B0067091B1066C5F48
:108330007F4F85E795E00E9482150C940D4A0FB699
:10834000F8946091A40D7091A50D8091A60D909167
:10835000A70D0FBE609336087093370880933808D6
:10836000909339082091B2063091B3064091B4063B
:108370005091B506621B730B840B950B28EE33E00E
:1083800040E050E00E945B78F22EE32ED42EC52E02
:108390004DB75EB7485050400FB6F8945EBF0FBE61
:1083A0004DBF0DB71EB70F5F1F4FCE010196EDB742
:1083B000FEB79283818386E791E0F80193838283FD
:1083C0006F2D7E2D8D2D9C2D2CE330E040E050E074
:1083D0000E945B78F801358324836F2D7E2D8D2DCF
:1083E0009C2D2CE330E040E050E00E945B78F801E7
:1083F000778366830E94A50BEFE3FCE064918F0115
:108400004DB75EB7485F5F4F0FB6F8945EBF0FBEC3
:108410004DBF08C089EA9DE00E9420120F5F1F4FE8
:10842000F80164916623B1F789EA9DE0BE016F5FB0
:108430007F4F8AC783E50E94B138882309F4EDC7CE
:108440000E94113A7B018C0180E50E94B13888239B
:1084500009F4E3C7C801B7010E94E6746B0177FF16
:1084600001C0DBC76F3F710511F00CF0D6C70E9449
:10847000113A0E94E6747B01EAE5F2E08081918185
:108480008E159F0509F4C9C7329622E0EE3CF2072B
:10849000A9F7F7FE01C0C1C78E2D0E94756BEE2DA6
:1084A000F0E00C2C0E94866B8E2DB6010E94306D80
:1084B000B4C78091770680933A0884E50E94B1386A
:1084C0008823E1F00E94113A0E94EB7460933A080D
:1084D0006623A1F0EFE3FCE064918F0108C089EA14
:1084E0009DE00E9420120F5F1F4FF80164916623E8
:1084F000B1F789EA9DE065E871E0EAC083E50E9492
:10850000B1388823F9F00E94113A6B017C01B090D8
:108510003A080B2D10E00E94E674DC01CB016B2DB4
:108520000E94A527000F111FF801EE5DFC4F9183FB
:108530008083000F111F065D1C4FF801C082D1829D
:10854000E282F3820E94DA2368C783E50E94B13891
:10855000882309F462C70E94113A0E94E674DC0184
:10856000CB010E94D223909325038093240355C707
:108570008091770680933A0884E50E94B138882379
:10858000E1F00E94113A0E94EB7460933A0866236E
:10859000A1F0EFE3FCE064918F0108C089EA9DE05F
:1085A0000E9420120F5F1F4FF80164916623B1F7FC
:1085B00089EA9DE06CE971E08BC0EAE5FDE0649139
:1085C0008F0108C089EA9DE00E9420120F5F1F4FB3
:1085D000F80164916623B1F760913A08E62FF0E064
:1085E000EE0FFF1FEA5DFC4F808191810E94D22433
:1085F000AB01BC0189EA9DE022E00E94C370E6E580
:10860000FDE064918F0108C089EA9DE00E9420127C
:108610000F5F1F4FF80164916623B1F78091280323
:10862000909129030E94D523AB01BC0189EA9DE00A
:1086300022E00E94C370E2E5FDE064918F0108C072
:1086400089EA9DE00E9420120F5F1F4FF80164919C
:108650006623B1F780913A0890E00E94CC23AC01E8
:10866000662757FD6095762F89EA9DE00E94B270DB
:1086700089EA9DE063EB71E00E94B21289EA9DE015
:108680006AE00E942012FCC68091770680933A0827
:1086900084E50E94B138882349F10E94113A0E9472
:1086A000EB7460933A08662309F1EFE3FCE0649110
:1086B0008F0108C089EA9DE00E9420120F5F1F4FC2
:1086C000F80164916623B1F789EA9DE064EB71E0FB
:1086D0000E94B21240913A0850E060E070E089EAEE
:1086E0009DE02AE000E00E94277092C683E50E9488
:1086F000B1388823F9F00E94113A6B017C01B090E7
:108700003A080B2D10E00E94E674DC01CB016B2DC2
:108710000E94A527000F111FF801EE5DFC4F918309
:108720008083000F111F065D1C4FF801C082D182AB
:10873000E282F3820E94DA230FB6F8946090A40DCF
:108740007090A50D8090A60D9090A70D0FBEE091A2
:108750003A08F0E0EE0FFF1FDF01AE5DBC4F2D9039
:108760003C90EA5DFC4F40805180AA24AA94BA2C28
:108770006501EFE4FDE024912F8FEBE4FDE04491EF
:1087800048A3E7E4FDE0549159A311C16F8D0FE4B4
:108790001DE008C089EA9DE00E9420120F5F1F4F74
:1087A000F80164916623B1F760913A08E62FF0E092
:1087B000EE0FFF1FEA5DFC4F808191810E94D22461
:1087C000AB01BC0189EA9DE022E00E94C37068A170
:1087D0000BE41DE008C089EA9DE00E9420120F5FB3
:1087E0001F4FF80164916623B1F740913A0850E0B9
:1087F000662757FD6095762F89EA9DE00E94B2704A
:1088000069A107E41DE008C089EA9DE00E942012EA
:108810000F5F1F4FF80164916623B1F7D7FC24C0A6
:108820000FB6F8942091A40D3091A50D4091A60D9E
:108830005091A70D0FBEC601B501605F784D8F4FF7
:108840009F4F621B730B840B950B28EE33E040E0C7
:1088500050E00E945B7889EA9DE0BA01A9012AE014
:1088600000E00E94277006C089EA9DE06BEC71E091
:108870000E94B21289EA9DE06AE00E9420120FB6BF
:10888000F8946090A40D7090A50D8090A60D909026
:10889000A70D0FBE0E94F62581E00E941D36FFEF56
:1088A000AF16FFEFBF06FFEFCF06FFEFDF0631F594
:1088B000E0913A08421453048CF4F0E0EE0FFF1FED
:1088C000DF01AA5DBC4FEE5DFC4F208131818D91AF
:1088D0009C91821793070CF043C04DC0F0E0EE0F5F
:1088E000FF1FDF01AA5DBC4FEE5DFC4F208131818F
:1088F0008D919C91281739079CF53DC0D7FC3BC052
:1089000060913A08E62FF0E0EE0FFF1FEA5DFC4FA2
:10891000808191810E94D2247B018C0160913A0870
:10892000E62FF0E0EE0FFF1FEE5DFC4F808191819E
:108930000E94D2249B01AC01C801B7010E949D7323
:108940000E94E67497FF07C0909580957095619599
:108950007F4F8F4F9F4F64307105810591055CF00B
:108960000FB6F894A090A40DB090A50DC090A60DE0
:10897000D090A70D0FBE2FEFA2162FEFB2062FEF4C
:10898000C2062FEFD20699F0D7FC4AC50FB6F8946D
:108990008091A40D9091A50DA091A60DB091A70D69
:1089A0000FBE8A199B098051974208F039C50FB64E
:1089B000F8948091A40D9091A50DA091A60DB09171
:1089C000A70D0FBE86199709A809B909895E9340BA
:1089D000A040B04008F0DACE5DCF83E50E94B13808
:1089E000882361F00E94113A0E94E674DC01CB01F9
:1089F0000E94D22390932503809324030FB6F8940A
:108A0000E090A40DF090A50D0091A60D1091A70D7A
:108A10000FBEE4E4FDE09490E0E4FDE0A490ECE31C
:108A2000FDE0B49081C00FB6F8948091A40D9091B0
:108A3000A50DA091A60DB091A70D0FBE8E199F098F
:108A4000A00BB10B895E9340A040B04008F467C012
:108A500060917706E62FF0E0EE0FFF1FEA5DFC4F16
:108A6000808191810E94D2246B017C01692D04E4F4
:108A70001DE008C089EA9DE00E9420120F5F1F4F91
:108A8000F80164916623B1F789EA9DE0B701A60178
:108A900022E00E94C3706A2D00E41DE008C089EA4C
:108AA0009DE00E9420120F5F1F4FF8016491662322
:108AB000B1F74091770650E0662757FD6095762F15
:108AC00089EA9DE00E94B2706B2D0CE31DE008C0A6
:108AD00089EA9DE00E9420120F5F1F4FF801649108
:108AE0006623B1F780912803909129030E94D52332
:108AF000AB01BC0189EA9DE022E00E94C37089EAD3
:108B00009DE06AE00E9420120FB6F894E090A40D58
:108B1000F090A50D0091A60D1091A70D0FBE0E941B
:108B2000F62581E00E941D36209124033091250313
:108B30008091280390912903821793070CF473CF37
:108B400082C483E50E94B1388823F9F00E94113A6B
:108B500020E030E040E050E00E947774882314F475
:108B600060E010C00E94113A20E030E04FE753E48B
:108B70000E948576181614F46FEF04C00E94113A13
:108B80000E94EB746093780648C48FEF8093780658
:108B900044C41092780641C4109257063EC481E046
:108BA000809357063AC483E50E94B138882399F030
:108BB0000E94113A20E030E04AE754E40E945777DF
:108BC0000E94EB74609340027093410280934202D2
:108BD0009093430222C488E50E94B138882309F0AB
:108BE00046C489E50E94B138882309F040C48AE56B
:108BF0000E94B138882309F03AC485E40E94B13854
:108C0000882309F034C40E94701B439A0E947D1B84
:108C100004C4779A89E50E94B1388111769A8AE571
:108C20000E94B1388111479A85E40E94B1388823A7
:108C300009F4F3C3439AF1C383E50E94B1380E945B
:108C4000113A20E030E04AE754E40E9457770E944E
:108C5000EB7460937D0670937E0680937F069093FD
:108C60008006DBC306E512E08DE5E82E88E0F82EED
:108C7000F80180810E94B138882339F00E94113AAE
:108C8000F70160837183828393830F5F1F4F44E0FA
:108C900050E0E40EF51E52E00A35150749F7BDC352
:108CA000EAE8FCE064918F0108C089EA9DE00E9437
:108CB00020120F5F1F4FF80164916623B1F7ADC317
:108CC000E7E8FCE064918F0108C089EA9DE00E941A
:108CD00020120F5F1F4FF80164916623B1F7409196
:108CE0005B0650915C0660915D0670915E0689EAB4
:108CF0009DE022E00E94C370E4E8FCE064918F01F3
:108D000008C089EA9DE00E9420120F5F1F4FF80102
:108D100064916623B1F740915F06509160066091BF
:108D200061067091620689EA9DE022E00E94C370AC
:108D3000E1E8FCE064918F0108C089EA9DE00E94AF
:108D400020120F5F1F4FF80164916623B1F7409125
:108D5000630650916406609165067091660689EA23
:108D60009DE022E00E94C370EEE7FCE064918F0179
:108D700008C089EA9DE00E9420120F5F1F4FF80192
:108D800064916623B1F7409167065091680660913F
:108D9000690670916A0689EA9DE022E00E94C3702C
:108DA000E4E7FCE064918F0108C089EA9DE00E943D
:108DB00020120F5F1F4FF80164916623B1F780E026
:108DC0000E943B1B0E94197520915D0830915E083E
:108DD00040915F08509160080E947E74AB01BC0115
:108DE00089EA9DE022E00E94C370E1E7FCE0649123
:108DF0008F0108C089EA9DE00E9420120F5F1F4F7B
:108E0000F80164916623B1F781E00E943B1B0E9448
:108E10001975209161083091620840916308509162
:108E200064080E947E74AB01BC0189EA9DE022E0E7
:108E30000E94C370EEE6FCE064918F0108C089EAED
:108E40009DE00E9420120F5F1F4FF801649166237E
:108E5000B1F782E00E943B1B0E94197520916508C2
:108E60003091660840916708509168080E947E74AE
:108E700011C2E7E6FCE064918F0108C089EA9DE039
:108E80000E9420120F5F1F4FF80164916623B1F713
:108E9000639903C06DEC71E002C060ED71E089EA96
:108EA0009DE00E94B212E0E6FCE064918F0108C0F0
:108EB00089EA9DE00E9420120F5F1F4FF801649124
:108EC0006623B1F7189B03C06DEC71E002C060ED42
:108ED00071E089EA9DE00E94B212E9E5FCE064914C
:108EE0008F0108C089EA9DE00E9420120F5F1F4F8A
:108EF000F80164916623B1F7649903C06DEC71E0E9
:108F000002C060ED71E089EA9DE00E94B212C9C121
:108F100016E5C12E12E0D12EEE24FF24F601808149
:108F20000E94B138882309F10E94113A8701035940
:108F3000174F0E94EB74F8016083718382839383DF
:108F40000E94113A87010756174FF701E35AF74F6E
:108F500020813181428153810E9457770E94EB74B6
:108F6000F80160837183828393830894C11CD11CB0
:108F700044E050E0E40EF51E5AE5C51652E0D50671
:108F800069F64BC206E512E0BDE4EB2EB8E0FB2E1D
:108F9000F80180810E94B138882339F00E94113A8B
:108FA000F70160837183828393830F5F1F4F44E0D7
:108FB00050E0E40EF51E52E00A35150749F72DC2C0
:108FC00083E50E94B138882351F00E94113A6093E2
:108FD000810870938208809383089093840884E5C5
:108FE0000E94B138882309F418C20E94113A609394
:108FF00085087093860880938708909388080DC22F
:1090000083E50E94B138882351F00E94113A6093A1
:109010007D0870937E0880937F089093800884E594
:109020000E94B138882351F00E94113A609395084C
:1090300070939608809397089093980882E40E9412
:10904000B138882361F00E94113A0E94EB7460935A
:10905000490870934A0880934B0890934C0888E520
:109060000E94B138882351F00E94113A6093890818
:1090700070938A0880938B0890938C088AE50E94ED
:10908000B138882351F00E94113A60938D08709393
:109090008E0880938F089093900885E40E94B138E1
:1090A000882309F4BAC10E94113A60939108709321
:1090B00092088093930890939408AFC106E512E05C
:1090C000ABE6EA2EA6E0FA2EF80180810E94B138C4
:1090D000882339F00E94113AF701608371838283FB
:1090E00093830F5F1F4F44E050E0E40EF51E52E003
:1090F0000935150749F791C183E50E94B1388823E6
:1091000009F48BC10E94113A0E94E67470933D02EB
:1091100060933C0281E080935A067FC183E50E9400
:10912000B138882309F479C10E94113A0E94E6748B
:1091300070933F0260933E0270C180E50E94B13897
:10914000882351F00E94113A6093190270931A0219
:1091500080931B0290931C0289E40E94B1388823FB
:1091600081F00E94113A2DEB37E346E05EE30E9466
:10917000577760931D0270931E0280931F02909395
:10918000200284E40E94B138882381F00E94113AC1
:109190002DEB37E346E05EE30E947E74609321028C
:1091A00070932202809323029093240283E40E940E
:1091B000B138882351F00E94113A609325027093D0
:1091C000260280932702909328020E94B52389EA01
:1091D0009DE063ED71E00E94B21289EA9DE066EDC8
:1091E00071E00E94B2124091190250911A026091EE
:1091F0001B0270911C0289EA9DE022E00E94C3706C
:1092000089EA9DE06AED71E00E94B21260911D0250
:1092100070911E0280911F02909120022DEB37E386
:1092200046E05EE30E947E74AB01BC0189EA9DE0EA
:1092300022E00E94C37089EA9DE06EED71E00E9419
:10924000B2126091210270912202809123029091CA
:1092500024022DEB37E346E05EE30E945777AB0133
:10926000BC0189EA9DE022E00E94C37089EA9DE08A
:1092700062EE71E00E94B2126091250270912602A6
:1092800080912702909128022DEB37E346E05EE3C0
:109290000E945777AB01BC0189EA9DE022E00E9461
:1092A000C37089EA9DE063EB71E04EC081E00E94EB
:1092B0000A5AB3C083E50E94B138882329F460E0DC
:1092C00070E086E193E402C00E94113A0E94E12816
:1092D000A4C00E94701BA1C080E001C081E00E9478
:1092E000D2389BC084E50E94B138882309F450C06D
:1092F0000E94113A0E94EB7460933A08EFE3FCE09D
:10930000662329F164918F0108C089EA9DE00E94DB
:1093100020120F5F1F4FF80164916623B1F789EAAD
:109320009DE066EE71E00E94B21240913A0850E072
:1093300060E070E089EA9DE02AE000E00E9427708A
:1093400089EA9DE068EE71E00E94B21261C010925D
:10935000770664918F0108C089EA9DE00E9420127F
:109360000F5F1F4FF80164916623B1F789EA9DE012
:1093700069EF71E00E94B2124091770650E06627D3
:1093800057FD6095762F89EA9DE00E94B27040C03B
:10939000EFE3FCE064918F0108C089EA9DE00E9440
:1093A00020120F5F1F4FF80164916623B1F7E7E4C5
:1093B000FCE064918F0108C089EA9DE00E942012C0
:1093C0000F5F1F4FF80164916623B1F72091A20649
:1093D0003091A30680E690E0289FB001299F700D90
:1093E000389F700D11246A54794F89EA9DE00E94DC
:1093F000B212E5E4FCE064918F0108C089EA9DE0C7
:109400000E9420120F5F1F4FF80164916623B1F78D
:1094100089EA9DE06AE00E9420120E94593530C01E
:109420000FB6F8948091A40D9091A50DA091A60D72
:10943000B091A70D0FBE8093B2069093B306A09390
:10944000B406B093B5060FB6F8948091A40D909130
:10945000A50DA091A60DB091A70D0FBE8093790622
:1094600090937A06A0937B06B0937C06D6CF0E9499
:10947000701B88E50E94B138882309F0CACBCACB9B
:10948000A1960FB6F894DEBF0FBECDBFCF91DF918E
:109490001F910F91FF90EF90DF90CF90BF90AF9012
:1094A0009F908F907F906F905F904F903F902F9004
:1094B00008953F924F925F926F927F928F929F9208
:1094C000AF92BF92CF92DF92EF92FF920F931F93D2
:1094D000DF93CF93CDB7DEB76E970FB6F894DEBFAC
:1094E0000FBECDBF20E6C22ED12CE1E9FDE0B49045
:1094F000AA24A394FAC12D3051F02A3341F080916F
:109500003C0890913D088F3591050CF4CAC1E0915B
:109510003C08F0913D08309709F4D1C2A0913F0872
:10952000B0914008AC9D7001AD9DF00CBC9DF00C5D
:109530001124EE0DFF1DEA54F94F108280913E0870
:10954000882309F0A9C110923E08AC55B94F1C926E
:1095500087010A54194FC8016EE470E00E945C0B49
:109560009C01009709F4FEC09093B1068093B00669
:109570002F5F3F4F201B310B2E0D3F1DC9018A5419
:10958000994F60E070E04AE050E00E94F409609377
:1095900041087093420880934308909344082091B7
:1095A000A8063091A9064091AA065091AB062F5FFC
:1095B0003F4F4F4F5F4F621773078407950709F4BA
:1095C00035C080913F08909140089C012C9DC001BE
:1095D0002D9D900D3C9D900D11248A54994F6BE068
:1095E00072E00E948B0B009709F5ECE0FCE06491BF
:1095F0007F0109C089EA9DE00E9420120894E11CC5
:10960000F11CF70164916623A9F7E4E0FEE06491A0
:109610007F0109C089EA9DE00E9420120894E11CA4
:10962000F11CF70164916623A9F777C080913F0888
:10963000909140088C9D80018D9D100D9C9D100D7A
:109640001124C8018A54994F6AE270E00E945C0BB1
:109650009C01009709F441C0FF2440E0C80102C00A
:10966000FE264F5FFC01E40FF11DEA54F94FE08143
:10967000EA32B1F73093B1062093B006C9010196E2
:1096800060E070E00E9497080E94E6742F2D30E0A1
:109690002617370709F455C0ECE0FCE064917F0120
:1096A00009C089EA9DE00E9420120894E11CF11C87
:1096B000F70164916623A9F7E6EEFDE064917F016E
:1096C00009C089EA9DE00E9420120894E11CF11C67
:1096D000F70164916623A9F720C0ECE0FCE06491F7
:1096E0007F0109C089EA9DE00E9420120894E11CD4
:1096F000F11CF70164916623A9F7EDEBFDE064919D
:109700007F0109C089EA9DE00E9420120894E11CB3
:10971000F11CF70164916623A9F74091A8065091C6
:10972000A9066091AA067091AB0689EA9DE00E94A5
:10973000B27089EA9DE06AE00E9420120E9484389B
:109740004AC08091410890914208A0914308B0918D
:1097500044088093A8069093A906A093AA06B09304
:10976000AB063EC0C8016AE270E00E945C0B009745
:1097700009F436C0ECE0FCE064917F0109C089EA9D
:109780009DE00E9420120894E11CF11CF7016491F5
:109790006623A9F7E4E9FDE064917F0109C089EA45
:1097A0009DE00E9420120894E11CF11CF7016491D5
:1097B0006623A9F74091A8065091A9066091AA06D0
:1097C0007091AB0689EA9DE00E94B27089EA9DE043
:1097D0006AE00E94201210923D0810923C0813C2C9
:1097E00080913F08909140088C9D70018D9DF00CF8
:1097F0009C9DF00C112487010A54194FC80167E49D
:1098000070E00E945C0B9C01009781F19093B1067F
:109810008093B0062F5F3F4F201B310B2E0D3F1D55
:10982000C9018A54994F60E070E00E9497080E9435
:10983000E67464307105D0F4809175058823B1F425
:109840006B2D91E9E92E9DE0F92E09C089EA9DE092
:109850000E9420120894E11CF11CF7016491662318
:10986000A9F789EA9DE06AE00E94201280913F08F2
:1098700090914008019664E070E00E9448789093CF
:10988000400880933F0880914508909146080196D2
:10989000909346088093450810923D0810923C082A
:1098A00024C02B3311F4A0923E0880913E088823F7
:1098B000E1F420913C0830913D0880913F0890915F
:1098C00040088C9DF0018D9DF00D9C9DF00D1124A4
:1098D000E20FF31FEA54F94F80913B0880832F5F1A
:1098E0003F4F30933D0820933C0889EA9DE00E9459
:1098F000D46D181619060CF081C18091450890911D
:10990000460804970CF07AC189EA9DE00E940D6E2A
:10991000282F80933B088A3009F0EDCDF8CD809157
:109920003C0890913D08892B09F41FC16CC14D3052
:1099300069F04A3359F080913C0890913D088F3589
:10994000910524F42F5F3F4F09F0EAC020914906AA
:1099500030914A0640914B0650914C068091410649
:1099600090914206A0914306B0914406281739070A
:109970004A075B0708F49CC0662D8EE7E82E8DE051
:10998000F82E09C089EA9DE00E9420120894E11C8B
:10999000F11CF70164916623A9F789EA9DE06AE06A
:1099A0000E9420120FB6F8946091A40D7091A50D3D
:1099B0008091A60D9091A70D0FBE6093360870930D
:1099C000370880933808909339082091B206309177
:1099D000B3064091B4065091B506621B730B840B1D
:1099E000950B28EE33E040E050E00E945B78F22EC9
:1099F000E32ED42EC52E2DB73EB7285030400FB6DB
:109A0000F8943EBF0FBE2DBF0DB71EB70F5F1F4F9F
:109A1000EDB7FEB7B282A182F801538242826F2D68
:109A20007E2D842F952F2CE330E040E050E00E9403
:109A30005B78F801358324836F2D7E2D8D2D9C2D31
:109A40002CE330E040E050E00E945B78F80177833F
:109A500066830E94A50B672D0FE3E02E0CE0F02E2D
:109A60002DB73EB7285F3F4F0FB6F8943EBF0FBEED
:109A70002DBF09C089EA9DE00E9420120894E11CD4
:109A8000F11CF70164916623A9F789EA9DE0B5010D
:109A90000E94B21289EA9DE06AE00E94201285E7E6
:109AA00095E00E94A21285E795E061E00E947C1794
:109AB00020913C0830913D082115310519F4109290
:109AC0003E08A1C080913F0890914008889DF00118
:109AD000899DF00D989DF00D1124E20FF31FEA54BB
:109AE000F94F1082FC01EC55F94F30822091450866
:109AF000309146082F5F3F4F30934608209345082A
:109B0000019664E070E00E9448789093400880934A
:109B10003F0810923E0810923D0810923C0838C051
:109B20004B3311F430923E0880913E08882381F532
:109B300020913C0830913D0880913F089091400869
:109B4000889DF001899DF00D989DF00D1124E20F84
:109B5000F31FEA54F94F80913B0880832F5F3F4FFA
:109B600030933D0820933C0813C010E6812E912CC1
:109B700033243394EEE7FDE064905E010894A11C69
:109B8000B11CB6E74B2EB1E05B2EEFE3FCE0749026
:109B90002091490630914A0640914B0650914C065F
:109BA0008091410690914206A0914306B0914406EF
:109BB000281739074A075B0730F5809145089091CF
:109BC0004608049704F580912E0690912F06A091E7
:109BD0003006B09131068093490690934A06A093CF
:109BE0004B06B0934C0686E296E060D69C01482F67
:109BF00080933B088A3009F09ACEA8CE80917605F2
:109C0000882309F08CCE6E960FB6F894DEBF0FBE97
:109C1000CDBFCF91DF911F910F91FF90EF90DF901B
:109C2000CF90BF90AF909F908F907F906F905F90FC
:109C30004F903F900895CF93DF9380914508909186
:109C4000460803970CF435DC85E795E060E00E9458
:109C50007C178091450890914608892B09F45FC0D4
:109C600080917505882309F442C02091A2063091A5
:109C7000A30680E690E0289FE001299FD00D389F41
:109C8000D00D1124CA54D94FCE0160E172E00E9478
:109C90008B0B0097A1F485E795E0BE010E94E812C6
:109CA000E8E4FEE06491EF0107C089EA9DE00E94CC
:109CB00020122196FE0164916623B9F712C085E750
:109CC00095E00E94D312E6E3FEE06491EF0107C045
:109CD00089EA9DE00E9420122196FE01649166238C
:109CE000B9F789EA9DE06AE00E94201202C00E9452
:109CF000B33A8091450890914608019790934608A1
:109D0000809345088091A2069091A306019664E095
:109D100070E00E9448789093A3068093A2060E9468
:109D2000F62581E00E941D360E94B022DF91CF917E
:109D30000895CF92DF92EF92FF920F931F93DF93DC
:109D4000CF9300D0CDB7DEB789EA9DE040E950ED72
:109D500063E070E00E94896FE9EFFEE064918F019B
:109D600008C089EA9DE00E9420120F5F1F4FF80192
:109D700064916623B1F789EA9DE06AE00E942012AF
:109D80003FE3C32E3CE0D32EF6016491860108C068
:109D900089EA9DE00E9420120F5F1F4FF801649135
:109DA0006623B1F784B7F82E80FF14C0E1EFFEE020
:109DB00064918F0108C089EA9DE00E9420120F5F24
:109DC0001F4FF80164916623B1F789EA9DE06AE0CC
:109DD0000E942012F1FE14C0E1EEFEE064918F01BA
:109DE00008C089EA9DE00E9420120F5F1F4FF80112
:109DF00064916623B1F789EA9DE06AE00E9420122F
:109E0000F2FE14C0E0EDFEE064918F0108C089EA23
:109E10009DE00E9420120F5F1F4FF801649166239E
:109E2000B1F789EA9DE06AE00E942012F3FE14C0B7
:109E3000E0ECFEE064918F0108C089EA9DE00E9499
:109E400020120F5F1F4FF80164916623B1F789EA72
:109E50009DE06AE00E942012F5FE14C0E0EBFEE0F7
:109E600064918F0108C089EA9DE00E9420120F5F73
:109E70001F4FF80164916623B1F789EA9DE06AE01B
:109E80000E94201214BEE7EAFEE064918F0108C030
:109E900089EA9DE00E9420120F5F1F4FF801649134
:109EA0006623B1F7EDE9FEE064918F0108C089EA0D
:109EB0009DE00E9420120F5F1F4FF80164916623FE
:109EC000B1F789EA9DE06AE00E942012F6016491F0
:109ED0000FE31CE008C089EA9DE00E9420120F5F9A
:109EE0001F4FF80164916623B1F7EDE8FEE064913D
:109EF0008F0108C089EA9DE00E9420120F5F1F4F6A
:109F0000F80164916623B1F7E2E8FEE064918F0105
:109F100008C089EA9DE00E9420120F5F1F4FF801E0
:109F200064916623B1F7E6E7FEE064918F0108C013
:109F300089EA9DE00E9420120F5F1F4FF801649193
:109F40006623B1F7E1E7FEE064918F0108C089EA7A
:109F50009DE00E9420120F5F1F4FF801649166235D
:109F6000B1F789EA9DE06AE00E942012F60164914F
:109F70000FE31CE008C089EA9DE00E9420120F5FF9
:109F80001F4FF80164916623B1F7E2E6FEE06491A9
:109F90008F0108C089EA9DE00E9420120F5F1F4FC9
:109FA000F80164916623B1F72091490230914A0289
:109FB000CE0101962115310519F4895B9D4002C03F
:109FC000821B930B9A83898349815A81662757FDA7
:109FD0006095762F89EA9DE00E94B270EBE4FEE086
:109FE00064918F0108C089EA9DE00E9420120F5FF2
:109FF0001F4FF80164916623B1F789EA9DE040EDB7
:10A0000054E060E070E00E94B27089EA9DE06AE08E
:10A010000E9420121092A4061092A5061092A60685
:10A020001092A70680E00E94D238EE24FF24870118
:10A030000756174FF701E359F74F6081718182810D
:10A0400093810E941775F701E35AF74F2081318100
:10A05000428153810E9457770E94EB74F80160831C
:10A0600071838283938384E090E0E80EF91E90E18F
:10A07000E916F104E1F60E9492280E944B5C0E94CE
:10A08000A91A0F900F90CF91DF911F910F91FF9020
:10A09000EF90DF90CF900895CF93DF93BC01809134
:10A0A00045089091460804970CF06AC020913F083B
:10A0B0003091400880E690E0AC01249FC001259FCC
:10A0C000900D349F900D11248A54994F0E94670B74
:10A0D000EFE3FCE06491EF0107C089EA9DE00E9494
:10A0E00020122196FE0164916623B9F7E1E0FFE0BA
:10A0F0006491EF0107C089EA9DE00E942012219639
:10A10000FE0164916623B9F720913F083091400821
:10A1100080E690E0289FB001299F700D389F700D58
:10A1200011246A54794F89EA9DE00E94B212EFEF40
:10A13000FEE06491EF0107C089EA9DE00E942012D1
:10A140002196FE0164916623B9F789EA9DE06AE0F1
:10A150000E94201280913F0890914008019664E08F
:10A1600070E00E9448789093400880933F08809167
:10A1700045089091460801969093460880934508BB
:10A18000DF91CF9108950F931F93CF93DF93DC015D
:10A19000EB018A0180E090E020E2FE01E80FF91F68
:10A1A000208301968B309105C1F757E040E024C031
:10A1B000622F2E3219F08CE09FE007C05A3051F127
:10A1C0005AE048E018C0321729F1FC010196349199
:10A1D0003323C9F75417F0F02132E0F02F37D0F4D1
:10A1E000822F81568A3110F4622F6052FE01E40FF3
:10A1F000F11D60834F5F11962C91222311F02F32B5
:10A20000B9F6F801B183A08390E08881803219F01B
:10A2100091E001C090E0892FDF91CF911F910F91C4
:10A2200008956F927F928F929F92AF92BF92CF923A
:10A23000DF92EF92FF920F931F93CF93DF93EC0186
:10A240007A018B012B81222309F480C089899A89A4
:10A25000AB89BC8984179507A607B70708F476C0B1
:10A2600085C0E114F1040105110551F41C821D8221
:10A270001E821F82188619861A861B8681E067C097
:10A28000288539854A855B85E98DFA8D858590E03D
:10A290000996215030404040504039014A01082E73
:10A2A00004C096948794779467940A94D2F72F5FAA
:10A2B0003F4F4F4F5F4F0894E108F1080109110922
:10A2C0005701680104C0D694C794B794A7948A959F
:10A2D000D2F70894E11CF11C011D111DA614B7044E
:10A2E000C804D90428F0211531054105510549F468
:10A2F0008D899E89AF89B88D8C839D83AE83BF8302
:10A3000016C0A618B708C808D90811C04C815D81CD
:10A310006E817F81898D9A8D94010E9449300894C5
:10A32000A108B108C108D108882331F40FC084E026
:10A33000882E912C8C0E9D1EA114B104C104D10451
:10A3400029F7E886F9860A871B8798CF80E0DF9196
:10A35000CF911F910F91FF90EF90DF90CF90BF9022
:10A36000AF909F908F907F906F900895223009F06A
:10A3700078CFE7CFCF93DF93EC018C859D85AE85B9
:10A38000BF8540E0611141E0BC01CD010E94242E57
:10A39000882319F420E030E00AC08889282F30E0B3
:10A3A00095E0220F331F9A95E1F722593C4FC901DE
:10A3B000DF91CF9108950F931F93CF93DF938C017B
:10A3C000FC0183818823D9F1818187FF35C0C801D1
:10A3D00061E0D0DFEC01009791F18881853E79F151
:10A3E000F8018381823040F481899289A389B489FC
:10A3F0008C8F9D8FAE8FBF8FF80185899689A78935
:10A40000B08D9B8F8A8FCD01AA27BB279D8B8C8B0C
:10A41000E0914708F0914808309751F0BE016A5E1C
:10A420007F4FCE0148960995888D998D9B8B8A8B9D
:10A43000F80181818F7781830E94EB2D04C081E038
:10A44000F801808380E0DF91CF911F910F910895F3
:10A450000F931F938C01AFDFF80113821F910F91AF
:10A460000895FC018381882311F0CF01F1CF089575
:10A470006F927F928F929F92AF92BF92CF92DF9214
:10A48000EF92FF920F931F93DF93CF9300D000D0F2
:10A49000CDB7DEB77C015A016B01DC0113968C91BC
:10A4A0001397813009F08EC011968C9181FF8AC07C
:10A4B0009DC00097A105B10511F481E084C0F701AA
:10A4C0006084718482849384C701B601A501A9DEEA
:10A4D000882309F477C0D70159968D919C915A979A
:10A4E000A114B104C104D10489F455964D915D9134
:10A4F0006D917C9158970E94BE30882309F462C008
:10A50000F701158A168A178A108E44C0D70114964F
:10A510004D915D916D917C9117979E012F5F3F4FFB
:10A520000E944930882309F44DC0D7015996ED9116
:10A53000FC915A9749815A816B817C81878980314E
:10A5400049F4483FBFEF5B07B0E06B07B0E07B0723
:10A5500048F020C0483F8FEF58078FEF68078FE023
:10A560007807C0F4CF010E94BE30882359F1D7018B
:10A5700014964D915D916D917C91179759968D919F
:10A580009C915A970FEF1FEF2FEF3FE00E94C32FD0
:10A590008823C1F0F701A18AB28AC38AD48A818153
:10A5A00080688183C70107DF882361F0B601A501B8
:10A5B0006A147B048C049D0410F4B401A301C70148
:10A5C00030DE01C080E00F900F900F900F90CF9180
:10A5D000DF911F910F91FF90EF90DF90CF90BF9090
:10A5E000AF909F908F907F906F900895F701818931
:10A5F0009289A389B48984179507A607B70708F03D
:10A6000058CFE0CFCF93DF93EC0140E050E060E023
:10A6100070E02EDF882361F0CE0161E0ABDEFC014B
:10A62000009731F085EE80831B820E94EB2D01C0E4
:10A6300080E0DF91CF9108952F923F924F925F92E9
:10A640006F927F928F929F92AF92BF92CF92DF9242
:10A65000EF92FF920F931F93CF93DF93EC012A01A8
:10A660008B81882309F4B6C0898180FFB3C0C8C03C
:10A6700025014E185F083B0174E0272E312C2C0E6B
:10A680003D1E4201A1C0288539854A855B856FEF53
:10A69000A62E61E0B62EA222B3228B8179018A0117
:10A6A00099E016950795F794E7949A95D1F7E98D77
:10A6B000FA8D823049F4428D538D648D758D4E0D27
:10A6C0005F1D601F711F3FC0D480DA94DE20A1148B
:10A6D000B104D9F4DD20C9F4211531054105510536
:10A6E00049F48D899E89AF89B88D8C839D83AE8313
:10A6F000BF830BC04C815D816E817F81CF01910151
:10A700000E944930882309F465C0E98DFA8D4C8197
:10A710005D816E817F814250504060407040058471
:10A7200004C0440F551F661F771F0A94D2F7868511
:10A730009785A089B189480F591F6A1F7B1F4D0D4E
:10A74000511D611D711D80E092E08A199B098401F1
:10A750008815990508F48C0182E00030180709F08B
:10A7600067C080916A0390916B03A0916C03B091D4
:10A770006D03481759076A077B0709F459C0809190
:10A780006E0590916F0593010E945334882349F41C
:10A7900021C0950122593C4FC301B901A8010E9473
:10A7A000480B600E711E980140E050E08885998545
:10A7B000AA85BB85820F931FA41FB51F8887998721
:10A7C000AA87BB87801A910A8114910409F05BCF94
:10A7D000A20102C04FEF5FEFCA01DF91CF911F913D
:10A7E0000F91FF90EF90DF90CF90BF90AF909F9030
:10A7F0008F907F906F905F904F903F902F90089533
:10A80000A988BA88CB88DC88E884F9840A851B8506
:10A810009A0140E050E0D601C5018E199F09A00BB6
:10A82000B10B281739074A075B0708F021CF23CF60
:10A83000CB01BA0140E00E94242E882309F0A9CF61
:10A84000C9CF0F931F93CF93DF938C01EB01FC01D2
:10A850008381823018F180859185A285B3858F71BF
:10A860009070A070B0700097A105B105B9F4C8014F
:10A87000BE0140E250E0E0DE8032910519F0892B04
:10A8800069F40EC08881882359F0853E81F38E32A9
:10A8900071F38B8583FDEBCF80E203C08FEF01C0A6
:10A8A00080E0DF91CF911F910F910895DF93CF93B7
:10A8B0000F92CDB7DEB7BE016F5F7F4F41E050E032
:10A8C000BBDE019719F02FEF3FEF03C08981282FDE
:10A8D00030E0C9010F90CF91DF910895EF92FF9280
:10A8E0000F931F93CF93DF93EC018B81823030F174
:10A8F000E884F9840A851B85CE01D8DF97FD1EC048
:10A9000088859985AA85BB854F96A11DB11D88872D
:10A910009987AA87BB87F5E016950795F794E79482
:10A92000FA95D1F72E2D30E02F703070E5E0220F30
:10A93000331FEA95E1F722593C4F02C020E030E096
:10A94000C901DF91CF911F910F91FF90EF90089572
:10A950000F931F93CF93DF93EC018B018B8188239F
:10A9600009F040C0FB018789803109F041C082E0D5
:10A970008B831D8A1E8A1F8A188E808D918DA0E080
:10A98000B0E025E0880F991FAA1FBB1F2A95D1F7B9
:10A99000898B9A8BAB8BBC8B13C083E08B83F801C4
:10A9A000428D538D648D758D4D8B5E8B6F8B788F43
:10A9B0009E012F5E3F4FC8010E941A31882391F0FB
:10A9C0001A8F098F81E089831C821D821E821F825B
:10A9D000188619861A861B861C861D861E861F866B
:10A9E000188A01C080E0DF91CF911F910F910895E7
:10A9F0008032C1F7D2CF1F93CF93DF93EC01142F96
:10AA0000262F30E0F90155E0EE0FFF1F5A95E1F7D0
:10AA1000E259FC4F8385817121F0842F827109F006
:10AA200067C080916A0390916B03A0916C03B09111
:10AA30006D038C879D87AE87BF87688BF90145E0E2
:10AA4000EE0FFF1F4A95E1F7E259FC4F8489958983
:10AA5000A0E0B0E0DC01992788278D8B9E8BAF8B1F
:10AA6000B88F228D338DA90160E070E0482B592BFF
:10AA70006A2B7B2B4D8B5E8B6F8B788F838590E061
:10AA800088719070009751F4848D958DA68DB78D47
:10AA9000898B9A8BAB8BBC8B81E00CC0409741F5C6
:10AAA0009E012F5E3F4F898D9A8D0E941A31882317
:10AAB000F9F084E08B83812F8F7089831C821D8243
:10AAC0001E821F82188619861A861B8614FF16C0DE
:10AAD000CE0140E050E060E070E0CADC882371F411
:10AAE00009C049895A896B897C89CE019ADB02C0E9
:10AAF0001B8280E0DF91CF911F91089515FDF1CF6A
:10AB000081E0F8CFCF93DF93EC019C012C5F3F4FA6
:10AB1000898D9A8D41E050E060E070E00E948531BF
:10AB20008823A1F08D899E89AF89B88D0097A105F2
:10AB3000B10559F48C819D81AE81BF818D8B9E8B37
:10AB4000AF8BB88F89818068898381E0DF91CF9155
:10AB500008952F923F924F925F927F928F929F9291
:10AB6000AF92BF92CF92DF92EF92FF920F931F931B
:10AB7000DF93CF9300D000D000D0CDB7DEB76C010B
:10AB8000162F072F5E834D83DC0113968C9113974C
:10AB9000813009F06CC111968C9181FF68C185C12B
:10ABA000F601418952896389748980859185A285DE
:10ABB000B38584179507A607B70729F0C60131DBCF
:10ABC000882309F454C1812F902F9C0119014D80D5
:10ABD0005E8012C1D6015996ED91FC915A97DA0127
:10ABE000C90149E0B695A795979587954A95D1F7FC
:10ABF00074807A9478228FEF882E81E0982E8222BA
:10AC00009322772009F052C08114910409F04EC0BC
:10AC1000D60114964D915D916D917C9117974115D8
:10AC200051056105710581F455968D919D910D90A9
:10AC3000BC91A02D0097A105B10561F1F6018483B7
:10AC40009583A683B78332C0CF019E012F5F3F4F0C
:10AC50000E944930882309F40AC129813A814B8135
:10AC60005C81D6015996ED91FC915A978789803184
:10AC700049F4283FBFEF3B07B0E04B07B0E05B076C
:10AC800070F008C0283FEFEF3E07EFEF4E07EFE010
:10AC90005E0728F0C60136DF882341F4E8C0D601FC
:10ACA00014962D933D934D935C93179780E092E01B
:10ACB0008819990952018415950508F45C01D6019B
:10ACC0005996ED91FC915A971496ED90FD900D9147
:10ACD0001C9117978EEF9FEFAFEFBFEFE80EF91EB5
:10ACE0000A1F1B1F058404C0EE0CFF1C001F111F50
:10ACF0000A94D2F786859785A089B189E80EF91E56
:10AD00000A1F1B1FE70CF11C011D111D90E0A91665
:10AD100092E0B90639F580916A0390916B03A09196
:10AD20006C03B0916D038E159F05A007B10771F4F8
:10AD3000109270058FEF9FEFAFEFBFEF80936A0324
:10AD400090936B03A0936C03B0936D0380916E0599
:10AD500090916F05B801A70191010E947E3388236D
:10AD6000B9F585C08114910419F5D60118962D9175
:10AD70003D914D915C911B9751968D919D910D90B8
:10AD8000BC91A02D281739074A075B0788F00E945D
:10AD9000EB2D882309F46BC081E080937005E0926D
:10ADA0006A03F0926B0300936C0310936D0308C069
:10ADB000C801B70141E00E94242E882309F457C03E
:10ADC000940122593C4FC901B101A5010E94480BD1
:10ADD000950140E050E0F60180859185A285B3851C
:10ADE000820F931FA41FB51F80879187A287B38707
:10ADF0002A0C3B1C4A185B08D60118962D913D91F0
:10AE00004D915C911B974114510409F0E3CE51968A
:10AE10008D919D910D90BC91A02D82179307A40751
:10AE2000B50748F4F601218B328B438B548B81811B
:10AE30008068818311C08091470890914808892BD0
:10AE400059F08D819E81892B39F0D60111968C9114
:10AE50001197806811968C93F601818183FF04C05D
:10AE6000C601A9DA882319F04D815E8105C081E011
:10AE7000D6018C934FEF5FEFCA0126960FB6F89478
:10AE8000DEBF0FBECDBFCF91DF911F910F91FF901D
:10AE9000EF90DF90CF90BF90AF909F908F907F907A
:10AEA0005F904F903F902F90089582FD79CE8BCE8A
:10AEB000DF92EF92FF920F931F93CF93DF93EC01FA
:10AEC00089899A89AB89BC89805E9F4FAF41B04028
:10AED00008F070C0CE0116DE882309F46BC00E9412
:10AEE000EB2D882309F466C0E98DFA8DEC80FD8096
:10AEF0000E811F818EEF9FEFAFEFBFEFE80EF91EBF
:10AF00000A1F1B1F058404C0EE0CFF1C001F111F2D
:10AF10000A94D2F786859785A089B189E80EF91E33
:10AF20000A1F1B1F81E080937005E0926A03F09274
:10AF30006B0300936C0310936D0380E092E0EEE6E8
:10AF4000F3E0DF019C011D9221503040E1F7DD2448
:10AF5000D39411C0B801A7014D0D511D611D711D84
:10AF600080916E0590916F052EE633E00E947E334E
:10AF7000882301F1D394E98DFA8D8481D81650F39A
:10AF800020E032E040E050E0058404C0220F331F8F
:10AF9000441F551F0A94D2F789899A89AB89BC89C5
:10AFA000820F931FA41FB51F898B9A8BAB8BBC8B11
:10AFB00081E001C080E0DF91CF911F910F91FF9060
:10AFC000EF90DF9008958F929F92AF92BF92CF92B1
:10AFD000DF92EF92FF920F931F93CF93DF936C0159
:10AFE000EB01942E852EA22E898D9A8DD6015A962C
:10AFF0009C938E935997CB0140E050E060E070E065
:10B0000010D9BB2437C0CE0169DCFC01009709F4DC
:10B0100090C055E016950795F794E7945A95D1F7A7
:10B020001E2D1F708081882311F0853EC9F4BB203E
:10B0300099F420916A0330916B0340916C03509115
:10B040006D03D6011C962D933D934D935C931F97F2
:10B0500050961C93BB24B3948081882359F418C064
:10B06000892D982DBF014BE050E00E943B0B0097CB
:10B0700009F46DC0E884F9840A851B8589899A8959
:10B08000AB89BC89E816F9060A071B0708F4BBCF91
:10B09000A6FE4FC0A1FE4DC0BB2049F0F6011089AD
:10B0A000C60161E067D9EC01009761F442C08B8171
:10B0B000823009F43EC0CE01FBDE8823D1F110E0DE
:10B0C000CEE6D3E080E2DE011D928A95E9F7DE014B
:10B0D000292D382DC901FC018BE001900D92815082
:10B0E000E1F7E0914708F0914808309739F0BE0148
:10B0F000625F7F4FCE014096099508C081E298E2D9
:10B10000998B888B80E098E09F878E8788899989C2
:10B110009B8B8A8B998F888F8E859F859F8B8E8B3B
:10B120000E94EB2D882329F0C601612F4A2D63DC94
:10B1300001C080E0DF91CF911F910F91FF90EF90C0
:10B14000DF90CF90BF90AF909F908F900895A7FE13
:10B15000EBCFEFCF2F923F924F925F926F927F9201
:10B160008F929F92AF92BF92CF92DF92EF92FF9217
:10B170000F931F93DF93CF93CDB7DEB7C654D04064
:10B180000FB6F894DEBF0FBECDBF3C016B01DE01F0
:10B19000AE5BBF4F11965C934E9325962FAF2597CC
:10B1A0001C861F861FA21AA66115710509F47CC0B2
:10B1B000FC018381882309F077C0FA0180818F32F6
:10B1C000F1F08601ECE0EE2EF12CEC0EFD1E72E4A7
:10B1D000A72EB12CAC0EBD1E4E010894811C911CF3
:10B1E0002796FFAEEEAE279767E2262E312C2C0E67
:10B1F0003D1E270123C01196B183A08301C0FD012C
:10B20000A081B1818C918F32B1F3D60113968C91CC
:10B21000139782508230A8F28E01095D1F4F599614
:10B220006D917C915A97C80193DB882359F63CC0F5
:10B23000342D252D8701832F922F7C01F5018081EC
:10B240009181B401A5010E94C350882329F42CC028
:10B250003196D501ED93FC93D501ED91FC91808160
:10B260008F32B1F38823B9F0C701B801A40121E0FE
:10B27000AADE8823C9F00C151D0511F0C801E8D815
:10B280002796EEADFFAD2797EE16FF0689F6C101B2
:10B29000322D292FCFCFC301B801A40125962FADA0
:10B2A000259791DE182F01C010E0CE018796D9D8DE
:10B2B000CE010C96D6D8812FCA5BDF4F0FB6F8941B
:10B2C000DEBF0FBECDBFCF91DF911F910F91FF90D9
:10B2D000EF90DF90CF90BF90AF909F908F907F9036
:10B2E0006F905F904F903F902F9008950F931F9312
:10B2F000DF93CF93CDB7DEB76B970FB6F894DEBF71
:10B300000FBECDBF9C01AB0119821C828E010F5F65
:10B310001F4FC801B90122E01DDF882311F410E09E
:10B3200003C0C8016FD9182FCE0101969AD8812F7A
:10B330006B960FB6F894DEBF0FBECDBFCF91DF91F5
:10B340001F910F91089590918A0D8091890D981702
:10B3500081F140918A0D242F30E08DE490E0289F08
:10B36000F001299FF00D389FF00D1124EF5FF64F8B
:10B37000308120E06DE470E016C0842F90E0869F5D
:10B38000F001879FF00D969FF00D1124EF5FF64FAF
:10B3900080819181A281B3810097A105B10509F057
:10B3A0002F5F4F5F4F708091890D481731F7E32F62
:10B3B00011C080917806882359F03E9A90E09093CE
:10B3C000990080939800809190008068809390000D
:10B3D00020E0E0E080917806882369F42223C9F414
:10B3E0003E9A109299001092980080919000806887
:10B3F000809390000895EE2361F03E9A8E2F90E0A6
:10B400009093990080939800809190008068809339
:10B410009000089580938B0D0895FC0160817181E7
:10B42000828193812091690830916A0840916B086C
:10B4300050916C080E9457770E9427776093B50857
:10B440007093B6088093B7089093B80885EB98E09E
:10B450000C942A1BAF92BF92CF92DF92EF92FF9291
:10B460000F931F93FC017B016A0159016081718177
:10B470008281938120915D0830915E0840915F0840
:10B48000509160080E9457770E94277709EA18E0D8
:10B490006093A9087093AA088093AB089093AC08B6
:10B4A000F7016081718182819381209161083091DF
:10B4B000620840916308509164080E9457770E9487
:10B4C00027776093AD087093AE088093AF08909390
:10B4D000B008F601608171818281938120916508B5
:10B4E0003091660840916708509168080E9457772C
:10B4F0000E94277728E0E22EF12CE00EF11E6093E7
:10B50000B1087093B2088093B3089093B408F50122
:10B5100060817181828193812091690830916A08EC
:10B5200040916B0850916C080E9457770E942777D2
:10B530009801245F3F4F6093B5087093B6088093DD
:10B54000B7089093B808C8010C5F1F4FB801A70156
:10B550000E94F01A80E090E0A0E0B0E080938C0DB3
:10B5600090938D0DA0938E0DB0938F0D8093900DC1
:10B570009093910DA093920DB093930D8093940DA1
:10B580009093950DA093960DB093970D8093980D81
:10B590009093990DA0939A0DB0939B0D80939C0D61
:10B5A00090939D0DA0939E0DB0939F0D1F910F91B1
:10B5B000FF90EF90DF90CF90BF90AF9008958F9263
:10B5C0009F92AF92BF92CF92DF92EF92FF920F9332
:10B5D0001F93CF93DF93EC016B01009709F45CC0DC
:10B5E0008FA9882309F058C0EEA0FFA008A519A5CF
:10B5F000FB01B6A0A7A090A481A4C801B7012B2D80
:10B600003A2D492D582D0E94777488230CF044C0A0
:10B61000C801B701A80197010E9457777B018C01EF
:10B620006AA97BA98CA99DA9905820E030E040E050
:10B6300050EC0E9457772EA53FA548A959A90E9412
:10B6400057779B01AC01C801B7010E949E730E940D
:10B65000C4777B018C016B2D7A2D892D982D970154
:10B66000A8010E947774882324F4EB2CFA2C092D6E
:10B67000182D6B2D7A2D892D982D9701A8010E94E8
:10B680007774882349F0C701D801F60186A397A3F0
:10B69000A0A7B1A781E086ABDF91CF911F910F9159
:10B6A000FF90EF90DF90CF90BF90AF909F908F90E2
:10B6B0000895EF92FF920F931F93CF93DF93F09033
:10B6C0008A0D00E010E020E030E04DE4E42E11C0EF
:10B6D000FE9CE0011124C754D74FC901B801AE0147
:10B6E0006EDF8F2D8F5F803109F480E0F82E980196
:10B6F0008E018091890DF81659F7C901B80140E013
:10B7000050E05DDFDF91CF911F910F91FF90EF909F
:10B710000895AF92BF92CF92DF92EF92FF920F9374
:10B720001F93CF93DF93EB018A016115710509F433
:10B7300066C04115510509F462C0DAA4CBA4BCA4CB
:10B74000ADA46EA17FA188A599A52D2D3C2D4B2DD3
:10B750005A2D0E947774882309F451C08FA9882339
:10B7600009F043C0F801E6A0F7A000A511A56D2DD2
:10B770007C2D8B2D9A2DA80197010E948576181695
:10B78000A4F5C801B701A80197010E9457777B0172
:10B790008C016AA97BA98CA99DA9905820E030E072
:10B7A00040E050EC0E9457772EA53FA548A959A923
:10B7B0000E9457779B01AC01C801B7010E949E739C
:10B7C0000E94C4777B018C016D2D7C2D8B2D9A2DD1
:10B7D0009701A8010E947774882324F4ED2CFC2C97
:10B7E0000B2D1A2DC701D80104C08D2D9C2DAB2D1A
:10B7F000BA2D8EA39FA3A8A7B9A781E08EABDF9136
:10B80000CF911F910F91FF90EF90DF90CF90BF905D
:10B81000AF900895CF92DF92FF920F93DF93CF9373
:10B8200000D0CDB7DEB78091890D8091890D209130
:10B830008A0D90E04096821B91098F70907004975A
:10B840000CF10091890D03500F70CC24DD2440E0F1
:10B8500050E06DE4F62E12C0802F002309F480E141
:10B86000082F01500F9DC00111248754974F9A83D0
:10B870008983B6014EDFA601C980DA8080918A0DE6
:10B88000081751F70F900F90CF91DF910F91FF9014
:10B89000DF90CF9008951092890D10928A0D80E16B
:10B8A000E9EAF8E0DF011D928A95E9F780E090E08F
:10B8B000A0E0B0E08093900D9093910DA093920D35
:10B8C000B093930D8093940D9093950DA093960D46
:10B8D000B093970D8093980D9093990DA0939A0D26
:10B8E000B0939B0D80939C0D90939D0DA0939E0D06
:10B8F000B0939F0D80938C0D90938D0DA0938E0D22
:10B90000B0938F0D08952F923F924F925F926F9256
:10B910007F928F929F92AF92BF92CF92DF92EF92DF
:10B92000FF920F931F93DF93CF93CDB7DEB7669748
:10B930000FB6F894DEBF0FBECDBF9E8B8D8B6A0114
:10B940007B0148015901DC01D8966D917D918D9163
:10B950009C91DB970E941775698B7A8B8B8B9C8BE4
:10B96000A70196010E9457770E9464740E94EB74AD
:10B970006D837E838F83988769897A898B899C8977
:10B98000A50194010E9457770E9464740E94EB7491
:10B9900069837A838B839C832D813E814F81588577
:10B9A000283731054105510540F448E750E060E093
:10B9B00070E04D835E836F83788769817A818B81A4
:10B9C0009C81683771058105910540F488E790E016
:10B9D000A0E0B0E089839A83AB83BC83AD89BE8944
:10B9E000AC5BBF4FAD90BD90CD90DC901397A4544D
:10B9F000B040BE8BAD8BDC966D917D918D919C910D
:10BA0000DF970E9417756D877E878F87988BC60199
:10BA1000B5010E9419751B012C0120E030E040E0C7
:10BA200050E00E947774882321F4E0E070E060E049
:10BA300028C069897A898B899C899B01AC010E9405
:10BA400057777B018C016D857E858F8598899B0159
:10BA5000AC010E9457779B01AC01C801B7010E945D
:10BA60009D737B018C01C201B101A20191010E9471
:10BA70009E739B01AC01C801B7010E947E74E62F42
:10BA8000692F2E2F372F482F562FB901CA010E9438
:10BA900064740E94E6743B014C01ED89FE89E05C10
:10BAA000FF4F60817181828193810E941775698740
:10BAB0007A878B879C8766277727CB016A197B0952
:10BAC0008C099D090E9419755B016C0120E030E032
:10BAD00040E050E00E947774882321F4E0E070E0B9
:10BAE00060E028C069857A858B859C859B01AC01C7
:10BAF0000E9457777B018C0169897A898B899C899F
:10BB00009B01AC010E9457779B01AC01C801B701B2
:10BB10000E949D737B018C01C601B501A6019501B0
:10BB20000E949E739B01AC01C801B7010E947E7404
:10BB3000E62F692F2E2F372F482F562FB901CA0114
:10BB40000E945475ED89FE89A088B188C288D38887
:10BB500086017501E618F708080919090E94E674BC
:10BB6000A8019701261B370B480B590B57FF71C0D3
:10BB7000C201B10120E030E040E050E00E94777463
:10BB8000882321F4E0E070E060E044C0C201B1012C
:10BB9000A20191010E949E737B018C01C601B50137
:10BBA0000E9417759B01AC01C801B7010E9457772D
:10BBB0007B018C016D857E858F8598899B01AC0109
:10BBC0000E9457779B01AC01C801B7010E949D7389
:10BBD0007B018C0169857A858B859C859B01AC01F5
:10BBE0000E9457779B01AC01C801B7010E949E7368
:10BBF0007B018C01C201B10120E030E040E850E45B
:10BC00000E9457779B01AC01C801B7010E947E7466
:10BC1000E62F692F2E2F372F482F562FB901CA0133
:10BC20000E9464740E94E674AC01CB01DA013C010D
:10BC30004D0197FE03C06624772443016A147B04F8
:10BC40008C049D0410F03501460120E030E040E016
:10BC500050E09FB7F8946D897E89645B7F4FDB016C
:10BC60008C91AC54B040BE8BAD8B882321F5FD0187
:10BC7000648A758A868A978A260D371D481D591D44
:10BC800058962D933D934D935C935B972D813E8108
:10BC90004F815885DC962D933D934D935C93DF97B0
:10BCA000A05CBF4F29813A814B815C812D933D93EC
:10BCB0004D935C9313979FBF66960FB6F894DEBFC3
:10BCC0000FBECDBFCF91DF911F910F91FF90EF90ED
:10BCD000DF90CF90BF90AF909F908F907F906F90AC
:10BCE0005F904F903F902F9008954F925F927F9278
:10BCF0008F929F92AF92BF92CF92DF92EF92FF927C
:10BD00000F931F93CF93DF9370908A0DC0E0D0E024
:10BD10007DE4472E512C45C02097A9F18EA9882398
:10BD200061F4849CF001859CF00D949CF00D11242D
:10BD3000E754F74F86A9882331F1EAA0FBA00CA1B4
:10BD40001DA16EA17FA188A599A5A80197010E94B8
:10BD50007E745B016C01849CF001859CF00D949CC9
:10BD6000F00D1124E754F74F66A177A180A591A5A6
:10BD7000A80197010E947E748B019C01CE01B6013F
:10BD8000A501C1DD1EAA739480E1781609F4772419
:10BD9000849CE001859CD00D949CD00D1124C75447
:10BDA000D74F872C992487FC90948091890D90E03F
:10BDB0008816990609F0B0CF2097E9F0EAA0FBA019
:10BDC0000CA11DA16EA17FA188A599A5A80197012D
:10BDD0000E947E745B016C0160E070E080E090E4A2
:10BDE000A80197010E947E748B019C01CE01B601CF
:10BDF000A50189DD1EAADF91CF911F910F91FF90C0
:10BE0000EF90DF90CF90BF90AF909F908F907F90FA
:10BE10005F904F900895FEDC4CDC67CF2F923F92ED
:10BE20004F925F926F927F928F929F92AF92BF924A
:10BE3000CF92DF92EF92FF920F931F93DF93CF93F6
:10BE4000CDB7DEB7C558D0400FB6F894DEBF0FBEF1
:10BE5000CDBF5C014B013A012901CE57DF4FE8828B
:10BE6000C258D040CD57DF4FF882C358D040CC578E
:10BE7000DF4F0883C458D040CB57DF4F1883C558D5
:10BE8000D040E296DFAECEAEE2978091890D8F5F13
:10BE9000803109F480E0282F332727FD309539AB16
:10BEA00028AB05C00E94F62581E00E941D368091D6
:10BEB0008A0D90E048A959A98417950799F3D501EF
:10BEC0006D917D918D919C9120915D0830915E08DE
:10BED00040915F08509160080E9457770E94277731
:10BEE000E0966CAF7DAF8EAF9FAFE097F4016081BD
:10BEF0007181828193812091610830916208409123
:10BF00006308509164080E9457770E942777AC9687
:10BF10006CAF7DAF8EAF9FAFAC97D3016D917D912C
:10BF20008D919C9120916508309166084091670839
:10BF3000509168080E9457770E942777A8966CAFA7
:10BF40007DAF8EAF9FAFA897F20160817181828132
:10BF500093812091690830916A0840916B08509153
:10BF60006C080E9457770E942777A4966CAF7DAF2C
:10BF70008EAF9FAFA4978091B5089091B608A0911D
:10BF8000B708B091B808A4962CAD3DAD4EAD5FADED
:10BF9000A497281739074A075B0709F45FC0609127
:10BFA0007706E62FF0E0EE0FFF1FEA5DFC4F808181
:10BFB00091810E94D22420E030E04AE253E40E94C2
:10BFC000777488230CF04AC080918B0D882309F088
:10BFD00045C0A4964CAD5DAD6EAD7FADA4974093CA
:10BFE000B5085093B6086093B7087093B808ECE1B1
:10BFF000FFE084918F017E010894E11CF11C0CC0CC
:10C00000898389EA9DE0B70141E050E00E94546EC7
:10C010000F5F1F4FF8018491882391F7E0E4FFE060
:10C0200084918F017E010894E11CF11C0CC089836E
:10C0300089EA9DE0B70141E050E00E94546E0F5F35
:10C040001F4FF8018491882391F78AE0898389EA58
:10C050009DE0B70141E050E00E94546E8091B50828
:10C060009091B608A091B708B091B808A4962CADED
:10C070003DAD4EAD5FADA497281B390B4A0B5B0B52
:10C08000CA01B90157FF07C09095809570956195D9
:10C090007F4F8F4F9F4F0E9419757B018C016091DC
:10C0A000690870916A0880916B0890916C0820E093
:10C0B00030E041E453E40E9457779B01AC01C80192
:10C0C000B7010E94857618160CF045C0A4964CADB9
:10C0D0005DAD6EAD7FADA4974093B5085093B608A3
:10C0E0006093B7087093B808ECE1FFE084918F018A
:10C0F0007E010894E11CF11C0CC0898389EA9DE053
:10C10000B70141E050E00E94546E0F5F1F4FF801ED
:10C110008491882391F7E2E2FFE084918F017E0110
:10C120000894E11CF11C0CC0898389EA9DE0B701E9
:10C1300041E050E00E94546E0F5F1F4FF801849160
:10C14000882391F78AE0898389EA9DE0B70141E07D
:10C1500050E00E94546E8091890D282F30E0A09607
:10C160003FAF2EAFA0978DE490E0289FF001299F6C
:10C17000F00D389FF00D1124E754F74FE45BFF4FAB
:10C180001082EC54F0404091A9085091AA086091A7
:10C19000AB087091AC086E964CAF5DAF6EAF7FAFE1
:10C1A0006E97E0968CAD9DADAEADBFADE097841BB4
:10C1B000950BA60BB70B6A968CAF9DAFAEAFBFAF1A
:10C1C0006A9780839183A283B383B7FF0BC0B09536
:10C1D000A095909581959F4FAF4FBF4F80839183DE
:10C1E000A283B3832091AD083091AE084091AF088F
:10C1F0005091B00866962CAF3DAF4EAF5FAF6697DB
:10C20000AC966CAD7DAD8EAD9FADAC97621B730BE4
:10C21000840B950B62966CAF7DAF8EAF9FAF62972C
:10C220008DE490E0A096AEADBFADA097A89FF001C1
:10C23000A99FF00DB89FF00D1124E754F74F6296B7
:10C240002CAD3DAD4EAD5FAD629724833583468303
:10C25000578357FF0DC0DA01C901B095A09590959D
:10C2600081959F4FAF4FBF4F84839583A683B7833C
:10C270004091B1085091B2086091B3087091B40830
:10C280002E964CAF5DAF6EAF7FAF2E97A8968CAD5C
:10C290009DADAEADBFADA897841B950BA60BB70B9C
:10C2A0002A968CAF9DAFAEAFBFAF2A978DE490E0DA
:10C2B000A096AEADBFADA097A89FF001A99FF00DCD
:10C2C000B89FF00D1124E754F74F2A962CAD3DADE1
:10C2D0004EAD5FAD2A97208731874287538757FF3E
:10C2E0000DC0DA01C901B095A095909581959F4F39
:10C2F000AF4FBF4F80879187A287B3872090B50843
:10C300003090B6084090B7085090B808A4964CAD4D
:10C310005DAD6EAD7FADA4974219530964097509EF
:10C320004AA75BA76CA77DA7E0913E02F0913F0270
:10C33000CB01BA0197FF07C09095809570956195E4
:10C340007F4F8F4F9F4F9F01442737FD4095542FBC
:10C350000E94297824E630E040E050E00E947D7899
:10C360008DE490E0A0966EAD7FADA097689FF00140
:10C37000699FF00D789FF00D1124E754F74FDF010E
:10C380001C96248711963C93119712964C93129702
:10C3900013965C936080718082809380A480B580C6
:10C3A000C680D780E084F18402851385C901DA0153
:10C3B0008E159F05A007B10714F4D801C7018A158F
:10C3C0009B05AC05BD0514F4D601C5019C01AD016A
:10C3D00086159705A805B90514F4A40193018DE409
:10C3E00090E0A096AEADBFADA097A89FB001A99F69
:10C3F000700DB89F700D11246754774FFB01208B8F
:10C40000318B428B538B263031054105510510F499
:10C410000C943E6BE85BFF4F8091780690E0A0E0C3
:10C42000B0E080839183A283B383DB0190961C925A
:10C43000E0962CAD3DAD4EAD5FADE0976E968CAD08
:10C440009DADAEADBFAD6E97281739074A075B07A4
:10C4500024F481E0DB0190968C93AC962CAD3DAD3D
:10C460004EAD5FADAC9766966CAD7DAD8EAD9FADBC
:10C470006697261737074807590794F48DE490E02C
:10C48000A096AEADBFADA097A89FF001A99FF00DFB
:10C49000B89FF00D1124E754F74F80A1826080A36C
:10C4A000A8962CAD3DAD4EAD5FADA8972E966CAD68
:10C4B0007DAD8EAD9FAD2E972617370748075907DC
:10C4C00094F48DE490E0A096AEADBFADA097A89F88
:10C4D000F001A99FF00DB89FF00D1124E754F74F1C
:10C4E00080A1846080A3A4962CAD3DAD4EAD5FAD20
:10C4F000A497221533054405550594F48DE490E086
:10C50000A0964EAD5FADA097489FF001499FF00DFA
:10C51000589FF00D1124E754F74F80A1886080A345
:10C520008DE490E0A0966EAD7FADA097689FF0017E
:10C53000699FF00D789FF00D1124E754F74FE296B4
:10C54000AEADBFADE2978C9181A320813181428154
:10C55000538126962CAF3DAF4EAF5FAF2697211586
:10C5600031054105510509F077988DE490E0A096DA
:10C570004EAD5FADA097489FF001499FF00D589FC9
:10C58000F00D1124E754F74F6481758186819781FE
:10C5900022966CAF7DAF8EAF9FAF2297611571056C
:10C5A0008105910509F076988DE490E0A096AEADF6
:10C5B000BFADA097A89FF001A99FF00DB89FF00D07
:10C5C0001124E754F74F608471848284938461144A
:10C5D00071048104910409F047988DE490E0A096DD
:10C5E0002EAD3FADA097289FF001299FF00D389FF9
:10C5F000F00D1124E754F74F84859585A685B785FE
:10C600000097A105B10551F0439820907D08309026
:10C610007E0840907F085090800808C020909508C0
:10C62000309096084090970850909808CE57DF4F6A
:10C630006881C258D040CD57DF4F7881C358D04071
:10C64000CC57DF4F8881C458D040CB57DF4F9881FB
:10C65000C558D040A20191010E94777487FD16C091
:10C66000CE57DF4F8881C258D040CD57DF4F9881D9
:10C67000C358D040CC57DF4FA881C458D040CB57C7
:10C68000DF4FB881C558D0401C012D018091890D24
:10C6900090918A0D482F50E0405F5F4F491B510930
:10C6A0004F7050705FA74EA7BA01882777FD80951D
:10C6B000982F0E9419757B018C0120E030E040E04A
:10C6C00051E40E94777488239CF46EA57FA56230A4
:10C6D000710574F0C201B101A80197010E9457775A
:10C6E00020E030E040E05EE30E9457771B012C0120
:10C6F0006A966CAD7DAD8EAD9FAD6A970E9419753F
:10C7000020915D0830915E0840915F08509160086B
:10C710000E947E74EB966FAFEB97EC967FAFEC9731
:10C72000ED968FAFED97EE969FAFEE97AC01CB01F4
:10C73000DA018A839B83AC83BD8362966CAD7DAD49
:10C740008EAD9FAD62970E9419752091610830915E
:10C75000620840916308509164080E947E74E796D5
:10C760006FAFE797E8967FAFE897E9968FAFE997C5
:10C77000EA969FAFEA97AC01CB01DA018E839F83E3
:10C78000A887B9872A966CAD7DAD8EAD9FAD2A97EF
:10C790000E941975209165083091660840916708DC
:10C7A000509168080E947E74E3966FAFE397E49619
:10C7B0007FAFE497E5968FAFE597E6969FAFE69754
:10C7C000AC01CB01DA018A879B87AC87BD87E090FB
:10C7D0003E02F0903F026AA57BA58CA59DA50E9414
:10C7E00019752091690830916A0840916B08509141
:10C7F0006C080E947E745B016C010027F7FC0095B9
:10C80000102FC801B7010E9419759B01AC01C60128
:10C81000B5010E94577720E030E048EC52E40E94D6
:10C820007E747B018C016E877F87888B998B26961F
:10C830008CAD9DADAEADBFAD26970097A105B105FE
:10C8400091F522962CAD3DAD4EAD5FAD22972115F1
:10C8500031054105510539F56114710481049104D4
:10C8600011F5C801B70120E030E040E050E00E943F
:10C870008576181624F017FB109517F910958DE49E
:10C8800090E0A0964EAD5FADA097489FF001499F04
:10C89000F00D589FF00D1124E754F74FE6A6F7A6C8
:10C8A00000AB11AB55C0EB962FADEB97EC963FADBF
:10C8B000EC97ED964FADED97EE965FADEE97B90123
:10C8C000CA010E940E783B014C01E7962FADE79715
:10C8D000E8963FADE897E9964FADE997EA965FADE8
:10C8E000EA97B901CA010E940E785B016C01E396D8
:10C8F0002FADE397E4963FADE497E5964FADE5970E
:10C90000E6965FADE697B901CA010E940E787B01F9
:10C910008C01C401B301A60195010E949E73A80178
:10C9200097010E949E730E94C4772DE430E0A09688
:10C93000AEADBFADA097A29FF001A39FF00DB29F37
:10C94000F00D1124E754F74F66A777A780AB91ABA2
:10C950008DE490E0A096EEADFFADA097E89F60015A
:10C96000E99FD00CF89FD00C112429EB38E0C20EBF
:10C97000D31ED6019E96ED90FD900D911C91D197FE
:10C9800060E070E080E89FE3A80197010E947E7458
:10C990009B01AC01C201B1010E9457774B015C01C0
:10C9A000C801B701A50194010E945777F60162A35F
:10C9B00073A384A395A360897189828993890E9456
:10C9C0001775A50194010E9457770E9464740E9414
:10C9D000EB74D601D8966D937D938D939C93DB97E2
:10C9E000EE24FF2442E1642E712C6C0E7D1E32E099
:10C9F000C32ED12CCC0EDD1E83010E0D1F1DF601A2
:10CA0000EE0DFF1D6081718182819381A5019401EA
:10CA10000E945777F801608371838283938324E0B7
:10CA200030E0E20EF31E30E1E316F10429F70F2E99
:10CA3000F0E06F2EF0E07F2EF0E88F2EFFE39F2EC8
:10CA4000F02D4424552422E1222E312C2C0E3D1EA3
:10CA5000F101E40DF51DE080F18002811381C80130
:10CA6000B70120E030E040E050E00E9485761816E3
:10CA70001CF4C801B70103C0C801B7019058F20106
:10CA8000E35BF74FA080B180C280D380A6019501FF
:10CA90000E948576181694F5C801B70120E030E0B1
:10CAA00040E050E00E94857618161CF4A80197011A
:10CAB00003C0A80197015058C601B5010E947E74B9
:10CAC0009B01AC01C401B3010E94777487FD16C0BD
:10CAD000C801B70120E030E040E050E00E948576D8
:10CAE000181624F017FB109517F91095C601B5011B
:10CAF000A80197010E947E743B014C0144E050E084
:10CB0000440E551E50E14516510409F0A1CFC40151
:10CB1000B30120E030E040E85FE30E9477748823AF
:10CB20000CF0B2C04424552492E1292E312C2C0E55
:10CB30003D1EF101E40DF51DE080F18002811381BD
:10CB4000C801B70120E030E040E050E00E94857667
:10CB500018161CF4C801B70103C0C801B7019058EA
:10CB6000F201E35BF74FA080B180C280D380A601C1
:10CB700095010E948576181694F5C801B70120E04A
:10CB800030E040E050E00E94857618161CF4A801C1
:10CB9000970103C0A80197015058C601B5010E9432
:10CBA0007E749B01AC01C401B3010E94777487FDC0
:10CBB00016C0C801B70120E030E040E050E00E941C
:10CBC0008576181624F017FB109517F91095C601F5
:10CBD000B501A80197010E947E743B014C0164E0FD
:10CBE00070E0460E571E70E14716510409F0A1CFC0
:10CBF0008E010E5E1F4F82E2E82EF12CEC0EFD1E20
:10CC0000D8016D917D918D919C91A40193010E9419
:10CC10005777F80161937193819391938F01EE158A
:10CC2000FF0571F78DE490E0A0962EAD3FADA09783
:10CC3000289F8001299F100D389F100D1124075443
:10CC4000174FD80192966D917D918D919C919597FA
:10CC5000A40193010E945777F80162A373A384A3F0
:10CC600095A360AD71AD82AD93AD0E941775A4011F
:10CC700093010E9457770E94EB74D801D8966D9368
:10CC80007D938D939C93DB978DE490E0A096EEAD21
:10CC9000FFADA097E89F8001E99F100DF89F100D50
:10CCA00011240754174FD80150966D917D918D91A5
:10CCB0009C9153970E941775F80126A537A540A9A6
:10CCC00051A90E947E741B012C01F8018081918181
:10CCD000A281B3810097A105B10549F584819581B1
:10CCE000A681B7810097A105B10509F580859185D9
:10CCF000A285B3850097A105B105C9F4C201B101B0
:10CD000020918508309186084091870850918808C5
:10CD10000E9457770E9464740C5B1F4F0E94EB7453
:10CD2000D8016D937D938D939C93139771C1C2012C
:10CD3000B10120918108309182084091830850917F
:10CD400084080E9457770E9464740E94EB742DE45B
:10CD500030E0A096EEADFFADA097E29F6001E39FAB
:10CD6000D00CF29FD00C112429EB38E0C20ED31E58
:10CD7000B4E46B2E712C6C0C7D1CD3016D937D93F0
:10CD80008D939C9313978090990890909A08A09007
:10CD90009B08B0909C080E9417757B018C01F601DE
:10CDA00060817181828193810E9419759B01AC0120
:10CDB000C801B7010E9457777B018C01D6015096BC
:10CDC0006D917D918D919C9153970E9417759B0158
:10CDD000AC01C801B7010E947E747B018C01C501C2
:10CDE000B4010E9417759B01AC01C801B7010E94F4
:10CDF000857618162CF4F30180829182A282B38288
:10CE000080909D0890909E08A0909F08B090A008E8
:10CE10008DE490E0A0962EAD3FADA097289F6001D5
:10CE2000299FD00C389FD00C112449EB58E0C40E38
:10CE3000D51EA4E46A2E712C6C0C7D1CD3016D915F
:10CE40007D918D919C910E9417757B018C01F6015B
:10CE500064817581868197810E9419759B01AC015F
:10CE6000C801B7010E9457777B018C01D60150960B
:10CE70006D917D918D919C9153970E9417759B01A7
:10CE8000AC01C801B7010E947E747B018C01C50111
:10CE9000B4010E9417759B01AC01C801B7010E9443
:10CEA000857618162CF4F30180829182A282B382D7
:10CEB0008090A5089090A608A090A708B090A80818
:10CEC0008DE490E0A0962EAD3FADA097289F600125
:10CED000299FD00C389FD00C112449EB58E0C40E88
:10CEE000D51EF4E46F2E712C6C0C7D1CD3016D915A
:10CEF0007D918D919C910E9417757B018C01F601AB
:10CF000064857585868597850E9419759B01AC019E
:10CF1000C801B7010E9457777B018C01D60150965A
:10CF20006D917D918D919C9153970E9417759B01F6
:10CF3000AC01C801B7010E947E747B018C01C50160
:10CF4000B4010E9417759B01AC01C801B7010E9492
:10CF5000857618162CF4F30180829182A282B38226
:10CF60008090A1089090A208A090A308B090A40877
:10CF70008DE490E0A0962EAD3FADA097289F600174
:10CF8000299FD00C389FD00C112449EB58E0C40ED7
:10CF9000D51EE4E46E2E712C6C0C7D1CD3016D91BA
:10CFA0007D918D919C910E9417757B018C01F601FA
:10CFB00060857185828593850E9419759B01AC01FE
:10CFC000C801B7010E9457777B018C01D6015096AA
:10CFD0006D917D918D919C9153970E9417759B0146
:10CFE000AC01C801B7010E947E747B018C01C501B0
:10CFF000B4010E9417759B01AC01C801B7010E94E2
:10D00000857618162CF4F30180829182A282B38275
:10D010008DE490E0A0962EAD3FADA097289F6001D3
:10D02000299FD00C389FD00C112449EB58E0C40E36
:10D03000D51EF601EC5BFF4F608171818281938187
:10D040000E9417757B018C01A20191010E947E74E0
:10D05000D601D2966D937D938D939C93D597C801FD
:10D06000B7012DEB37E346E051E40E9457770E9469
:10D07000E674F601648F758F868F978F20918908EB
:10D0800030918A0840918B0850918C082AAF3BAFB1
:10D090004CAF5DAF4A8D5B8D6C8D7D8D4EA35FA3D4
:10D0A00068A779A7CB01BA0120E030E040E050E06A
:10D0B0000E94857618162CF4EEA0FFA008A519A5ED
:10D0C00008C0EEA0FFA008A519A517FB109517F939
:10D0D000109560918D0870918E0880918F089091C5
:10D0E00090086EAB7FAB88AF99AF20E030E040E0B6
:10D0F0005FE30E9457775B016C01C801B701A6018D
:10D1000095010E948576181664F06AAD7BAD8CADF2
:10D110009DAD20E030E040E05FE30E9457775B0187
:10D120006C018DE490E0A096AEADBFADA097A89F36
:10D13000F001A99FF00DB89FF00D1124E754F74FAF
:10D14000B2A1EF96BFAFEF9723A1C158DF4F28835D
:10D15000CF57D04034A1C058DF4F3883C058D0409B
:10D1600045A1CF57DF4F4883C158D040C601B50114
:10D170002B2FC158DF4F3881CF57D040C058DF4FD9
:10D180004881C058D040CF57DF4F5881C158D04058
:10D190000E94777487FD14C0EF968FADEF97C1584A
:10D1A000DF4F9881CF57D040C058DF4FA881C0587B
:10D1B000D040CF57DF4FB881C158D0405C016D01DE
:10D1C0006E8D7F8D88A199A16AA37BA38CA39DA35B
:10D1D00020E030E040E050E00E94857618162CF404
:10D1E000EAA0FBA00CA11DA108C0EAA0FBA00CA115
:10D1F0001DA117FB109517F910958091910890913A
:10D200009208A0919308B09194088AAB9BABACAB09
:10D21000BDABBC01CD0120E030E040E05FE30E9407
:10D2200057773B014C01C801B701A40193010E944B
:10D230008576181644F4C601B501A40193010E9435
:10D240007774882314F435014601AEA5BFA5129763
:10D250000CF40FC160918C0D70918D0D80918E0D2D
:10D2600090918F0D20E030E040E050E00E94857604
:10D2700018160CF0FEC0A090900DB090910DC090CB
:10D28000920DD090930D6A897B898C899D89A60126
:10D2900095010E949D739B01AC010E9457777B0111
:10D2A0008C012090940D3090950D4090960D5090EB
:10D2B000970D6E897F89888D998DA20191010E94B9
:10D2C0009D739B01AC010E9457779B01AC01C80183
:10D2D000B7010E949E730E94C4777B018C01C60136
:10D2E000B50120E030E040E050E00E9477748823F0
:10D2F00051F4C201B10120E030E040E050E00E9472
:10D3000077748823A1F0EF968FADEF97C158DF4F68
:10D310009881CF57D040C058DF4FA881C058D04027
:10D32000CF57DF4FB881C158D0403C014D01C801F3
:10D33000B7012AAD3BAD4CAD5DAD0E9485761816A8
:10D3400084F46AAD7BAD8CAD9DADA80197010E94C0
:10D350007E749B01AC01C401B3010E9457773B016D
:10D360004C016EA17FA188A599A52091980D3091BF
:10D37000990D40919A0D50919B0D0E949D737B01D8
:10D380008C0120E030E040E050E00E9485761816E5
:10D390001CF4C801B70103C0C801B70190582EA9F9
:10D3A0003FA948AD59AD0E9485761816F4F4C8011E
:10D3B000B70120E030E040E050E00E94857618168A
:10D3C00024F017FB109517F910956EA97FA988AD69
:10D3D00099ADA80197010E947E749B01AC01C40124
:10D3E000B3010E9457773B014C016AA17BA18CA13C
:10D3F0009DA120919C0D30919D0D40919E0D5091CD
:10D400009F0D0E949D737B018C0120E030E040E085
:10D4100050E00E94857618161CF4C801B70103C0BD
:10D42000C801B70190582AA93BA94CA95DA90E943F
:10D4300085761816F4F4C801B70120E030E040E02A
:10D4400050E00E948576181624F017FB109517F906
:10D4500010956AA97BA98CA99DA9A80197010E9492
:10D460007E749B01AC01C401B3010E9457773B015C
:10D470004C018DE490E0A096EEADFFADA097E89F43
:10D480008001E99F100DF89F100D11240754174FCC
:10D49000D8019A966D927D928D929C929D97D2968C
:10D4A0006D917D918D919C91D597905820E030E0C1
:10D4B00040E050EC0E945777F80126A537A540A917
:10D4C00051A90E94577720E030E040E850E40E94E4
:10D4D0009E730E94C477F62EE72ED82EC92EC40163
:10D4E000B3012F2D3E2D4D2D5C2D0E94777487FDAD
:10D4F00006C08F2D9E2DAD2DBC2D3C014D018DE420
:10D5000090E0A0962EAD3FADA097289F8001299F67
:10D51000100D389F100D11240754174FD8019696FF
:10D520006D927D928D929C92999792966D917D913C
:10D530008D919C9195972F2D3E2D4D2D5C2D0E9408
:10D540007774181624F081E0F80187AB03C0D80186
:10D55000D7961C928DE490E0A0962EAD3FADA0979B
:10D56000289FF001299FF00D389FF00D1124E754FA
:10D57000F74F81E086ABA0E9BDE0FE01729680E145
:10D5800001900D928150E1F78DE490E0A0964EADB0
:10D590005FADA097489F6001499FD00C589FD00C69
:10D5A000112469EB78E0C60ED71ED6019296ED9055
:10D5B000FD900D911C919597E0928C0DF0928D0D40
:10D5C00000938E0D10938F0D96966D917D918D9198
:10D5D0009C919997A80197010E947E744B015C0170
:10D5E00060E070E080E090E4A80197010E947E7402
:10D5F0008B019C01C601B501A4010E94835CB8A9FE
:10D60000B093890DA4962CAD3DAD4EAD5FADA49702
:10D610002093B5083093B6084093B7085093B808E4
:10D62000A8964CAD5DAD6EAD7FADA8974093B108A7
:10D630005093B2086093B3087093B408AC966CAD85
:10D640007DAD8EAD9FADAC976093AD087093AE0885
:10D650008093AF089093B008E0968CAD9DADAEADD1
:10D66000BFADE0978093A9089093AA08A093AB0858
:10D67000B093AC080E940B5F0E94A31ACB57DF4FF8
:10D680000FB6F894DEBF0FBECDBFCF91DF911F91D3
:10D690000F91FF90EF90DF90CF90BF90AF909F9051
:10D6A0008F907F906F905F904F903F902F90089554
:10D6B000DB010D900020E9F71197A61BB70B03962D
:10D6C000AD010C94A955DF93CF930F92CDB7DEB780
:10D6D00069830396BE016F5F7F4F41E050E00E9477
:10D6E000A9550F90CF91DF9108958E3270F4EAE53D
:10D6F000FFE0880FE80FF11D9591E491F0E02FB75E
:10D70000F8948181892B81832FBF0895002039F0FF
:10D7100000C0EE3250F4EE0FEA56F4490994EE32AE
:10D7200020F4EE0FEE50F44909940895589AB6C0CB
:10D73000599AD0C05A9A08955B9A08955C9A0895B0
:10D740005D9A08955E9A08955F9A0895709A089573
:10D75000719A0895409A0895419A0895429A0895B9
:10D76000439A0895449AC8C0459AC0C0469AB8C022
:10D77000479A0895769A0895779A0895289A089571
:10D78000299A08952A9A08952B9A08952C9A9CC054
:10D790002D9A88C02E9A8CC02F9A90C0109A089506
:10D7A000119A0895129A0895139A0895149A089553
:10D7B000159A0895169A0895179A0895749A0895D7
:10D7C000759A0895889A0895899A08958A9A08956D
:10D7D0008B9A08958C9A08958D9A08958E9A08953B
:10D7E0008F9A089558985AC0599874C05A980895B5
:10D7F0005B9808955C9808955D9808955E980895E3
:10D800005F980895709808957198089540980895C4
:10D8100041980895429808954398089544986CC09B
:10D82000459864C046985CC04798089576980895D6
:10D830007798089528980895299808952A98089522
:10D840002B9808952C9840C02D982CC02E9830C04D
:10D850002F9834C01098089511980895129808953B
:10D860001398089514980895159808951698089592
:10D87000179808957498089575980895889808954C
:10D88000899808958A9808958B9808958C9808959A
:10D890008D9808958E9808958F980895E4B5EF7D3A
:10D8A000E4BD0895E0918000EF77E0938000089553
:10D8B000E0918000EF7DE09380000895E09180008A
:10D8C000E77FE09380000895E091B000EF77E09368
:10D8D000B0000895E091B000EF7DE093B0000895AE
:10D8E000E0919000EF77E09390000895E091900030
:10D8F000EF7DE09390000895E0919000E77FE09342
:10D90000900008951DBA109268001CBC10BE1FBA8A
:10D9100010927A0010926E0010926F0010927000B8
:10D92000109271001092C9001092BC0011B814B886
:10D9300017B81AB81DB810BA12B815B818B81BB86D
:10D940001EB811BA0895F89480E29EE40197F1F7A9
:10D9500081E08093E00080E28093D80080E69AEE38
:10D960000197F1F7CFDF0C9400FEFFCFF894CADFE8
:10D9700080E69AEE0197F1F70C940000FFCF8F93A9
:10D980008FB78F938091A80D8D5F8D37D0F48093E2
:10D99000A80D8091A40D8F5F8093A40DD8F0809185
:10D9A000A50D8F4F8093A50DA8F08091A60D8F4FE8
:10D9B0008093A60D78F08091A70D8F4F8093A70DCF
:10D9C00009C08D578093A80D8091A40D8E5F809320
:10D9D000A40D28F78091A00D8C5F8093A00D58F0C6
:10D9E0008091A10D8F4F8093A10D28F08091A20D01
:10D9F0008F4F8093A20D8F918FBF8F9118959B01B0
:10DA0000AC0114D0FB010CC011D06E1B7F0B685E03
:10DA10007340D0F32150304040405040E851FC4F1B
:10DA2000211531054105510579F708950FB6F89490
:10DA300066B515B27091A00D8091A10D9091A20DC7
:10DA40000FBE10FE05C06F3F19F07C5F8F4F9F4FD8
:10DA500011240024660F001C660F001C7029089515
:10DA60001F93CF93DF93182FEB013FDE103109F4A2
:10DA70004FC0113160F4113009F442C01130A8F0E8
:10DA80001E3009F455C01F3009F05CC049C019317F
:10DA9000B9F01A3120F4183109F054C02BC01A31F2
:10DAA000B9F01B3109F04EC01DC0209721F45898E1
:10DAB00084B58F7D03C0C8BD84B5806284BD4AC073
:10DAC000D0938900C093880080918000806807C04F
:10DAD000D0938B00C0938A008091800080628093F5
:10DAE000800038C0D0938D00C0938C00809180005E
:10DAF0008860F5CFC093B3008091B000806805C006
:10DB0000C093B4008091B00080628093B00022C0C6
:10DB1000D0939900C09398008091900080680FC0C6
:10DB2000D0939B00C0939A0080919000806207C0C0
:10DB3000D0939D00C0939C0080919000886080935A
:10DB4000900008C0E12FF0E0C038D10514F4E7DD03
:10DB500001C0DFDDDF91CF911F910895F894E1E6D8
:10DB6000F0E020E82083108283E084BD85BDEEE6EE
:10DB7000F0E080818160808391E09093800082E07A
:10DB8000809381009093B0008093B10090939000B7
:10DB90008093910086E880937A0020937B00109216
:10DBA0007E00A5D378940895FC019FB7F8948091E6
:10DBB000B90D882311F420E010C083E08093E900C0
:10DBC0002091F200222349F48091E80082FF05C0F1
:10DBD00085FD03C08BE68093E8009FBF808591851B
:10DBE00097FD03C02F3F09F02F5F822F90E008952B
:10DBF000CF93DF93EC018885998597FF09C0E88171
:10DC0000F9810680F781E02DCE01099599878887F3
:10DC100088859985DF91CF910895FC012085318514
:10DC200037FD05C08FEF9FEF9187808722C02FB708
:10DC3000F8948091B90D882369F083E08093E9001E
:10DC40009BE68091E80085FD09C082FF03C09093A8
:10DC5000E800F7CF2FBF2FEF3FEF0CC09091F100FE
:10DC60008091E80085FD03C08BE68093E8002FBF1C
:10DC7000292F30E0C9010895FC018091B90D882356
:10DC800071F09FB7F89483E08093E9002BE602C01F
:10DC90002093E8008091E80085FDFACF9FBF8FEFC9
:10DCA0009FEF9187808708956F927F928F929F92C6
:10DCB000AF92BF92CF92DF92EF92FF920F931F939A
:10DCC000CF93DF933C018B018091B90D882329F418
:10DCD00081E0D30112968C9311C03FB7F89484E091
:10DCE0008093E9008091B50D882369F08091E80068
:10DCF00085FD07C03FBF81E0E3018A838824992422
:10DD0000DAC01092B50D8824992474E0A72E60E43F
:10DD1000B62E21EFE22EF12C9AE3C92E83E0D82E05
:10DD2000C5C09091E400915F8091E80085FD19C025
:10DD30003FBF8091E400891731F481E08093B50DF5
:10DD4000F3018283B8C08091B90D882329F481E062
:10DD5000D30112968C93AFC03FB7F894A092E9001C
:10DD6000E3CF8091F2002B2D281B822F90E04817E3
:10DD7000590708F4242F622F70E0E801D701E0E48E
:10DD8000E21BE03428F4EE0FFF27E753F149099432
:10DD900080C089918C9389918C9389918C9389917E
:10DDA0008C9389918C9389918C9389918C9389918F
:10DDB0008C9389918C9389918C9389918C9389917F
:10DDC0008C9389918C9389918C9389918C9389916F
:10DDD0008C9389918C9389918C9389918C9389915F
:10DDE0008C9389918C9389918C9389918C9389914F
:10DDF0008C9389918C9389918C9389918C9389913F
:10DE00008C9389918C9389918C9389918C9389912E
:10DE10008C9389918C9389918C9389918C9389911E
:10DE20008C9389918C9389918C9389918C9389910E
:10DE30008C9389918C9389918C9389918C938991FE
:10DE40008C9389918C9389918C9389918C938991EE
:10DE50008C9389918C9389918C9389918C938991DE
:10DE60008C9389918C9389918C9389918C938991CE
:10DE70008C9389918C9389918C9389918C938991BE
:10DE80008C9389918C9389918C9389918C938991AE
:10DE90008C938E018091E80085FD02C0C092E8005D
:10DEA000461B570B860E971ED092B30D4115510598
:10DEB00009F037CF3FBFC401DF91CF911F910F9180
:10DEC000FF90EF90DF90CF90BF90AF909F908F909A
:10DED0007F906F900895E9EAFDE08AE0DF011D92EE
:10DEE0008A95E9F71092AB0D88EE93E0A0E0B0E0E0
:10DEF0008093AC0D9093AD0DA093AE0DB093AF0D8C
:10DF00001092B00D80ED92E09093AA0D8093A90D30
:10DF100008952FEF3FEFFC0131872087E8D10FB63E
:10DF2000F8948091A40D9091A50DA091A60DB091AB
:10DF3000A70D0FBEAC018091B90D882329F068ECC4
:10DF400070E080E090E05BCD8091BA0D882309F10C
:10DF50000FB6F8948091A40D9091A50DA091A60DF7
:10DF6000B091A70D0FBE9C0110C00FB6F894809120
:10DF7000A40D9091A50DA091A60DB091A70D0FBE77
:10DF8000821B930B8B3F9105A8F48091BA0D8823D7
:10DF900061F70FB6F8948091A40D9091A50DA09112
:10DFA000A60DB091A70D0FBE841B950B855C994003
:10DFB00008F4C1CF0895D2DD0E94994E0E941B4EF5
:10DFC000FDCFCF92DF92EF92FF920F931F93CF93EB
:10DFD000DF937C016B018A01C0E0D0E00FC0D60165
:10DFE0006D916D01D701ED91FC910190F081E02DD3
:10DFF000C7010995C80FD91F01501040011511051F
:10E0000071F7CE01DF91CF911F910F91FF90EF90AB
:10E01000DF90CF900895DF93CF9300D0CDB7DEB7D8
:10E02000DC018DE089838AE08A83ED91FC91119770
:10E030000280F381E02DCD01BE016F5F7F4F42E092
:10E0400050E009950F900F90CF91DF9108954F9276
:10E050005F926F927F928F929F92AF92BF92CF9278
:10E06000DF92EF92FF920F931F93DF93CF93CDB781
:10E07000DEB7A1970FB6F894DEBF0FBECDBF3C014F
:10E080006A017B01222349F4DC01ED91FC910190AE
:10E09000F081E02D642F09954EC0213009F42AE06B
:10E0A000C114D104E104F10421F480E389A310E256
:10E0B00027C010E2822E9924AA24BB242E010894A2
:10E0C000411C511CC701B601A5019401F4D76A3067
:10E0D00010F4605D01C0695CF201E10FF11D608325
:10E0E000C701B601A5019401E6D7C901DA016C01A7
:10E0F0007D01C114D104E104F10411F01150E2CF0B
:10E10000002331F01150FE01E10FF11D8DE28183FA
:10E11000812F90E0D301ED91FC91BE016F5F7F4FA5
:10E12000680F791F41E250E0481B590B0280F381D0
:10E13000E02DC3010995A1960FB6F894DEBF0FBE7E
:10E14000CDBFCF91DF911F910F91FF90EF90DF90A6
:10E15000CF90BF90AF909F908F907F906F905F9087
:10E160004F9008950F9377FD02C000E008C07095AE
:10E170006095509541955F4F6F4F7F4F0DE22AE0BC
:10E1800066DF0F9108953F924F925F926F927F9258
:10E190008F929F92AF92BF92CF92DF92EF92FF92B7
:10E1A0000F931F93DF93CF93CDB7DEB728970FB6AA
:10E1B000F894DEBF0FBECDBF3C017A018B01522E19
:10E1C000CB01BA0120E030E040E050E090D387FD81
:10E1D00002C0442406C017FB109517F9109544247B
:10E1E000439420E030E040E05FE3DD240AC0CA0150
:10E1F000B9012DEC3CEC4CEC5DE359D69B01AC0134
:10E20000D394D514A0F3C801B70198D24B015C0197
:10E21000E2D36B017C01C301B701A6012AE0042D02
:10E2200016DF482E392E552009F447C0C701B60124
:10E23000FED39B01AC01C501B4017FD29B01AC01AF
:10E240008EE28983D52C87E0851510F487E0D82EDF
:10E25000BD2CCC24C3944E010894811C911C1FC07A
:10E26000CA01B90120E030E040E251E420D67B0150
:10E270008C01B1D3F401EC0DF11D605D608360533E
:10E28000C39470E0882777FD8095982FD2D39B01A7
:10E29000AC01C801B70151D29B01AC01BA94BB20BB
:10E2A000F9F6D301ED91FC91D3940280F381E02D36
:10E2B000C301B4014D2D50E00995842D932D28966E
:10E2C0000FB6F894DEBF0FBECDBFCF91DF911F9187
:10E2D0000F91FF90EF90DF90CF90BF90AF909F9005
:10E2E0008F907F906F905F904F903F9008958091B6
:10E2F000D80087FF02C085FF1BC081E88093D7004C
:10E3000080EA8093D80086E189BD09B400FEFDCF84
:10E3100080E98093D8001092E0001092B90D10921D
:10E32000BA0D1092B60D1092E1008DE08093E200DC
:10E3300008951F920F920FB60F920BB60F921124F1
:10E340002F933F934F935F936F937F938F939F93FD
:10E35000AF93BF93EF93FF931092E9008091E80091
:10E3600083FF57C12091F1009091F1004091F1009D
:10E370005091F1006091F1007091F100A091F100D5
:10E38000B091F10082EF8093E800963009F044C02C
:10E39000E6ECFFE020E0859195918417950711F058
:10E3A000359617C0859195918617970711F033968A
:10E3B00010C0259135914491CD01AF3FB10519F0C1
:10E3C00010F08FEF90E0841708F4482FF9015EEF0A
:10E3D00004C02F5F2630F9F61CC18091E800282F79
:10E3E00030E0C90185709070892BB9F322FD14C10A
:10E3F000242F413208F020E2922F04C085918093AF
:10E40000F10091509923D1F7421B5093E800442327
:10E4100021F7203211F300C1953061F48EEF809323
:10E42000E8008091E80080FFFCCF842F8068809313
:10E43000E300F2C0993009F5222309F0EAC04093C5
:10E44000B90D1092B60D1092B30D8EEF8093E800C7
:10E45000E0EFFFE091E09093E90085918093EB007D
:10E46000882331F085918093EC0085918093ED00B5
:10E470009F5F953081F78EE1C7C0983061F42038F6
:10E4800009F0C7C08091E80080FFFCCF8091B90DF2
:10E490008093F10096C09132A9F4213A09F0B9C0F5
:10E4A0008091E80080FFFCCF20E030E0F901E55BDF
:10E4B000FD4F80818093F1002F5F3F4F2730310562
:10E4C000A9F77FC0903209F04BC0213209F0A1C0FA
:10E4D0008091E80082FFFCCF20E030E0F901E55BAD
:10E4E000FD4F8091F10080832F5F3F4F2730310532
:10E4F000A9F78BEF8093E8008EEF8093E80080917E
:10E500004B0290914C02A0914D02B0914E02863880
:10E510009105A105B10519F48FE08093B40D8091A8
:10E520004B0290914C02A0914D02B0914E0286395F
:10E530009105A105B10509F06FC084E08093E90061
:10E540002FEF06C02093E8008091E80082FDFCCF09
:10E550008091EE0090E083709070892B99F706DA35
:10E56000923251F4213209F054C04093B60D80919B
:10E57000E80080FFFCCF25C0933241F4213209F03E
:10E5800048C08091E80080FFFCCF1BC09923E9F4CC
:10E590008091E80080FFFCCF223811F080E00DC0B0
:10E5A0006093E9008091EB0090E025E096958795D7
:10E5B0002A95E1F781701092E9008093F1001092A2
:10E5C000F1008EEF8093E80027C0913011F0933076
:10E5D00001F52230F1F4452BE1F4262F2F77822F1D
:10E5E00081508630B0F48EEF8093E8002093E900EC
:10E5F000933079F089E18093EB0081E090E002C0F4
:10E60000880F991F2A95E2F78093EA001092EA009A
:10E6100003C081E28093EB00FF91EF91BF91AF9136
:10E620009F918F917F916F915F914F913F912F912A
:10E630000F900BBE0F900FBE0F901F9018951F925A
:10E640000F920FB60F920BB60F9211242F933F9398
:10E650004F935F936F937F938F939F93AF93BF93EA
:10E66000EF93FF938091E1001092E100982F83FFD8
:10E6700011C01092E90081E08093EB001092EC0051
:10E6800082E28093ED0088E08093F0001092B90D53
:10E690001092B60D92FF1DC08091B90D8823C9F06C
:10E6A0008091B30D882359F081508093B30D882356
:10E6B00031F484E08093E9008AE38093E80080915C
:10E6C000B40D882331F081508093B40D882309F470
:10E6D0003AD990FF0CC080E18093E2001092B90D0E
:10E6E00081E08093BA0D80EA8093D80019BC8091B4
:10E6F000BA0D882379F094FF0DC086E189BD09B475
:10E7000000FEFDCF80E98093D8008DE08093E20089
:10E710001092BA0DFF91EF91BF91AF919F918F91A0
:10E720007F916F915F914F913F912F910F900BBE11
:10E730000F900FBE0F901F9018955058BB27AA2717
:10E740000ED081C241D230F046D220F031F49F3F4A
:10E7500011F41EF411C20EF4E095E7FBDCC1E92FC1
:10E7600094D280F3BA17620773078407950718F0ED
:10E7700071F49EF5C3C20EF4E0950B2EBA2FA02DB6
:10E780000B01B90190010C01CA01A0011124FF275E
:10E79000591B99F0593F50F4503E68F11A16F04059
:10E7A000A22F232F342F4427585FF3CF4695379558
:10E7B0002795A795F0405395C9F77EF41F16BA0B1D
:10E7C000620B730B840BBAF09150A1F0FF0FBB1FCB
:10E7D000661F771F881FC2F70EC0BA0F621F731F14
:10E7E000841F48F4879577956795B795F7959E3F71
:10E7F00008F0B3CF9395880F08F09927EE0F9795FF
:10E8000087950895E1D158F080E891E009F49EEFF2
:10E81000E2D128F040E851E059F45EEF09C0ACC104
:10E820006DC2E92FE07831D268F3092E052AC1F3D1
:10E83000261737074807590738F00E2E07F8E02546
:10E8400069F0E025E0640AC0EF6307F8009407FA76
:10E85000DB01B9019D01DC01CA01AD01EF935DD07F
:10E86000F2D10AD05F91552331F02BED3FE049E41E
:10E8700050FD49EC63CF0895DF93DD27B92FBF77B3
:10E8800040E85FE31616170648075B0710F4D92F18
:10E89000A1D29F938F937F936F93C0D3E8E9F0E069
:10E8A0006ED1D1D12F913F914F915F910CD3DD2348
:10E8B00049F09058A2EA2AED3FE049EC5FE3D078B6
:10E8C0005D274DDFDF91BFC102D280F09F3740F45A
:10E8D00091110EF414C260E070E080E89FE30895A7
:10E8E00026F01B16611D711D811D1BC135C1EFD0A6
:10E8F00008F481E0089577D1E395B6C10CD0A3C1A7
:10E900006AD140F061D130F021F45F3F19F003C1CA
:10E910005111F5C131C1B9D198F39923C9F35523E8
:10E92000B1F3951B550BBB27AA2762177307840702
:10E9300038F09F5F5F4F220F331F441FAA1FA9F3B8
:10E9400033D00E2E3AF0E0E830D091505040E695AA
:10E95000001CCAF729D0FE2F27D0660F771F881F0B
:10E96000BB1F261737074807AB07B0E809F0BB0BFA
:10E97000802DBF01FF2793585F4F2AF09E3F51051E
:10E9800068F0C9C0BCC15F3FECF3983EDCF38695EC
:10E9900077956795B795F7959F5FC9F7880F911D94
:10E9A0009695879597F90895E1E0660F771F881F80
:10E9B000BB1F621773078407BA0720F0621B730B33
:10E9C000840BBA0BEE1F88F7E095089504D0689485
:10E9D000B11195C1089561D188F09F5790F0B92F7A
:10E9E0009927B751A0F0D1F0660F771F881F991FA4
:10E9F0001AF0BA95C9F712C0B13081F07FD1B1E0F9
:10EA000008957CC1672F782F8827B85F39F0B93F08
:10EA1000CCF3869577956795B395D9F73EF49095A5
:10EA20008095709561957F4F8F4F9F4F0895E89423
:10EA300009C097FB3EF490958095709561957F4F46
:10EA40008F4F9F4F9923A9F0F92F96E9BB279395F4
:10EA5000F695879577956795B795F111F8CFFAF404
:10EA6000BB0F11F460FF1BC06F5F7F4F8F4F9F4F35
:10EA700016C0882311F096E911C0772321F09EE893
:10EA8000872F762F05C0662371F096E8862F70E0F9
:10EA900060E02AF09A95660F771F881FDAF7880FD3
:10EAA0009695879597F9089512D180F09F3740F495
:10EAB00091110EF024C160E070E080E89FEB0895B2
:10EAC00026F41B16611D711D811D2BC045C0990FB9
:10EAD0000008550FAA0BE0E8FEEF16161706E80728
:10EAE000F907C0F012161306E407F50798F0621B49
:10EAF000730B840B950B39F40A2661F0232B242B1E
:10EB0000252B21F408950A2609F4A140A6958FEF3C
:10EB1000811D811D089597F99F6780E870E060E08E
:10EB20000895882371F4772321F09850872B762F4E
:10EB300007C0662311F499270DC09051862B70E011
:10EB400060E02AF09A95660F771F881FDAF7880F22
:10EB50009695879597F908959F3F49F0915028F42D
:10EB6000869577956795B7959F5F80389F4F880FFB
:10EB70009695879597F908959FEF80EC0895DF9318
:10EB8000CF931F930F93FF92EF92DF927B018C0143
:10EB9000689405C0DA2EEF0196D1FE01E894A591A4
:10EBA0002591359145915591AEF3EF01D8DDFE01E8
:10EBB0009701A801DA9479F7DF90EF90FF900F9119
:10EBC0001F91CF91DF91089500240A94161617061D
:10EBD00018060906089500240A941216130614064E
:10EBE00005060895C9CF59D0E8F3E894EFEFBB27A5
:10EBF0003FE048EC5FE76B3D73078407950708F13A
:10EC0000FF279F57B25A6A4D7F40894CF04032F43B
:10EC1000BE556542704F8643FF4F0894EE1F9150DA
:10EC200030F0BB0F661F771F881FFF1FEBCF9EE7DB
:10EC3000882332F0BB0F661F771F881F9A95C1F794
:10EC40009395E09589CF092E0394000C11F4882345
:10EC500052F0BB0F40F4BF2B11F460FF04C06F5F94
:10EC60007F4F8F4F9F4F0895EF93E0FF06C0A2EABA
:10EC70002AED3FE049EC5FEB72DDE5DF0F90039496
:10EC800001FC9058E5ECF0E0D3C157FD9058440FDB
:10EC9000551F59F05F3F71F04795880F97FB991FFB
:10ECA00061F09F3F79F087950895121613061406B8
:10ECB000551FF2CF4695F1DF08C016161706180645
:10ECC000991FF1CF86957105610508940895E5DFD8
:10ECD000A0F0BEE7B91788F4BB279F3860F416167A
:10ECE000B11D672F782F8827985FF7CF8695779586
:10ECF0006795B11D93959639C8F30895E894BB279D
:10ED000066277727CB0197F90895E1DE08F48FEFA6
:10ED100008955ADF19F05FDF09F02ECFFCCEB9015C
:10ED2000CA011ACF9F775F77B0DF98F39923B9F3C1
:10ED30005523B9F3FF27951758F4E52FE91BED305C
:10ED400070F75E3B10F0F1E41CC09034E0F40AC0B0
:10ED5000E92FE51BED3028F79E3B10F0F1E411C0E0
:10ED6000503488F4F9EA88232AF09A95660F771FC1
:10ED7000881FDAF744232AF05A95220F331F441FC5
:10ED8000DAF79F1B5F1BFF931F930F93FF92EF9286
:10ED900079018A01BB27AB2F9B01AC0196D097016B
:10EDA000A801BF937B018C01AA27BA2FB901CA0120
:10EDB0008CD0AF919701A801EF90FF900F911F9118
:10EDC000CEDC41DFE1D04F9140FF0895552747FD4C
:10EDD000509509C09B01AC0160E070E080E89FE3C2
:10EDE0008DCD99CEB9CE59DFE8F39923D9F3940F9D
:10EDF000511DBBF39150504094F059F0882332F0EC
:10EE0000660F771F881F91505040C1F79E3F5105F4
:10EE100044F7880F911D9695879597F908955F3F60
:10EE2000ACF0983E9CF0BB27869577956795B79593
:10EE300008F4B1609395C1F7BB0F58F711F460FF68
:10EE4000E8CF6F5F7F4F8F4F9F4FE3CF58CF25DFC6
:10EE500058F19E5758F19851A0F0E9F0983020F5FC
:10EE6000092E9927660F771F881F991F0A94D1F7DB
:10EE700012C0062E672F782F8827985F11F4000C98
:10EE800007C0993FB4F38695779567959395D9F721
:10EE9000611D711D811D3EF4909580957095619561
:10EEA0007F4F8F4F9F4F0895689429CF27CF0BD066
:10EEB000CACE8ADE28F08FDE18F0952309F02BCE1B
:10EEC0005BCE11241CCFE1DEA0F3959FD1F3950F0B
:10EED00050E0551F629FF001729FBB27F00DB11DDE
:10EEE000639FAA27F00DB11DAA1F649F6627B00D6E
:10EEF000A11D661F829F2227B00DA11D621F739F57
:10EF0000B00DA11D621F839FA00D611D221F749F64
:10EF10003327A00D611D231F849F600D211D822FAB
:10EF2000762F6A2F11249F5750408AF0E1F08823F2
:10EF30004AF0EE0FFF1FBB1F661F771F881F9150FF
:10EF40005040A9F79E3F510570F0E5CDD8CE5F3F08
:10EF5000ECF3983EDCF3869577956795B795F79532
:10EF6000E7959F5FC1F7FE2B880F911D96958795BA
:10EF700097F908959F9337DE0F9007FCEE5F74CEEC
:10EF800011F40EF4F9CDE8CD88DED0F39923D9F34E
:10EF9000CEF39F57550B87FF44D056959795B0E019
:10EFA00020F4660F771F881FBB1F1F930F93002449
:10EFB0009001A0018001F001A0E80E0F1F1F0A1EA2
:10EFC000511D601B710B8009B50B48F4600F711F58
:10EFD000801DB51F0E1B1F0B0A0A510907C02E0FFB
:10EFE0003F1F4A1F0E0F1F1F0A1E511D660F771F5E
:10EFF000881FBB1FA695F795E795F8F60617170724
:10F0000008065B07211D311D411D0F911F91B9019C
:10F01000842F9158880F9695879508959B01AC0190
:10F0200046CF91505040660F771F881FD2F7089542
:10F030009F938F937F936F93FF93EF939B01AC010B
:10F0400036DFEF91FF919BDD2F913F914F915F91C3
:10F050002ECF629FD001739FF001829FE00DF11DC2
:10F06000649FE00DF11D929FF00D839FF00D749F42
:10F07000F00D659FF00D9927729FB00DE11DF91FEE
:10F08000639FB00DE11DF91FBD01CF01112408954B
:10F0900097FB092E07260AD077FD04D049D006D069
:10F0A00000201AF4709561957F4F0895F6F79095BA
:10F0B00081959F4F0895A1E21A2EAA1BBB1BFD014B
:10F0C0000DC0AA1FBB1FEE1FFF1FA217B307E40747
:10F0D000F50720F0A21BB30BE40BF50B661F771F9F
:10F0E000881F991F1A9469F760957095809590957F
:10F0F0009B01AC01BD01CF01089597FB092E0526A8
:10F100000ED057FD04D0D7DF0AD0001C38F450953C
:10F110004095309521953F4F4F4F5F4F0895F6F73B
:10F1200090958095709561957F4F8F4F9F4F089573
:10F13000AA1BBB1B51E107C0AA1FBB1FA617B7071D
:10F1400010F0A61BB70B881F991F5A95A9F7809539
:10F150009095BC01CD010895EE0FFF1F0590F4912D
:10F16000E02D099491110EC0803219F0895085501C
:10F17000D0F708959111089581548A5108F4805E62
:10F18000855A08959927882708952F923F924F9284
:10F190005F926F927F928F929F92AF92BF92CF9227
:10F1A000DF92EF92FF920F931F93CF93DF93CDB730
:10F1B000DEB7CA1BDB0B0FB6F894DEBF0FBECDBFA8
:10F1C00009942A88398848885F846E847D848C8479
:10F1D0009B84AA84B984C884DF80EE80FD800C8182
:10F1E0001B81AA81B981CE0FD11D0FB6F894DEBF65
:10F1F0000FBECDBFED01089510E1C2EDD0E103C017
:10F20000FE01ACDF2296C43DD107D1F7F894FFCFC1
:10F210004D383420582059205A2045006175746FAC
:10F2200025692E67004D3233202573004D3234009E
:10F230002F0043616E6E6F74206F70656E20737562
:10F240006264697200005374657072617465207441
:10F250006F2068696768203A2000005049442041C7
:10F2600075746F74756E6520737461727400557374
:10F27000696E672044656661756C7420736574748B
:10F28000696E67733A002569206D696E2C202569C7
:10F2900020736563004D31303420496E76616C69AE
:10F2A0006420657874727564657220004D31303564
:10F2B00020496E76616C6964206578747275646546
:10F2C000722000004D31303920496E76616C6964DE
:10F2D00020657874727564657220003F004C2000D0
:10F2E0004820006F6B0020703A0020693A002064CB
:10F2F0003A0020633A005400496E76616C696420DC
:10F30000657874727564657200416374697665200E
:10F3100045787472756465723A20004D3131300061
:10F320004D32390001010101010000F04185F41066
:10F330003E107059440000803FFF3F0100803B4574
:10F3400000803B450000F0430000000064006400C2
:10F3500060EA00000080BB4401BB0D00E10000003A
:10F3600000080000000058595A45000001001C0028
:10F370001D0013002F00FFFF1E001F0012001400CD
:10F38000FFFF2000210011002400FFFFFFFFFFFF0F
:10F390000E001000220023000D000F000300FFFFED
:10F3A000FFFF020028230000282300006400000063
:10F3B000102700000000FA430000FA430000A040BC
:10F3C00000003442B89E2F43B89E2F43E17A9D44FB
:10F3D0009A99BC4200000000636BE16F00000000DE
:0CF3E0002012546ED46D0D6EF86D3C6E62
:00000001FF
